:100000000C942C040C945D040C945D040C945D041D
:100010000C945D040C945D040C945D040C945D04DC
:100020000C945D040C945D040C945D040C945D04CC
:100030000C945D040C945D040C945D040C94885A3B
:100040000C945D040C945D040C945D040C945D04AC
:100050000C945D040C945D040C945D040C94105A93
:100060000C945D040C94E6590C94BC590C945D04FA
:100070000C945D040C945D040C945D040C946E5A15
:100080000C945D040C945D040C945D040C945A5A19
:100090000C9492590C9468590C945D040C945D0472
:1000A0000C945D040C945D040C945D040C945D044C
:1000B0000C945D040C945D040C945D040C945D043C
:1000C0000C945D040C945D040C945D040C943E59F6
:1000D0000C9414590C945D040C945D040C945D0410
:1000E0000C945D0407634236B79BD8A71A3968564B
:1000F00018AEBAAB558C1D3CB7CC5763BD6DEDFD4A
:10010000753EF6177231BF000000803F0800000006
:10011000BE922449123EABAAAA2ABECDCCCC4C3EFC
:1001200000000080BEABAAAAAA3E00000000BF00EB
:100130000000803F0000000000084178D3BB4387E7
:10014000D1133D190E3CC3BD4282AD2B3E68EC82FB
:1001500076BED98FE1A93E4C80EFFFBE01C4FF7F80
:100160003F00000000000C9451070C948F150C9474
:100170001B610C94DB170C9404180C941D180C9440
:1001800073160C949E600C940C130C9449480C94B8
:1001900033070C947B140C946B130C9403160C947F
:1001A00070130C942F160C945D650C94AF0D0C9489
:1001B00047070C94C6160C941E070C945E070C940B
:1001C000E4640C94FC0D0C94FB170C945C130C94DD
:1001D0005D140C948E620C9461130C9401140C94B5
:1001E000BB130C9422060C942B140C9415140C9431
:1001F0004F600C94AF160C94A2130C9490170C94AF
:1002000090110C9467050C9479150C94FC130C94C4
:100210004E140C945F070C94ED160C944D0D0C9439
:1002200038160C94F7130C94E7110C9457130C9494
:1002300062140C945A160C943D070C94B5620C94FD
:10024000B7470C9422180C94AE170C947D160C949E
:1002500059050C94AC130C945F170C9443130C9435
:1002600085140C946D150C9447170C94F40D0C9494
:10027000F2130C943F140C945F160C9467140C94B6
:1002800042160C9463070C9482470C94E2170C946A
:10029000D4130C948C160C943E110C9480650C9421
:1002A00093130C94F2110C94C0130C948E130C94B1
:1002B000F1140C9483150C94DC110C9420130C9401
:1002C00052130C941E140C940B140C94F8610C949F
:1002D00088630C942C070C9405640C9428070C94E8
:1002E00039070C94D1170C94D6170C940F160C9454
:1002F000EF150C942F130C9455640C94D5050C94A5
:1003000020150C9455160C94CC170C9419140C94BD
:100310004C160C94C7150C9448130C94B1130C9400
:1003200003150C94BD160C940C150C9476140C94B7
:1003300010480C9487160C942A630C94B6130C94F2
:1003400036480C9439130C9478640C9444140C942F
:10035000F0040C946C140C9406140C9464160C9415
:1003600028140C9453170C94DB150C947F600C9498
:1003700080140C9498130C94C0640C94D9130C94AE
:1003800045050C94AF610C9455070C942B120C94FA
:1003900034150C9416150C9426180C948E610C943C
:1003A00025130C946B610C94D1470C9430140C946D
:1003B0007B170C94A5150C949B150C9449140C9464
:1003C000F9150C9443150C9430070C9466130C9497
:1003D00009130C9475130C942A130C94B1150C94F6
:1003E0002B150C949D130C94F2170C94E5150C949A
:1003F000C5130C94E8130C94BF600C94C2170C94B2
:100400004B070C9471140C9411130C9469160C94F2
:100410009A170C940D180C9425160C94B8170C947C
:1004200036050C94DE130C941B130C94A4160C9438
:10043000BD150C949A5A0C9491160C944F630C941D
:10044000D20D0C943B170C9459070C94D8620C9461
:100450004D150C9423140C9443070C943A140C94EB
:1004600092470C94A9630C94FA140C9484130C9482
:1004700061150C94A50D0C944D130C947A130C94E7
:1004800034130C9410140C94ED130C949B640C9482
:1004900024070C94A7130C949A160C9416180C9419
:1004A0001B160C9453140C9439150C94A4170C942B
:1004B00036650C94D4610C943E130C94E9170C949B
:1004C0007F130C9489130C94D1150C9457150C942C
:1004D0007C480C946F170C9466170C94CA130C94F8
:1004E000830D0C9487170C9416130C9435140C94EC
:1004F0009B0D0C94E3130C9414170C94B8160C94E5
:10050000CF130C945814000005800F800A001B8044
:100510001E0014001180338036003C003980280012
:100520002D8027802200638066006C00698078003F
:100530007D8077807200500055805F805A004B802C
:100540004E0044004180C380C600CC00C980D80062
:10055000DD80D780D200F000F580FF80FA00EB80CC
:10056000EE00E400E180A000A580AF80AA00BB807F
:10057000BE00B400B180938096009C0099808800F2
:100580008D8087808200838186018C01898198011A
:100590009D8197819201B001B581BF81BA01AB8184
:1005A000AE01A401A181E001E581EF81EA01FB81B7
:1005B000FE01F401F181D381D601DC01D981C801AA
:1005C000CD81C781C201400145814F814A015B81D4
:1005D0005E0154015181738176017C01798168014A
:1005E0006D8167816201238126012C0129813801F7
:1005F0003D8137813201100115811F811A010B8164
:100600000E0104010181038306030C03098318030F
:100610001D8317831203300335833F833A032B83F3
:100620002E0324032183600365836F836A037B8326
:100630007E0374037183538356035C035983480319
:100640004D8347834203C003C583CF83CA03DB8343
:10065000DE03D403D183F383F603FC03F983E803B9
:10066000ED83E783E203A383A603AC03A983B80366
:10067000BD83B783B203900395839F839A038B83D3
:100680008E0384038183800285828F828A029B820B
:100690009E0294029182B382B602BC02B982A80281
:1006A000AD82A782A202E382E602EC02E982F802AE
:1006B000FD82F782F202D002D582DF82DA02CB829B
:1006C000CE02C402C182438246024C0249825802D1
:1006D0005D8257825202700275827F827A026B823B
:1006E0006E0264026182200225822F822A023B82EE
:1006F0003E0234023182138216021C021982080261
:100700000D820782020200002100240027002A0037
:100710002D003000330001010000040107010A012F
:1007200000002200250028002B002E00310034009C
:1007300002010000050108010B0100002000230058
:10074000260029002C002F003200000100000301C8
:100750000601090105050505070508080808020244
:1007600002020A0A0808040404040101010101014B
:1007700001010303030303030303040707070C0C2E
:100780000C0C0C0C0C0C02020202060606060606F5
:1007900006060B0B0B0B0B0B0B0B0A0A0A0A0A0AB9
:1007A00008080707050505040404010210202008B5
:1007B00008102040102040800201020108040201BC
:1007C000010204081020408080402010080402012B
:1007D0008004020180402010080402010804020184
:1007E000010204081020408001020408102040800B
:1007F000040810204080048008100440801020402D
:1008000000000A0B02090C0D0E080703040100008A
:1008100000000000000000000000000000000000D8
:100820000000000000000000000000001211100095
:1008300000000000000000000000000000000000B8
:1008400000000000000000000000000000000000A8
:100850000000000000009A5A11241FBECFEFD1E221
:10086000DEBFCDBF00E00CBF14E0A0E0B2E0EEE5DB
:10087000FAEE00E00BBF02C007900D92A233B10761
:10088000D9F72CE0A2E3B4E001C01D92AF31B2076A
:10089000E1F714E0CCE2D4E000E006C021970109C2
:1008A000802FFE010E940F73CB32D10780E0080732
:1008B000A9F70E94C35B0C942D750C940000CF9394
:1008C000DF93EC018AAD882359F1888D998D892BAE
:1008D00039F12C853D854E855F8560E070E0CB0168
:1008E0000E944C706C877D878E879F872889398905
:1008F0004A895B8960E070E0CB010E944C70688B94
:10090000798B8A8B9B8B2C893D894E895F8960E02E
:1009100070E0CB010E944C706C8B7D8B8E8B9F8B1B
:10092000198E188EDF91CF910895CF92DF92EF92BA
:10093000FF92CF93DF93EC016A017B0160E874E8DA
:100940008EE190E0A70196010E941B7021503109B1
:10095000410951095695479537952795E889F989B1
:1009600082E08083211580E1380798F0E889F989D1
:10097000108260E472E48FE090E0A70196010E948B
:100980001B702150310941095109569547953795FA
:100990002795EC85FD853083EE85FF852083188EB5
:1009A000EC89FD8986E08083EA89FB89808180610A
:1009B0008083EA89FB89808188608083EA89FB895A
:1009C000808180688083EA89FB8980818F7D808334
:1009D000DF91CF91FF90EF90DF90CF900895089531
:1009E000AF92BF92CF92DF92EF92FF920F931F933D
:1009F000CF93DF936C017B018B01040F151FEB017B
:100A00005E01AE18BF08C017D10759F06991D60131
:100A1000ED91FC910190F081E02DC6011995892B93
:100A200079F7C501DF91CF911F910F91FF90EF9062
:100A3000DF90CF90BF90AF900895FC01A089B1895D
:100A40008C91A689B78982FD0FC09C91818D8F5FA3
:100A50008F73228D821749F0A18DAE0FBF2FB11D6C
:100A60005D969C93818F08958C910895FC01538D20
:100A7000448D252F30E0842F90E0821B930B541778
:100A800010F0CF96089501970895FC01918D828D05
:100A9000981761F0A28DAE0FBF2FB11D5D968C919E
:100AA000928D9F5F9F73928F90E008958FEF9FEFDD
:100AB0000895FC01918D828D981731F0828DE80F99
:100AC000F11D858D90E008958FEF9FEF0895FC0153
:100AD000918D228D892F90E0805C9F4F821B910920
:100AE0008F73992708958CEA98E00E94670521E0AA
:100AF000892B09F420E0822F089580E797E00E9477
:100B0000670521E0892B09F420E0822F08958DE00C
:100B100098E00E94670521E0892B09F420E0822FEC
:100B20000895CF93DF93EC01E881F9810680F78186
:100B3000E02D1995EA89FB8980818F7E8083EA897F
:100B4000FB898081877F8083EA89FB8980818F7719
:100B50008083EA89FB8980818F7D80838A8D898F5C
:100B6000DF91CF910895FC01A48DA80FB92FB11D7D
:100B7000A35ABF4F2C91848D90E001968F739927D3
:100B8000848FA689B7892C93A089B1898C918370B1
:100B900080648C93938D848D981306C00288F389AA
:100BA000E02D80818F7D80830895EF92FF920F93D7
:100BB0001F93CF93DF93EC0181E0888F9B8D8C8D09
:100BC00098131AC0E889F989808185FF15C09FB7FD
:100BD000F894EE89FF896083E889F98980818370C0
:100BE000806480839FBF81E090E0DF91CF911F916F
:100BF0000F91FF90EF900895F62E0B8D10E00F5F90
:100C00001F4F0F731127E02E8C8D8E110CC00FB665
:100C100007FCFACFE889F989808185FFF5CFCE01FD
:100C20000E94B305F1CFEB8DEC0FFD2FF11DE35AC0
:100C3000FF4FF0829FB7F8940B8FEA89FB89808180
:100C40008062CFCFCF93DF93EC01888D8823B9F0FA
:100C5000AA89BB89E889F9898C9185FD03C08081C7
:100C600086FD0DC00FB607FCF7CF8C9185FFF2CF44
:100C7000808185FFEDCFCE010E94B305E9CFDF91E2
:100C8000CF9108950F931F93CF93DF9380913807EF
:100C900081116CC0809167068111ADC080917F0584
:100CA000811128C08CEA98E00E946705049714F12E
:100CB0008CEA98E00E944505809326068CEA98E02D
:100CC0000E944505809327068CEA98E00E9445051E
:100CD000809328068CEA98E00E94450580932906B7
:100CE00094E0980F90934E068250823218F581E07E
:100CF00080937F058CEA98E00E946705D0914E06AC
:100D00004D2F4450550B841795070CF474C08091F7
:100D10007F05882309F46FC00AE216E0C4E0CD170E
:100D2000A0F48CEA98E00E944505F80181938F01B8
:100D3000CF5FF5CF8CEA98E00E946705892BD1F24E
:100D40008CEA98E00E944505F5CF83E08093670622
:100D500010927F058CEA98E00E946705892B09F4C0
:100D60004AC08CEA98E00E944505F4CF813009F032
:100D700042C08CEA98E00E94670518161906ACF587
:100D8000D1E08CEA98E00E946705C0917E05892B2E
:100D900061F18CEA98E00E9445054C2F50E0FA0181
:100DA000E052FA4F8083C230E0F02091E10530E05C
:100DB0002D5F3F4F42175307A1F48D3079F4D09344
:100DC000F20510927E058CEA98E00E946705892B57
:100DD000C1F28CEA98E00E944505F5CF1092F20529
:100DE000F0CFCF5FC0937E05CCCF80917E0586305B
:100DF00010F010927E05DF91CF911F910F91089511
:100E00008150823108F05AC0E82FF0E08827E45F73
:100E1000F84F8F4F0C940F732C0730071E072407D1
:100E200028075E07330739073D07430747074B0786
:100E3000510755075E0759075F07630780918000D8
:100E40008F77809380000895809180008F7DF9CF07
:100E500080918000877FF5CF84B58F7784BD08951A
:100E600084B58F7DFBCF8091B0008F778093B000E9
:100E700008958091B0008F7DF9CF809190008F7799
:100E8000809390000895809190008F7DF9CF80919C
:100E90009000877FF5CF8091A0008F778093A0008E
:100EA00008958091A0008F7DF9CF8091A000877F69
:100EB000F5CF809120018F77809320010895809154
:100EC00020018F7DF9CF80912001877FF5CFCF93CF
:100ED000DF93282F30E0F901E050F84F8491F901B9
:100EE000E655F84FD491F901EC5AF84FC491CC2350
:100EF000A1F081110E940007EC2FF0E0EE0FFF1F20
:100F0000E65CF84FA591B491EC91ED2381E090E07F
:100F100009F480E0DF91CF91089580E090E0FACF6E
:100F20001F93CF93DF93282F30E0F901E050F84F63
:100F30008491F901E655F84FD491F901EC5AF84F34
:100F4000C491CC23A9F0162F81110E940007EC2F29
:100F5000F0E0EE0FFF1FE05EF84FA591B4918FB760
:100F6000F894EC91111108C0D095DE23DC938FBF6B
:100F7000DF91CF911F910895DE2BF8CFCF93DF93B0
:100F800090E0FC01E655F84F24918C5A984FFC01F3
:100F900084918823D1F090E0880F991FFC01EA5FCB
:100FA000F84FA591B491FC01E05EF84FC591D49142
:100FB00061110EC09FB7F8948C91E22FE0958E23BB
:100FC0008C932881E223E8839FBFDF91CF9108951E
:100FD0008FB7F894EC91E22BEC938FBFF6CF86534A
:100FE00020917B00982F987F277F922B90937B00F6
:100FF00020911E0290E4299F900111248770822B7A
:1010000080937C0080917A00806480937A00809144
:101010007A0086FDFCCF8091780090917900089548
:101020003FB7F8948091DA059091DB05A091DC053B
:10103000B091DD0526B5A89B05C02F3F19F001969C
:10104000A11DB11D3FBFBA2FA92F982F8827BC0122
:10105000CD01620F711D811D911D43E0660F771F49
:10106000881F991F4A95D1F708958F929F92AF924A
:10107000BF92CF92DF92EF92FF924B015C010E94F0
:1010800010086B017C010E9410086C197D098E0903
:101090009F09683E734081059105A8F321E0821AFB
:1010A0009108A108B10888EEC80E83E0D81EE11CA3
:1010B000F11C81149104A104B10429F7FF90EF9071
:1010C000DF90CF90BF90AF909F908F9008952FB7F3
:1010D000F8946091D6057091D7058091D8059091CC
:1010E000D9052FBF08950F931F93CF938091760555
:1010F00081110DC00E94670860937205709373059B
:10110000809374059093750581E0809376050E9425
:101110006708009172051091730520917405309154
:101120007505601B710B820B930B69357B41810543
:10113000910510F01092710580E797E00E94670515
:1011400018161906A4F5C1E080E797E00E9467052C
:10115000892B69F180E797E00E9445059091710520
:10116000492F50E0FA01E751F94F80839230D8F0CF
:101170002091EA06022E000C330B2D5F3F4F4217E1
:10118000530789F48D3061F4809185068111C093F5
:10119000F706109284061092830610927105D4CF40
:1011A0001092F706FACF9F5F90937105CDCF0E9402
:1011B000670860937205709373058093740590932C
:1011C0007505CF911F910F9108952F923F924F92E5
:1011D0005F926F927F928F929F92AF92BF92CF92C7
:1011E000DF92EF92FF920F931F93CF93DF93CDB7D0
:1011F000DEB72F970FB6F894DEBF0FBECDBF9F8727
:101200008E870E9467086D837E838F839887EE8523
:10121000FF8582A193A1A4A1B5A14D815E816F81BB
:101220007885481B590B6A0B7B0B86A597A5A0A94F
:10123000B1A9481759076A077B0708F426C1048C2F
:10124000F58DE02D80819181A281B38189839A837C
:10125000AB83BC83AE85BF859096ED91FC912981CF
:101260003A814B815C8160817181828193810E948E
:101270004C704B015C01EE85FF8522A533A544A58A
:1012800055A569817A818B819C810E944C706B018C
:101290007C01AE85BF8550962D913D914D915C911D
:1012A0005397C501B4010E94156FEE85FF8526A1F5
:1012B00037A140A551A50E944D702B013C01AE8580
:1012C000BF8596964D925D926D927C929997DB9632
:1012D000BC91B987B11118C0EE85FF85248535858D
:1012E00046855785C701B6010E94156F9B01AC0169
:1012F000C301B2010E944C70AE85BF8596966D9376
:101300007D938D939C939997EE85FF8546A057A07A
:1013100060A471A416A907A930AC21AC212F302FED
:10132000432D522DC301B2010E94617118160CF0B9
:101330008FC0812F902FA32DB22DEE85FF8586A320
:1013400097A3A0A7B1A7F985FF2309F49AC0AE859A
:10135000BF851C962D913D914D915C911F97C501C4
:10136000B4010E94156F4B015C01EE85FF85248955
:10137000358946895789C701B6010E94156F9B01BF
:10138000AC01AE85BF8596966D917D918D919C91B6
:1013900099970E944C70A50194010E944D706B01B9
:1013A0007C019B01AC01612F702F832D922D0E9437
:1013B000AF6E87FD14C0EE85FF8512A903A934A87E
:1013C00025A8212F302F432D522DB601C7010E9491
:1013D000AF6E87FD04C01C2D0D2D3E2C2F2CAE852D
:1013E000BF855E96ED91FC91812F902FA32DB22D9C
:1013F00080839183A283B38389819A81AB81BC81ED
:10140000EE85FF8582A793A7A4A7B5A78D819E81AE
:10141000AF81B88582A393A3A4A3B5A381E02F963F
:101420000FB6F894DEBF0FBECDBFDF91CF911F91F5
:101430000F91FF90EF90DF90CF90BF90AF909F9073
:101440008F907F906F905F904F903F902F90089576
:10145000AE85BF85D2968D919D910D90BC91A02DAA
:101460008A879B87AC87BD879C01AD01C301B20110
:101470000E94AF6E87FF67CF8A859B85AC85BD854F
:101480005CCF812C912C540170CF80E0C8CF8F921B
:101490009F92AF92BF92CF92DF92EF92FF921F93F3
:1014A000CF93DF93EC01162F117061307105A1F518
:1014B0008AAD811131C0EE8DFF8DC080D180E28078
:1014C000F380CEA2DFA2E8A6F9A6EC8DFD8D808187
:1014D0009181A281B3818AA79BA7ACA7BDA78EA843
:1014E0009FA8A8ACB9ACA5019401C701B6010E94A0
:1014F000617118162CF48EA29FA2A8A6B9A60CC0E2
:101500008AA89BA8ACA8BDA8A5019401C701B601F3
:101510000E94AF6E87FDEFCF1AAFDF91CF911F9181
:10152000FF90EF90DF90CF90BF90AF909F908F9003
:1015300008952F923F924F925F926F927F928F9277
:101540009F92AF92BF92CF92DF92EF92FF920F9352
:101550001F93CF93DF93EC016A017B01480159018E
:10156000A9019801CB01B6010E94617187FF4FC0AC
:10157000CAAADBAAECAAFDAA8EAA9FAAA8AEB9AEF7
:101580008AAD882309F443C02E8C3F8CF101408042
:10159000518062807380A3019201C501B8010E944D
:1015A000AF6E87FF1AC0F10180829182A282B3825E
:1015B0008EA09FA0A8A4B9A4CEA8DFA8E8ACF9ACDF
:1015C000A7019601C501B4010E94617118169CF42F
:1015D000CEA2DFA2E8A6F9A61AC0A3019201C70114
:1015E000B6010E94617118161CF7F101C082D18208
:1015F000E282F382DDCFCAA8DBA8ECA8FDA8A70190
:101600009601C501B4010E94AF6E87FDE1CFDF9165
:10161000CF911F910F91FF90EF90DF90CF90BF90EF
:10162000AF909F908F907F906F905F904F903F9082
:101630002F9008954F925F926F927F928F929F9218
:10164000AF92BF92CF92DF92EF92FF920F931F93D0
:10165000CF93DF9300D000D0CDB7DEB79E838D83CC
:101660002A013B014801590120E030E0A901CB01EA
:10167000B2010E94AF6E87FD89C020E030E0A90171
:10168000C501B8010E94AF6E87FD80C020E030E048
:10169000A901C701B6010E94AF6E87FD77C081E046
:1016A000ED81FE81228D338D2130310509F080E0FE
:1016B000ED81FE8183AF4082518262827382848297
:1016C0009582A682B782C086D186E286F38666A519
:1016D00077A580A991A90E94B46E20E030E04AE786
:1016E00054E40E94B97069837A838B839C83ED8173
:1016F000FE8144865586668677869B01AC01C501CE
:10170000B4010E94156F4B015C01ED81FE81808A5E
:10171000918AA28AB38A29813A814B815C81C7016F
:10172000B6010E94B9706B017C01ED81FE81C48A13
:10173000D58AE68AF78A808D918D019739F5A301C4
:10174000920160E070E0CB010E944C70ED81FE815F
:101750006487758786879787A501940160E070E0AC
:10176000CB010E944C70ED81FE81608B718B828B6E
:10177000938BA701960160E070E0CB010E944C7052
:10178000ED81FE81648B758B868B978B26960FB6C9
:10179000F894DEBF0FBECDBFDF91CF911F910F91A7
:1017A000FF90EF90DF90CF90BF90AF909F908F9081
:1017B0007F906F905F904F900895DC014C9111964F
:1017C000EC911197F0E0E627EE0FFF1FEA5FFA4F6A
:1017D0008591949120E0342F282739272D933C932D
:1017E00008956F927F928F929F92AF92BF92CF9205
:1017F000DF92EF92FF920F931F93CF93DF9323E833
:10180000C22E29E0D22EFF24F39434E8A32E39E02F
:10181000B32E47E0642E56E0852E65E0762E74E008
:10182000E72EE3E09E2E8091AA089091AB08DC01A0
:10183000ED91FC910480F581E02D1995892B09F437
:101840004BC28091AA089091AB08DC01ED91FC910C
:101850000680F781E02D1995EC01182F20E030E08B
:1018600040E85FE360914B0970914C0980914D090C
:1018700090914E090E94AF6E8111D2C00E94100853
:1018800020915B0930915C0940915D0950915E099E
:10189000621B730B840B950B2091530930915409F3
:1018A000409155095091560926173707480759079F
:1018B00070F4109251090E94100860935B097093B4
:1018C0005C0980935D0990935E09109267090E94FC
:1018D000100860935B0970935C0980935D09909395
:1018E0005E0980915109823009F45CC040F488237C
:1018F00089F1813009F44BC01092510994CF8330A3
:1019000009F46AC08430C1F780917A098095809388
:101910007A09C0937B0918137EC080918209809355
:101920006D0980936E0980917209909173090297F5
:1019300020914F09D0927D09C0927C09909375093E
:1019400080937409213009F0C4C110926F0910E02E
:1019500000E063C0809167098823A1F0C093690902
:10196000809168098F3F49F41F3F39F4109267094D
:1019700010927A09F092510956CFC09368091092DB
:10198000690951CFC0936809F09267094CCFC093A1
:101990006C0982E08093510980917A09C80FC09345
:1019A0007A0941CFCE0199279093730980937209E8
:1019B00090925109109271091092700920917A0940
:1019C000C20FC0937A09883C91050CF488C110922B
:1019D00051090AE010E08AC1809170099091710963
:1019E000FC01E75BF64FC1AF20917A09C20FC093AB
:1019F0007A09019690937109809370092091720978
:101A000030917309215031098217930708F40BCFE5
:101A1000E092510908CF0DE010E0109251097EC00C
:101A20000E94100820915B0930915C0940915D098A
:101A300050915E09621B730B840B950B2091530927
:101A4000309154094091550950915609261737078E
:101A50004807590720F410925109109267090E9413
:101A6000100860935B0970935C0980935D09909303
:101A70005E09E0915109E83008F03ECFF0E0882798
:101A8000EB5BF24F8F4F0C940F734D0D830D9B0D3D
:101A9000A50DAF0DD20DF40DFC0D809167098230BC
:101AA00048F1C0936A0980916909909168099F3F44
:101AB000D1F48F3FC1F41D3FB1F410926709109229
:101AC0007709109276096FEF86E799E00E94DD0BA7
:101AD0006FEF86E799E00E94DD0B6DEF86E799E0F6
:101AE0000E94DD0B47CF80936809C093690910926B
:101AF0006A0999CEE82FF0E0E75BF64FC78F8F5F5A
:101B00008093670990CE1D3F71F4109251090CE04B
:101B100010E06C2F86E799E00E94DD0B0130110583
:101B200009F481CEE3C0C0936B0982E08093510930
:101B300001E010E0EECFC0936C09909251096C2F38
:101B400086E799E00E94DD0B6ECECE019927909337
:101B5000730980937209E09251096C2FF1CF3C2FE9
:101B600022278091720990917309822B932B909375
:101B70007309809372097092510910927109109241
:101B800070096C2F86E799E00E94DD0B8091720945
:101B9000909173098C3C910508F019CF039708F4D4
:101BA000A1C041CEE0917009F0917109E75BF64F59
:101BB000C1AF6C2F86E799E00E94DD0B8091700920
:101BC0009091710901969093710980937009209109
:101BD000720930917309225031098217930708F472
:101BE00022CE809251091FCEDD27D0937909C09370
:101BF00078096092510917CEDC2FCC2780917809A3
:101C000090917909C82BD92BD0937909C093780981
:101C10004091720950917309E2E8F9E030E020E068
:101C200090E080E084179507F8F482309105A8F0E1
:101C3000DC01A058B64F6C916F3F79F4DC01AE57D0
:101C4000B64F6C91DC01AF57B64F7C917F3F29F4C2
:101C50006D3F19F401962F5F3F4FDC01AE57B64F31
:101C60006C9161930196DECF809172099091730916
:101C7000821B930B909373098093720940917809AA
:101C80005091790920917609309177090EE010E0A2
:101C90004217530709F0C1CE2091820920936D09A4
:101CA0003091830930936E09253551F4B0927D0946
:101CB000A0927C090497909375098093740945CE8E
:101CC000D0927D09C0927C09039790937509809307
:101CD0007409F0926F093BCE01E010E007C0029753
:101CE0000CF0A1CD1092510907E010E0C801DF917E
:101CF000CF911F910F91FF90EF90DF90CF90BF9009
:101D0000AF909F908F907F906F900895AF92BF9209
:101D1000CF92DF92EF92FF920F931F93CF93DF93B7
:101D20001F921F92CDB7DEB7E82EF62E6A01890109
:101D300020E030E040E85FE360914B0970914C098E
:101D400080914D0990914E090E94AF6E81114BC058
:101D50000C3C110508F0E4C08FEF8093670A809374
:101D6000680AE092690AF0926B0AC8010296F80EBE
:101D7000FE0CF6016CE67AE0A601400F511FE41755
:101D8000F50759F02191DB012D93BD019F012150F1
:101D90003109D9012C91F20EF2CF80936A0AF80131
:101DA000E459F54FF094F0828091AA089091AB0825
:101DB000A8014A5F5F4FDC01ED91FC910284F3853D
:101DC000E02D67E67AE0199590E080E00F900F90A3
:101DD000DF91CF911F910F91FF90EF90DF90CF9007
:101DE000BF90AF9008950C3C110508F099C0A80170
:101DF0004D5F5F4F8FEF8093670A8093680A8DEF86
:101E00008093690A10926A0AE0926B0AF0926E0A55
:101E1000F601AFE6BAE09601200F311FE217F30793
:101E200019F081918D93FACFC8010196039708F4B8
:101E300042C0ECE6FAE090E080E030E020E0F12CF7
:101E4000E12C01501109E016F10620F5B9016F5F90
:101E50007F4FD280D901AE57B64FDC92B2E0EB167D
:101E6000F10490F0A081AF3F79F4A181AF3F61F41C
:101E7000D280ADEFDA1208C06E57764FDB01DC92EC
:101E80000196B9016E5F7F4FBFEFEB1AFB0A3196E7
:101E90009B01D9CF009779F0E9E4F9E0BF016954DB
:101EA00079406217730748F461ADDF01AB5DBE4F47
:101EB0006C933196F3CF90E080E08A01080F191FF0
:101EC00000936C0A10936D0A1A82198287E6A82E75
:101ED0008AE0B82ED12CC12C7801E5E0EE0EF11C81
:101EE000CE14DF0458F4D5016D915D01CE01019649
:101EF0000E94DD0BBFEFCB1ADB0AF2CF99818A81FA
:101F0000F701E959F54F9083F801E359F54F8083C4
:101F10008091AA089091AB08A801495F5F4F4BCF11
:101F20008AE090E053CF4F925F926F927F928F92B0
:101F30009F92AF92BF92CF92DF92EF92FF920F9358
:101F40001F93CF93DF93E0914909F0914A091281E1
:101F5000111118C08BE090E09093340B8093330BF9
:101F6000812FDF91CF911F910F91FF90EF90DF9024
:101F7000CF90BF90AF909F908F907F906F905F9029
:101F80004F90089569017A01EB01082F20E030E0BD
:101F900040E85FE360914B0970914C0980914D09D5
:101FA00090914E090E94AF6EAE0170E060E0811129
:101FB00016C000936C0AADE3B7E0EDE6FAE0812CC1
:101FC000912C540184169506A606B706D8F58D9176
:101FD00081938FEF881A980AA80AB80AF3CF009362
:101FE0006F0A1092700A2DE337E0E1E7AE2EEAE0C7
:101FF000BE2E80E090E0DC0184179507A607B707A6
:10200000B8F022969FE6A92E9AE0B92E0E941008F9
:102010002B013C019E01A50163E081E00E94860E38
:102020009093340B8093330B892B91F010E098CF71
:10203000F90101919F01F50101935F010196A11D35
:10204000B11DDACF21968CE6A82E8AE0B82EDECF1D
:102050000E941008641975098609970960935F0941
:102060007093600980936109909362090E946708E8
:102070004B015C010E9410082B013C010E94F10BF6
:102080009093340B8093330B0097C9F480916F09C0
:102090008111CCCF0E9467080E941008641975094D
:1020A00086099709609363097093640980936509B1
:1020B0009093660980916E098093320B51CF0197FE
:1020C00009F0B4CF0E946708681979098A099B0949
:1020D0006C157D058E059F0588F283E090E0909356
:1020E000340B8093330BA2CF4F925F926F927F920B
:1020F0008F929F92AF92BF92CF92DF92EF92FF9218
:102100000F931F93CF93DF9300D01F92CDB7DEB70D
:10211000E0914909F0914A09928191110AC08BE03E
:1021200090E09093340B8093330B6FEF7FEFCB01F4
:102130007EC0270138018901F42EE62ED82E20E03A
:1021400030E040E85FE360914B0970914C09809169
:102150004D0990914E090E94AF6EE98281115FC0D6
:10216000FA820E9410084B015C0124E030E0AE01CD
:102170004F5F5F4F62E08D2D0E94860E9093340B6F
:102180008093330B0E941008681979098A099B090A
:1021900060935F097093600980936109909362096D
:1021A0000E9467086B017C010E9410084B015C01D2
:1021B0000E94F10B9093340B8093330B009709F03E
:1021C0004BC080916F098111B0CF0E9467080E94B7
:1021D0001008681979098A099B096093630970934B
:1021E0006409809365099093660920917409309180
:1021F00075090217130708F49801B90190E080E00F
:10220000A0917C09B0917D09EDE3F7E0A901435C61
:10221000584FE417F50739F02D912193FACF1A8220
:10222000FB821C829ECF20916E092093320B0F906F
:102230000F900F900F90DF91CF911F910F91FF9012
:10224000EF90DF90CF90BF90AF909F908F907F9056
:102250006F905F904F900895019709F066CF0E94AC
:1022600067086C197D098E099F0964157505860537
:10227000970508F49DCF83E090E053CFEF92FF9253
:102280000F931F93CF93DF93EC018B017A018D8124
:102290009E81019691F061E08F810E94900761E03C
:1022A0008D810E9490078D810E9467070197D9F761
:1022B0008F810E9467070197B1F78B819C81DC01B8
:1022C000ED91FC910280F381E02DA701B8011995F1
:1022D0008C018D819E810196D9F08B819C81DC01DE
:1022E000ED91FC910680F781E02D199560E08D81DC
:1022F0000E94900760E08F810E9490078D810E946C
:102300006707892BD9F78F810E946707892BB1F75F
:10231000C801DF91CF911F910F91FF90EF90089529
:102320000F931F93CF93DF93EC01162F8D819E8126
:10233000019691F061E08F810E94900761E08D81AC
:102340000E9490078D810E9467070197D9F78F81BE
:102350000E9467070197B1F78B819C81DC01ED91A9
:10236000FC910190F081E02D612F19958C018D81F8
:102370009E810196D9F08B819C81DC01ED91FC91CD
:102380000680F781E02D199560E08D810E9490070D
:1023900060E08F810E9490078D810E946707892BE2
:1023A000D9F78F810E946707892BB1F7C801DF91A8
:1023B000CF911F910F910895DC0113968D919C91FF
:1023C000DC01ED91FC910284F385E02D1994DC0190
:1023D00013968D919C91DC01ED91FC910084F18527
:1023E000E02D1994CF93DF93EC018B819C810E94A7
:1023F00091051A82DF91CF910895CF93DF93EC017D
:1024000049875A876B877C878B819C810E949504C2
:102410008D819E818F3F9807C9F061E00E94BE07C1
:1024200061E08F810E94BE0760E08D810E9490076D
:1024300060E08F810E9490078D810E946707892B41
:10244000D9F78F810E946707892BB1F781E08A83D2
:10245000DF91CF910895FC01418552856385748594
:102460000C94FD1160E08EE10E94900760E08FE126
:102470000E9490078EE10E946707892BD9F78FE1B0
:102480000E946707892BB1F7089580910D0C88236E
:1024900021F083ED9BE00C94E5080895CF938DE047
:1024A00098E00E946705181619065CF5C1E08DE0FA
:1024B00098E00E946705892B21F18DE098E00E9449
:1024C000450590917005492F50E0FA01E350F94F0E
:1024D0008083923090F02091FE0630E02D5F3F4FD8
:1024E0004217530751F48D3029F4C0930F0710920F
:1024F0007005DDCF10920F07FACF9F5F90937005A4
:10250000D6CFCF9108950E94870581110E944E1267
:102510000E947D0581110E9473080E94730581113C
:102520000E94420680E090E0892B49F080E090E034
:10253000892B29F00E94000081110C94000008955D
:102540008D518D3508F0E1C1E82FF0E08827E45582
:10255000FD4E8F4F0C940F730C13111316131B1396
:10256000201325132A132F13341339133E13431347
:1025700048134D13521357135C13611366136B13F7
:10258000701375137A137F13841389138E139313A7
:1025900098139D13A213A713AC13B113B613BB1357
:1025A000C013C513CA13CF13D413D913DE13E31307
:1025B000E813ED13F213F713FC13091301140614B7
:1025C0000B14101485148514851485148514851432
:1025D0008514851485148514851485148514851433
:1025E0008514151419141E14231428142B143014D4
:1025F00035143A143F14441449144E145314581407
:102600005D14621467146C147114761485147B14B1
:10261000801484E391E0089580911C0790911D0738
:10262000089580916E0590916F05089580916C05D5
:1026300090916D05089580916A0590916B050895BC
:1026400080911D0690911E060895809168059091D5
:1026500069050895809166059091670508958091B8
:10266000640590916505089580910B0690910C0684
:1026700008958091620590916305089580916005A9
:1026800090916105089580915E0590915F05089590
:1026900080915C0590915D05089580915A05909117
:1026A0005B05089580915805909159050895809192
:1026B00056059091570508958091540590915505C0
:1026C00008958091520590915305089580910506D3
:1026D000909106060895809103069091040608954E
:1026E000809114079091150708958091210790918A
:1026F0002207089580915005909151050895809189
:10270000220690912306089580914E0590914F05E1
:10271000089580914C0590914D05089580914A054A
:1027200090914B0508958091FE059091FF050895C5
:10273000809101069091020608958091480590913C
:10274000490508958091F8059091F90508958091C3
:10275000F4059091F50508958091FA059091FB0597
:10276000089580912406909125060895809146054C
:1027700090914705089580914405909145050895ED
:102780008091420590914305089580914005909174
:102790004105089580913E0590913F0508958091EF
:1027A0003C0590913D05089580913A0590913B0537
:1027B00008958091380590913905089580913605E6
:1027C00090913705089580913405909135050895CD
:1027D0008091E2069091E3060895809132059091F0
:1027E00033050895809130059091310508958091C9
:1027F0002E0590912F05089580912C0590912D051F
:10280000089580910E0690910F0608958091140608
:1028100090911506089580911206909113060895DF
:10282000809110069091110608958091380790E0EC
:1028300008958091A2059091A30508958091A40523
:102840009091A50508958091BA059091BB050895D2
:1028500080918405ECCF809187059091880508953B
:1028600080912A0590912B050895809128059091DB
:102870002905089580919C0590919D05089580916A
:102880008505909186050895809182059091830534
:10289000089580919A0590919B05089580919805DF
:1028A00090919905089580919605909197050895C6
:1028B00080918C0590918D05089580918E05909161
:1028C0008F050895809126059091270508958091A0
:1028D0008A0590918B0508958091940590919505B6
:1028E00008958091920590919305089580919005A7
:1028F0009091910508958091A0059091A10508956A
:1029000080919E0590919F05089590E080E0089544
:102910008D518D3508F09AC3E82FF0E08827EC56EA
:10292000FB4E8F4F0C940F73F114FA1403150C1512
:10293000161520152B153415391543154D1557153A
:1029400061156D15791583158F159B15A515B11595
:10295000BD15C715D115DB15E515EF15F9150316CE
:102960000F161B1625162F16381642164C1655161E
:102970005A165F166416691673167D1687168C161E
:1029800091169A16A416AF16B8162618BD16C616B6
:10299000ED1614173B174717531726182618261835
:1029A0002618261826182618261826182618261837
:1029B00026185F1766176F177B17871790179A17D8
:1029C000A417AE17B817C217CC17D117D617DB1735
:1029D000E217E917F217FB1704180D1816181D183F
:1029E00022186F3F760709F431C370931D07609377
:1029F0001C0708956F3F760709F428C370936F058D
:102A000060936E0508956F3F760709F41FC37093B6
:102A10006D0560936C050895693E83E0780708F0C2
:102A200015C370936B0560936A050895693C2FEA9E
:102A3000720708F00BC370931E0660931D0608957D
:102A4000CB018897813C934008F000C370936905DF
:102A50006093680508956536710508F0F7C27093B4
:102A60006705609366050895709365056093640536
:102A70000895613283E0780708F0E8C270930C068D
:102A800060930B060895613D27E0720708F0DEC2EF
:102A900070936305609362050895613D87E0780750
:102AA00008F0D4C270936105609360050895613D9C
:102AB00027E0720708F0CAC270935F0560935E0555
:102AC0000895CB01885293428137974108F0BEC2E6
:102AD00070935D0560935C050895CB018852934225
:102AE0008930924508F0B2C270935B0560935A0535
:102AF000089561368AEE780708F0A8C270935905E8
:102B0000609358050895CB018852934281379741CD
:102B100008F09CC270935705609356050895CB0149
:102B2000885293428930924508F090C270935505BF
:102B300060935405089561368AEE780708F086C2DE
:102B400070935305609352050895CB0188529342C8
:102B50008137974108F07AC27093060660930506A4
:102B60000895CB01885293428930924508F06EC295
:102B700070930406609303060895613A8FE0780726
:102B800008F064C270931507609314070895613AC2
:102B90002FE0720708F05AC2709322076093210752
:102BA0000895653B83EC780708F050C27093510597
:102BB0006093500508956D3B22E0720708F046C20D
:102BC00070932306609322060895613A8CEF78078C
:102BD00008F03CC270934F0560934E050895613A2A
:102BE0002CEF720708F032C270934D0560934C05CC
:102BF0000895613A8CEF780708F028C270934B056E
:102C000060934A050895CB0180549F4181369D4DC4
:102C100008F01CC27093FF056093FE050895CB0178
:102C200080549F4181369D4D08F010C2709302067A
:102C3000609301060895613A8CEF780708F006C2A8
:102C400070934905609348050895653F21E0720738
:102C500008F0FCC17093F9056093F80508956B3F87
:102C6000710508F0F3C17093F5056093F4050895BC
:102C7000693E83E0780708F0E9C17093FB05609333
:102C8000FA050895693E23E0720708F0DFC17093EA
:102C900025066093240608956531710508F0D6C1B4
:102CA00070934705609346050895709345056093BA
:102CB0004405089570934305609342050895709309
:102CC000410560934005089570933F0560933E056C
:102CD0000895613A8CEF780708F0B8C170933D050C
:102CE00060933C050895613A2FE0720708F0AEC189
:102CF00070933B0560933A050895613B84E0780743
:102D000008F0A4C170933905609338050895709355
:102D10003705609336050895709335056093340543
:102D200008956330710508F091C17093E3066093D4
:102D3000E20608956F3F710511F008F087C17093A6
:102D40003305609332050895CB01889789379F40FA
:102D500008F07CC1709331056093300508956536A5
:102D6000710508F073C170932F0560932E050895C7
:102D700070932D0560932C0508956536710508F054
:102D800065C170930F0660930E060895CB018852BB
:102D90009342893B9B4020F4709315066093140680
:102DA000CB01805596448137974138F4CB019695F5
:102DB00087959093150680931406CB01805A9C4802
:102DC000813E9E4208F042C176956795769567955B
:102DD00070931506609314060895CB0180519742B5
:102DE000813A9F4020F47093130660931206CB0142
:102DF00080529E4481349F4138F4CB01969587954B
:102E00009093130680931206CB0180549C4981381D
:102E10009E4308F01BC176956795769567957093EC
:102E20001306609312060895CB01805E9E42813A9C
:102E30009F4020F47093110660931006CB01805CD4
:102E40009D4581349F4138F4CB01969587959093A9
:102E5000110680931006CB0180589B4B81389E430E
:102E600008F0F4C07695679576956795709311068E
:102E7000609310060895CB01885293428933974C92
:102E800008F0E4C070932505609324050895CB01F4
:102E9000885293428933974C08F0D8C07093230529
:102EA000609322050895CB01885293428933974C51
:102EB00008F0CCC07093210560932005089563301D
:102EC000710508F0C3C06093380708956430710538
:102ED00008F0BCC07093A3056093A2050895CB01D0
:102EE000845691098134964008F0B0C07093A505CE
:102EF0006093A4050895CB01845691098D3D9540BA
:102F000008F0A4C07093BB056093BA050895CB0187
:102F10000197883C910508F099C060938405089555
:102F2000673282E0780708F091C07093880560935B
:102F300087050895673222E0720708F087C0709312
:102F40002B0560932A050895693883E1780708F016
:102F50007DC070932905609328050895693823E1A1
:102F6000720708F073C070939D0560939C050895E7
:102F7000693582E0780708F069C070938605609330
:102F800085050895693522E0720708F05FC07093E7
:102F9000830560938205089570939B0560939A055D
:102FA0000895709399056093980508957093970517
:102FB00060939605089577FD49C070938D056093E1
:102FC0008C05089577FD42C070938F0560938E0540
:102FD0000895613187E27807C8F5709327056093FB
:102FE0002605089561312EE0720780F570938B05F8
:102FF00060938A050895611580E4780738F5709329
:103000009505609394050895611520E47207F0F426
:1030100070939305609392050895611580E4780795
:10302000A8F470939105609390050895623071053E
:1030300020F4862F817080931B077093A105609305
:10304000A005089570939F0560939E0508951092C2
:103050000F071092FA061092F9061092F8061092D5
:10306000FC061092FB061092F2051092DF051092FA
:10307000DE051092A0061092180610928806109293
:1030800063061092640610926506109266068CEA3A
:1030900098E00E94910540E855E260E070E08CEA1B
:1030A00098E00E9495048CEA98E00E946705892BBD
:1030B00029F08CEA98E00E944505F5CF1092380778
:1030C0000895CF92DF92EF92FF920F931F93811595
:1030D00024E0920710F08FEF93E09C01ABEAB3E09D
:1030E0000E943D7008E115E72FE030E068017901AA
:1030F000C61AD70AE80AF90AD701C60124E0B6952C
:10310000A795979587952A95D1F71F910F91FF90D5
:10311000EF90DF90CF9008950F931F93853102EFCA
:103120009007F8F4B0E0A0E024E0880F991FAA1FF0
:10313000BB1F2A95D1F748E155E76FE070E08A019F
:103140009B01081B190B2A0B3B0BC901B8012BEA89
:1031500033E040E050E00E941B70C901233E31057E
:1031600010F483EE90E01F910F910895CF93DF93B9
:10317000AC01FB018091D904893108F44DC0109253
:10318000D9048091D7049091D8049B01205E3C4FD4
:1031900028173907E0F1805E9C4F86179707B8F132
:1031A000C091D504D091D6042091D3043091D40499
:1031B000A7E0B0E00E943D704C175D0700F5C41B0E
:1031C000D50B6C0F7D1F811D911D23E09695879572
:1031D000779567952A95D1F77093D4046093D304BB
:1031E0005093D6044093D504F093D804E093D704C9
:1031F0008091D3049091D404DF91CF9108959A01E6
:103200002C1B3D0B620F731F811D911DDECF109291
:10321000D4041092D304E4CF8F5F8093D904E8CF15
:10322000CF92DF92EF92FF92809128079091290729
:10323000893263E2960708F49AC089396AE39607EF
:1032400048F5B0E0A0E09C01AD01285233424109AD
:103250005109A3E2B0E00E94087020E737E140E0A6
:1032600050E00E94E96FC0902206D0902306F12C16
:10327000E12C2C153D054E055F0508F469012AE097
:103280002C9DC0012D9D900D1124FF90EF90DF909B
:10329000CF900895893A61E69607B8F4B0E0A0E0CF
:1032A0009C01AD0128593A4341095109A5E5B0E017
:1032B0000E94087020E137E240E050E00E94E96F90
:1032C0002D5D3F4F4F4F5F4FCECF893B68E896074C
:1032D000B8F4B0E0A0E09C01AD01285A31464109A4
:1032E0005109A1E6B0E00E94087020E137E240E019
:1032F00050E00E94E96F28583F4F4F4F5F4FB3CFC8
:10330000893C6FEA9607B8F4B0E0A0E09C01AD01FB
:10331000285B384841095109A0ECB0E00E940870D0
:1033200020E137E240E050E00E94E96F27523F4F32
:103330004F4F5F4F98CF893D66ED960708F093CFCA
:10334000B0E0A0E09C01AD01285C3F4A4109510971
:10335000A1EFB0E00E94087020E137E240E050E0C9
:103360000E94E96F27563E4F4F4F5F4F7CCF20E0C2
:1033700030E0A90178CF8C3524E4920708F44EC0E0
:103380009C0150E040E0893265E59607F0F42C5549
:10339000344441095109AEE6B0E00E9408702CECBB
:1033A00030E140E050E00E94E96F80912206909168
:1033B00023062817390708F4C9012AE0AC01249F25
:1033C000C001259F900D11240895813B984698F4E3
:1033D0002852354541095109ABE4B0E00E9408701C
:1033E00028E833E140E050E00E94E96F22593F4F66
:1033F0004F4F5F4FDACF205B384641095109AFE9A3
:10340000B1E00E94087020EA3AE540E050E00E94F6
:10341000E96F27543F4F4F4F5F4FC7CF30E020E059
:10342000C4CF88332AE4920708F46AC09C0150E0B4
:1034300040E0813B6FE4960718F528533A44410970
:103440005109CA01B90122E0660F771F881F991F31
:103450002A95D1F728E735E040E050E00E94E96F77
:1034600080912206909123062817390708F4C90194
:103470002AE0AC01249FC001259F900D11240895DE
:10348000893769E6960798F4205B3F444109510962
:10349000ACE1B0E00E94087028EC39E140E050E077
:1034A0000E94E96F2C5F3F4F4F4F5F4FD9CF81395B
:1034B0009E4798F42857394641095109A4E4B0E0E1
:1034C0000E94087028E135E140E050E00E94E96F79
:1034D000205E3F4F4F4F5F4FC3CF20593E474109BA
:1034E0005109ACECB1E00E94087020EC34E440E0FB
:1034F00050E00E94E96F2C593F4F4F4F5F4FB0CFC4
:1035000030E020E0ADCFDB01EC91F0E0E558FD4F7D
:10351000E081E927F0E0E558FD4F908189278C9301
:1035200008954F925F926F927F928F929F92AF9287
:10353000BF92CF92DF92EF92FF924091A8065091F6
:10354000A90670E060E04C01B12CA12CC090A60649
:10355000D090A706F12CE12CC41AD50AE60AF70A86
:1035600082339105E0F582E3482E512C612C712CB9
:10357000D301C201841B950BA60BB70B9C01AD01B7
:10358000A1E0B8E00E940870A70196010E94E96FCF
:1035900021503C4F4F4F5F4FC501B4010E94EB7269
:1035A000A30192010E94E96F622F232F862F922F91
:1035B0008115A0E19A0714F08FEF9FE097FF02C0FA
:1035C00090E080E0FF90EF90DF90CF90BF90AF90C1
:1035D0009F908F907F906F905F904F900895D5014E
:1035E000841B950BA60BB70B9C01AD01A1E0B8E0C5
:1035F0000E940870A70196010E94E96FDA01C901D3
:1036000081509C4FAF4FBF4F682F292FCFCF1F93B3
:10361000CF93DF93182F0E94EF07EC01812F0E94B8
:10362000EF07C80FD91F812F0E94EF07C80FD91FBE
:10363000812F0E94EF078C0F9D1FDF91CF911F916B
:103640000895CF92DF92EF92FF92CF93DF9382E4BF
:103650000E94071B811520E1920710F08FEF9FE079
:103660000E94911AC0911C07D0911D0720911C0245
:1036700030911D02A90170E060E06C01F12CE12C99
:10368000CF3586E0D80708F48BC0A3E0B0E00E94F5
:103690003D7053E0CC0CDD1CEE1CFF1C5A95D1F79D
:1036A000DC01CB018C0D9D1DAE1DBF1D6C017D018C
:1036B00062E0F694E794D794C7946A95D1F7D092D4
:1036C0001D02C0921C0220911C0230911D02ABEC25
:1036D000BFE00E943D70DC01CB012BE0B695A795C1
:1036E000979587952A95D1F7909329078093280776
:1036F00088359B4108F474C083E40E94071B811540
:1037000020E1920710F08FEF9FE00E94911A209124
:10371000C2053091C305A90170E060E06C01F12C95
:10372000E12CCF35D64008F44BC0A3E0B0E00E94B6
:103730003D70A3E0CC0CDD1CEE1CFF1CAA95D1F75C
:10374000DC01CB018C0D9D1DAE1DBF1D6C017D01EB
:10375000B2E0F694E794D794C794BA95D1F7D09293
:10376000C305C092C2052091C2053091C305ACE2E9
:10377000BAE00E943D703BE09695879577956795F6
:103780003A95D1F77093200760931F078091D40575
:10379000882359F1813009F4BEC01092D405A0C02D
:1037A00033E0CC0CDD1CEE1CFF1C3A95D1F7C40EA7
:1037B000D51EE61EF71EF694E794D794C7947FCFE4
:1037C000E3E0CC0CDD1CEE1CFF1CEA95D1F7C40E27
:1037D000D51EE61EF71EF694E794D794C794BFCF84
:1037E0001092200710921F07D1CF8091C6059091AB
:1037F000C7058833914030F488E391E09093C70582
:103800008093C6058091C6059091C705855D90435C
:103810008A329F4C30F484ED90E39093C7058093F7
:10382000C6052091C6053091C705C12CD12C760163
:103830002F3F320751F050E040E060ED72E183E14C
:1038400090E00E94E96F69017A012091C4053091EE
:10385000C505A3E0B0E00E943D70C3E0CC0CDD1CC8
:10386000EE1CFF1CCA95D1F76C0D7D1D8E1D9F1D92
:10387000D2E09695879577956795DA95D1F770930D
:10388000C5056093C4059B0183E0369527958A950D
:10389000E1F7309324072093230794E0769567950A
:1038A0009A95E1F7620F731F7093190760931807D9
:1038B0002091D2053091D3054FE1429FC001439F33
:1038C000900D1124680F791F25E0769567952A954C
:1038D000E1F77093D3056093D20581E08093D4051E
:1038E0002091280730912907A0911F07B091200748
:1038F0000E943D7020EA36E841E050E00E941B70D3
:103900003093C5062093C406DF91CF91FF90EF90CE
:10391000DF90CF9008958AE30E94071B811520E174
:10392000920710F08FEF9FE02091CA0521110DC082
:103930009C01B3E0220F331FBA95E1F73093C9051C
:103940002093C80521E02093CA050E94911AAC017A
:103950002091C8053091C905A7E0B0E00E943D70F4
:103960009A0150E040E0E3E0220F331F441F551F4F
:10397000EA95D1F7260F371F481F591FF3E05695D8
:10398000479537952795FA95D1F73093C905209338
:10399000C80544275527ABECBFE00E940870ABE098
:1039A0009695879577956795AA95D1F770932B078C
:1039B00060932A07F2CE60E08AE20E94900761E0FD
:1039C0008AE20E949007A8950895CF93DF93EB01B8
:1039D0009093BF068093BE067093B7066093B606B9
:1039E0000097B1F4809120018F778093200160E0EF
:1039F0008EE20E94900780912001209799F48F7D9C
:103A00008093200160E08DE2DF91CF910C949007CC
:103A10002091200120682093200190932901809318
:103A20002801E9CF806280932001D0932B01C093BD
:103A30002A01DF91CF910895CF93DF93EB0190930B
:103A4000BD068093BC067093B5066093B4060097DC
:103A5000B1F48091A0008F7D8093A00060E087E0AA
:103A60000E9490078091A000209799F48F7780930F
:103A7000A00060E086E0DF91CF910C949007209148
:103A8000A00020622093A0009093AB008093AA0036
:103A9000E9CF80688093A000D093A900C093A800CC
:103AA000DF91CF9108958F929F92AF92BF92CF9264
:103AB000DF92EF92FF92C090DD06D090DE06F12CEF
:103AC000E12C20911405222309F48DC0A701960151
:103AD000281B390B41095109A0913E05B0913F05C2
:103AE0000E9408708090160290901702A090180211
:103AF000B0901902860E971EA81EB91E809110055F
:103B000090911105A0911205B0911305A70196019E
:103B1000281B390B4A0B5B0BA0914005B091410566
:103B20000E940870860E971EA81EB91E809212026F
:103B300090921302A0921402B0921502C092100546
:103B4000D0921105E0921205F092130580911202B5
:103B500090911302A0911402B09115028093160265
:103B600090931702A0931802B09319028130904CE1
:103B7000AF4FB10564F080E090ECAFEFB0E0809320
:103B8000120290931302A0931402B0931502809135
:103B9000120290911302A0911402B0911502B7FF86
:103BA00008C0109212021092130210921402109286
:103BB00015028091120290911302A0911402B0910B
:103BC00015022EE0B595A795979587952A95D1F77B
:103BD000BC01FF90EF90DF90CF90BF90AF909F908F
:103BE0008F900C941C1D2FEF2093140570E060E063
:103BF00085392FE7920750F425E93FE7A901481BD3
:103C0000590BCA0168E170E00E94FB7290E080E00D
:103C10003EE0660F771F881F991F3A95D1F7609392
:103C2000120270931302809314029093150286CFB0
:103C3000CF93DF93EB019093BB068093BA0670930A
:103C4000B3066093B2060097B1F48091A000877F1D
:103C50008093A00060E088E00E949007809120019E
:103C6000209799F4877F8093200160E08CE2DF91B8
:103C7000CF910C9490072091A00028602093A00081
:103C80009093AD008093AC00E9CF886080932001D1
:103C9000D0932D01C0932C01DF91CF9108958F9285
:103CA0009F92AF92BF92CF92DF92EF92FF920F93CB
:103CB0001F93C0901E05D0901F05F12CE12C209180
:103CC0000F05222309F48FC0A7019601281B390B89
:103CD00041095109A0914205B09143050E94087025
:103CE00080900B0590900C05A0900D05B0900E05EE
:103CF000860E971EA81EB91E809107059091080593
:103D0000A0910905B0910A05A7019601281B390B5E
:103D10004A0B5B0BA0914405B09145050E940870C9
:103D2000860E971EA81EB91E809203059092040568
:103D3000A0920505B0920605C0920705D09208052D
:103D4000E0920905F0920A0580910305909104051F
:103D5000A0910505B091060580930B0590930C0585
:103D6000A0930D05B0930E058130904CAF4FB10577
:103D700064F080E090ECAFEFB0E0809303059093A7
:103D80000405A0930505B093060580910305909165
:103D90000405A0910505B0910605B7FF08C0109273
:103DA00003051092040510920505109206058091F6
:103DB000030590910405A0910505B09106052EE03C
:103DC000B595A795979587952A95D1F7BC011F9131
:103DD0000F91FF90EF90DF90CF90BF90AF909F90AA
:103DE0008F900C94181E2FEF20930F0530E020E0E9
:103DF0008B3F0EE99007D8F4B0E0A0E045E0880FD3
:103E0000991FAA1FBB1F4A95D1F749E45FED63E1F3
:103E100070E08A019B01081B190B2A0B3B0BC9019F
:103E2000B8012DEC35E040E050E00E941B70C90164
:103E3000B0E0A0E03EE0880F991FAA1FBB1F3A9593
:103E4000D1F78093030590930405A0930505B093E3
:103E5000060572CF81E40E94071B811520E19207BD
:103E600010F08FEF9FE00E94911AFC0120913E0418
:103E700030913F04AFE1B0E00E943D7023E0EE0FCF
:103E8000FF1F2A95E1F79B01AC012E0F3F1F411D3B
:103E9000511D65E056954795379527956A95D1F759
:103EA00030933F0420933E04ACE2BAE00E940870D5
:103EB000DC01CB017BE0B695A795979587957A9520
:103EC000D1F7089580E40E94071B811520E1920735
:103ED00010F08FEF9FE00E94911AFC0120913C04AA
:103EE00030913D04AFE1B0E00E943D7023E0EE0F61
:103EF000FF1F2A95E1F79B01AC012E0F3F1F411DCB
:103F0000511D65E056954795379527956A95D1F7E8
:103F100030933D0420933C04ACE2BAE00E94087068
:103F2000DC01CB017BE0B695A795979587957A95AF
:103F3000D1F708958BE30E94071B811520E19207BA
:103F400010F08FEF9FE02091340421110DC09C01EF
:103F500043E0220F331F4A95E1F730933304209357
:103F6000320421E0209334040E94911A60913204BB
:103F700070913304B0E0A0E09C01AD0183E0220F1A
:103F8000331F441F551F8A95D1F7260F371F411D38
:103F9000511D5695479537952795309333042093B7
:103FA000320444275527A7E3B0E20E940870DC01E1
:103FB000CB012DE0B695A795979587952A95D1F7D2
:103FC000089580910205813009F484C048F0823060
:103FD00009F4F8C0833009F472C110920205089503
:103FE0000E949A1F9093DE068093DD0680912C0735
:103FF00090912D0788359B4108F462C00E94621F92
:104000009093AF068093AE0680912E0790912F0774
:1040100088359B4108F459C00E942A1F9093AD0631
:104020008093AC068EE30E94071B811520E1920766
:1040300010F08FEF9FE02091DC0421110DC09C0156
:1040400043E0220F331F4A95E1F73093DB042093BE
:10405000DA0421E02093DC040E94911AFC012091F3
:10406000DA043091DB04A7E0B0E00E943D70A3E0E9
:10407000EE0FFF1FAA95E1F79B01AC012E0F3F1F2A
:10408000411D511DB3E05695479537952795BA9533
:10409000D1F73093DB042093DA04A7E3B0E20E9467
:1040A00008702DE096958795779567952A95D1F7B5
:1040B00070932D0760932C0781E08093020508958B
:1040C0001092AF061092AE069FCF1092AD061092DE
:1040D000AC06A8CF0E949A1F9093DE068093DD065F
:1040E00080912C0790912D0788359B4108F460C082
:1040F0000E94621F9093AF068093AE0680912E07B8
:1041000090912F0788359B4108F457C00E942A1FC1
:104110009093AD068093AC068FE30E94071B811538
:1041200020E1920710F08FEF9FE02091E60421112B
:104130000DC09C01F3E0220F331FFA95E1F7309395
:10414000E5042093E40421E02093E6040E94911A00
:10415000FC012091E4043091E504A7E0B0E00E9466
:104160003D7023E0EE0FFF1F2A95E1F79B01AC01A4
:104170002E0F3F1F411D511D63E056954795379502
:1041800027956A95D1F73093E5042093E404A7E3DB
:10419000B0E20E940870EDE0969587957795679557
:1041A000EA95D1F770932F0760932E0782E085CFB1
:1041B0001092AF061092AE06A1CF1092AD061092EB
:1041C000AC06AACF0E949A1F9093DE068093DD066C
:1041D00080912C0790912D0788359B4108F465C08C
:1041E0000E94621F9093AF068093AE0680912E07C7
:1041F00090912F0788359B4108F45CC00E942A1FCC
:104200009093AD068093AC068CE30E94071B81154A
:1042100020E1920710F08FEF9FE02091F004211130
:104220000DC09C01B3E0220F331FBA95E1F7309324
:10423000EF042093EE0421E02093F0040E94911AF1
:10424000AC012091EE043091EF04A7E0B0E00E94B1
:104250003D709A0150E040E0E3E0220F331F441F1D
:10426000551FEA95D1F7260F371F481F591FF3E056
:104270005695479537952795FA95D1F73093EF04E2
:104280002093EE0444275527A1E7B2E00E9408706E
:10429000AEE09695879577956795AA95D1F7709337
:1042A000B9066093B80683E008CF1092AF0610926B
:1042B000AE069CCF1092AD061092AC06A5CF0E9420
:1042C0009A1F9093DE068093DD0680912C079091D3
:1042D0002D0788359B4108F464C00E94621F9093AB
:1042E000AF068093AE0680912E0790912F078835F8
:1042F0009B4108F45BC00E942A1F9093AD068093F7
:10430000AC068DE30E94071B811520E1920710F097
:104310008FEF9FE02091FA0421110DC09C01B3E0C2
:10432000220F331FBA95E1F73093F9042093F80474
:1043300021E02093FA040E94911AAC012091F80424
:104340003091F904A7E0B0E00E943D709A0150E07E
:1043500040E0E3E0220F331F441F551FEA95D1F7D9
:10436000260F371F481F591FF3E05695479537957D
:104370002795FA95D1F73093F9042093F804442750
:104380005527A1E7B2E00E940870AEE096958795A8
:1043900077956795AA95D1F77093B1066093B006AB
:1043A0001CCE1092AF061092AE069DCF1092AD06B5
:1043B0001092AC06A6CFEF92FF921F93CF93DF939C
:1043C0001F92CDB7DEB781E08983E0906A05F09057
:1043D0006B05BE016F5F7F4FC7010E94831A8091FA
:1043E0001D0690911E0612E0893C2FEA920738F4D0
:1043F00011E049EEE41643E0F40608F410E0BE01D3
:104400006F5F7F4F0E94831A8091680590916905C4
:104410009C0128523109213C334008F013E0BE01D1
:104420006F5F7F4F0E94831A8091660590916705A8
:104430008536910508F014E0BE016F5F7F4F0E9442
:10444000831ABE016F5F7F4F80916405909165056F
:104450000E94831A80910B0690910C06813223E012
:10446000920708F016E0BE016F5F7F4F0E94831A2B
:104470008091620590916305813D47E0940708F0C3
:1044800017E0BE016F5F7F4F0E94831A8091600525
:1044900090916105813D27E0920708F018E0BE0188
:1044A0006F5F7F4F0E94831A80915E0590915F0538
:1044B000813D47E0940708F019E0BE016F5F7F4F30
:1044C0000E94831A80915C0590915D059C012852A1
:1044D00033422137374108F01AE0BE016F5F7F4F4A
:1044E0000E94831A80915A0590915B059C01285285
:1044F00033422930324508F01BE0BE016F5F7F4F29
:104500000E94831A809158059091590581362AEEB0
:10451000920708F01CE0BE016F5F7F4F0E94831A74
:1045200080915605909157059C01285233422137BE
:10453000374108F01DE0BE016F5F7F4F0E94831A74
:1045400080915405909155059C01285233422930A1
:10455000324508F01EE0BE016F5F7F4F0E94831A54
:10456000809152059091530581362AEE920708F00A
:104570001FE0BE016F5F7F4F0E94831A8091050686
:10458000909106069C01285233422137374108F0AA
:1045900010E1BE016F5F7F4F0E94831A8091030676
:1045A000909104069C01285233422930324508F08C
:1045B00011E1BE016F5F7F4F0E94831A8091140743
:1045C00090911507813A2FE0920708F012E1BE01A1
:1045D0006F5F7F4F0E94831A80912107909122077D
:1045E000813A4FE0940708F013E1BE016F5F7F4FFF
:1045F0000E94831A8091500590915105853B23ECD0
:10460000920708F014E1BE016F5F7F4F0E94831A8A
:1046100080912206909123068D3B42E0940708F09A
:1046200015E1BE016F5F7F4F0E94831A80914E0596
:1046300090914F05813A2CEF920708F016E1BE01E8
:104640006F5F7F4F0E94831A80914C0590914D05BA
:10465000813A4CEF940708F017E1BE016F5F7F4F7E
:104660000E94831A80914A0590914B05813A2CEF64
:10467000920708F018E1BE016F5F7F4F0E94831A16
:104680008091FE059091FF059C0120543F41213609
:104690003D4D08F019E1BE016F5F7F4F0E94831A04
:1046A00080910106909102069C0120543F412136E1
:1046B0003D4D08F01AE1BE016F5F7F4F0E94831AE3
:1046C0008091480590914905813A2CEF920708F0B6
:1046D0001BE1BE016F5F7F4F0E94831A8091F80536
:1046E0009091F905853F41E0940708F01CE1BE0177
:1046F0006F5F7F4F0E94831A8091F4059091F505BA
:104700008B3F910508F01DE1BE016F5F7F4F0E9456
:10471000831A8091FA059091FB05893E23E0920768
:1047200008F01EE1BE016F5F7F4F0E94831A8091E7
:10473000240690912506893E43E0940708F01FE186
:10474000BE016F5F7F4F0E94831ABE016F5F7F4F74
:1047500080914405909145050E94831ABE016F5FC8
:104760007F4F80914205909143050E94831ABE01BC
:104770006F5F7F4F80914005909141050E94831AA1
:10478000BE016F5F7F4F80913E0590913F050E9473
:10479000831A80914605909147058531910508F06F
:1047A00014E2BE016F5F7F4F0E94831A80913C0527
:1047B00090913D05813A2CEF920708F015E2BE0179
:1047C0006F5F7F4F0E94831A80913A0590913B055D
:1047D000813A4FE0940708F016E2BE016F5F7F4F09
:1047E0000E94831A8091380590913905813B24E01D
:1047F000920708F017E2BE016F5F7F4F0E94831A95
:10480000BE016F5F7F4F80913605909137050E9402
:10481000831ABE016F5F7F4F8091340590913505FB
:104820000E94831A8091E2069091E30683309105FD
:1048300008F01AE2BE016F5F7F4F0E94831A8091D9
:104840003205909133058F3F910511F008F01BE27E
:10485000BE016F5F7F4F0E94831A80913005909157
:1048600031059C012852310929373F4008F01CE2EC
:10487000BE016F5F7F4F0E94831A80912E05909139
:104880002F058536910508F01DE2BE016F5F7F4F51
:104890000E94831ABE016F5F7F4F80912C0590911B
:1048A0002D050E94831A80910E0690910F06853681
:1048B000910508F01FE2BE016F5F7F4F0E94831ACF
:1048C00080911C0790911D078F3F980709F410E312
:1048D000BE016F5F7F4F0E94831A80916E05909199
:1048E0006F058F3F980709F411E3BE016F5F7F4F9B
:1048F0000E94831A80916C0590916D058F3F9807F7
:1049000009F412E3BE016F5F7F4F0E94831A80910A
:104910001406909115069C0128523342293B3B40D6
:1049200008F013E3BE016F5F7F4F0E94831A8091EE
:104930001206909113069C0120513742213A3F40C4
:1049400008F014E3BE016F5F7F4F0E94831A8091CD
:104950001006909111069C01205E3E42213A3F4094
:1049600008F015E3BE016F5F7F4F0E94831A8091AC
:104970002405909125059C01285233422933374C58
:1049800008F016E3BE016F5F7F4F0E94831A80918B
:104990002205909123059C01285233422933374C3C
:1049A00008F017E3BE016F5F7F4F0E94831A80916A
:1049B0002005909121059C01285233422933374C20
:1049C00008F018E3BE016F5F7F4F0E94831A809149
:1049D0003807833008F015E4BE016F5F7F4F90E029
:1049E0000E94831A8091A2059091A30584309105BD
:1049F00008F011E0BE016F5F7F4F0E94831A809123
:104A0000A4059091A5059C01245631092134364016
:104A100008F012E0BE016F5F7F4F0E94831A809101
:104A2000BA059091BB059C01245631092D3D3540B6
:104A300008F013E0BE016F5F7F4F0E94831A8091E0
:104A400084059FEF980F983C08F014E0BE016F5F5B
:104A50007F4F90E00E94831A80918705909188058E
:104A6000873222E0920708F015E0BE016F5F7F4FAA
:104A70000E94831A80912A0590912B05873242E08B
:104A8000940708F016E0BE016F5F7F4F0E94831A03
:104A90008091280590912905893823E1920708F033
:104AA00017E0BE016F5F7F4F0E94831A80919C05C3
:104AB00090919D05893843E1940708F018E0BE0104
:104AC0006F5F7F4F0E94831A8091850590918605C4
:104AD000893522E0920708F019E0BE016F5F7F4F31
:104AE0000E94831A8091820590918305893542E066
:104AF000940708F01AE0BE016F5F7F4F0E94831A8F
:104B0000BE016F5F7F4F80919A0590919B050E9437
:104B1000831ABE016F5F7F4F809198059091990530
:104B20000E94831ABE016F5F7F4F8091960590911E
:104B300097050E94831A80918C0590918D0597FDB1
:104B40001EE0BE016F5F7F4F0E94831A80918E0529
:104B500090918F0597FD1FE0BE016F5F7F4F0E9410
:104B6000831A8091260590912705813127E29207CB
:104B700008F010E1BE016F5F7F4F0E94831A8091A1
:104B80008A0590918B0581314EE0940708F011E180
:104B9000BE016F5F7F4F0E94831A809194059091B0
:104BA0009505811520E4920708F012E1BE016F5FC0
:104BB0007F4F0E94831A80919205909193058115F1
:104BC00040E4940708F013E1BE016F5F7F4F0E943D
:104BD000831A8091900590919105811520E49207A8
:104BE00008F014E1BE016F5F7F4F0E94831ABE017F
:104BF0006F5F7F4F8091A0059091A1050E94831A5D
:104C0000BE016F5F7F4F80919E0590919F050E942E
:104C1000831AE981F0E0E558FD4F908180914004CE
:104C200098131FEF812F0F90DF91CF911F91FF906D
:104C3000EF9008952F923F924F925F926F927F92E2
:104C40008F929F92AF92BF92CF92DF92EF92FF929C
:104C50000F931F93CF93DF9300D01F92CDB7DEB792
:104C60001C0127013801DC015F965C934E935E972F
:104C70005D967C936E935C9791963C932E93909760
:104C8000DA961C92FC0112AA13AA14AA15AA80E0B3
:104C900090E0AFE7B3E486AB97ABA0AFB1AF84E6EB
:104CA00090E0A0E0B0E086A797A7A0ABB1ABC101B0
:104CB0000E945F0420E030E0A901C801B7010E9412
:104CC000AF6E87FD91C020E030E0A901C601B501BB
:104CD0000E94AF6E87FD88C020E030E0A9016A8D98
:104CE0007B8D8C8D9D8D0E94AF6E87FD7DC0D10127
:104CF0005B961C921E925A97DB961C92DB97F101F1
:104D000040825182628273821496AD92BD92CD929E
:104D1000DC9217978A8D9B8DAC8DBD8D8087918796
:104D2000A287B38766A577A580A991A90E94B46ED2
:104D300020E030E04AE754E40E94B97069837A8346
:104D40008B839C83D1011C964D925D926D927C92D7
:104D50001F979B01AC01C601B5010E94156F4B0165
:104D60005C01F101808A918AA28AB38A29813A8101
:104D70004B815C816A8D7B8D8C8D9D8D0E94B9707D
:104D80006B017C01D1015496CD92DD92ED92FC92A3
:104D9000579758968D919C91019731F5A8019201F2
:104DA00060E070E0CB010E944C70F1016487758770
:104DB00086879787A501940160E070E0CB010E948F
:104DC0004C70D10150966D937D938D939C93539726
:104DD000A701960160E070E0CB010E944C70F101E8
:104DE000648B758B868B978B0E946708D1019E968A
:104DF000CD90DD90ED90FC90D1976C197D098E09D6
:104E00009F09F10162A373A384A395A30F900F9050
:104E10000F900F90DF91CF911F910F91FF90EF9026
:104E2000DF90CF90BF90AF909F908F907F906F90CA
:104E30005F904F903F902F90089561E08EE10E9427
:104E4000900761E08FE10E9490078EE10E94670762
:104E50000197D9F78FE10E9467070197B1F708958D
:104E60001F93CF93DF93182FEB01E0916F07F0E0D2
:104E7000E558FD4F8081892780936F07692FCE0108
:104E80000E94DB6FE0916F07F0E0E558FD4F8081F5
:104E9000812780936F07612FCE010196DF91CF911B
:104EA0001F910C94DB6F81E080936F0770E060E0EE
:104EB00080916A0590916B050E94302762E070E056
:104EC00080911D0690911E060E94302764E070E0DC
:104ED00080916805909169050E94302766E070E036
:104EE00080916605909167050E94302768E070E028
:104EF00080916405909165050E9430276AE070E01A
:104F000080910B0690910C060E9430270E94DB1CBA
:104F10006CE070E080916205909163050E943027FB
:104F20006EE070E080916005909161050E943027ED
:104F300060E170E080915E0590915F050E943027EE
:104F400062E170E080915C0590915D050E943027E0
:104F500064E170E080915A0590915B050E943027D2
:104F600066E170E080915805909159050E943027C4
:104F70000E94DB1C68E170E0809156059091570516
:104F80000E9430276AE170E08091540590915505A8
:104F90000E9430276CE170E080915205909153059A
:104FA0000E9430276EE170E0809105069091060620
:104FB0000E94302760E270E0809103069091040621
:104FC0000E94302762E270E08091140790911507EB
:104FD0000E9430270E94DB1C64E270E08091210770
:104FE000909122070E94302766E270E08091500580
:104FF000909151050E94302768E270E0809122066E
:10500000909123060E9430276AE270E080914E055D
:1050100090914F050E9430276CE270E080914C0522
:1050200090914D050E9430276EE270E080914A0514
:1050300090914B050E9430270E94DB1C60E370E0DA
:105040008091FE059091FF050E94302762E370E099
:1050500080910106909102060E94302764E370E07F
:1050600080914805909149050E94302766E370E0E1
:105070008091F8059091F9050E94302768E370E06F
:105080008091F4059091F5050E9430276AE370E065
:105090008091FA059091FB050E9430270E94DB1C4D
:1050A0006CE370E080912406909125060E943027E1
:1050B0006EE370E080914405909145050E94302791
:1050C00060E470E080914205909143050E94302792
:1050D00062E470E080914005909141050E94302784
:1050E00064E470E080913E0590913F050E94302776
:1050F00066E470E080914605909147050E94302754
:105100000E94DB1C68E470E080913C0590913D05B5
:105110000E9430276AE470E080913A0590913B0547
:105120000E9430276CE470E0809138059091390539
:105130000E9430276EE470E080913605909137052B
:105140000E94302760E570E080913405909135052C
:105150000E94302762E570E08091E2069091E306BC
:105160000E9430270E94DB1C64E570E080913205CC
:10517000909133050E94302766E570E080913005FC
:10518000909131050E94302768E570E080912E05EE
:1051900090912F050E9430276AE570E080912C05E0
:1051A00090912D050E9430276CE570E080910E06ED
:1051B00090910F060E9430276EE570E080911C07E9
:1051C00090911D070E9430270E94DB1C60E670E072
:1051D00080916E0590916F050E94302762E670E025
:1051E00080916C0590916D050E94302764E670E017
:1051F00080911406909115060E94302766E670E0B3
:1052000080911206909113060E94302768E670E0A4
:1052100080911006909111060E9430270E94DB1C9D
:105220006AE670E080912405909125050E94302760
:105230006CE670E080912205909123050E94302752
:105240006EE670E080912005909121050E94302744
:105250000E94DB1C8091380760E770E090E00E94BC
:10526000302762E770E08091A2059091A3050E942B
:10527000302764E770E08091A4059091A5050E9415
:10528000302766E770E08091BA059091BB050E94D7
:1052900030278091840568E770E090E00E94302715
:1052A0006AE770E080918705909188050E94302719
:1052B0000E94DB1C6CE770E080912A0590912B0521
:1052C0000E9430276EE770E080919C0590919D05CB
:1052D0000E94302760E870E08091280590912905B0
:1052E0000E94302762E870E08091850590918605E4
:1052F0000E94302764E870E08091820590918305D8
:105300000E94302766E870E080919A0590919B0595
:105310000E9430270E94DB1C68E870E080919805AD
:10532000909199050E9430276AE870E08091960577
:10533000909197050E9430276CE870E080918C0571
:1053400090918D050E9430276EE870E080918E0567
:1053500090918F050E94302760E970E080912605CA
:10536000909127050E94302762E970E080918A05BC
:1053700090918B050E9430270E94DB1C64E970E04D
:1053800080919405909195050E94302766E970E020
:1053900080919205909193050E94302768E970E012
:1053A00080919005909191050E9430276AE970E004
:1053B0008091A0059091A1050E9430276CE970E0D2
:1053C00080919E0590919F050E9430270E94DB1CD2
:1053D000E0916F07F0E0E558FD4F808180936F0703
:1053E0006CEA70E090E00C943027CF92DF92EF925D
:1053F000FF926230710581059105ACF06B017C0173
:105400000E942D6EA70196012150310941095109D1
:105410000E94E96F6F5F7F4F8F4F9F4FFF90EF901C
:10542000DF90CF90089561E070E080E090E0F6CFEB
:10543000FB0101900020E9F73197AF01461B570BA4
:105440000C94F004CF93DF93BC018DE098E00E94B0
:10545000182AEC016DE973E08DE098E00E94182AAB
:105460008C0F9D1FDF91CF9108950F931F93CF93C2
:10547000DF93EC0188819981009759F02A813B8163
:105480002617370730F081E0DF91CF911F910F9100
:1054900008958B016F5F7F4F0E943C74009759F015
:1054A000998388831B830A832C813D81232B59F7A1
:1054B000FC011082E8CF80E0E7CFCF93DF93EC01CF
:1054C00088819981009711F00E94B3731982188224
:1054D0001D821C821B821A82DF91CF910895EF9268
:1054E000FF920F931F93CF93DF93EC01FB01E080BA
:1054F000F180E114F10411F1048115810115110508
:10550000A9F08C819D81080F191FB801CE010E945E
:10551000352A882399F0288139818C819D81B701B2
:10552000820F931F0E9426751D830C83CE01DF918D
:10553000CF911F910F91FF90EF900895CE010E949F
:105540005D2AF4CFEF92FF920F931F93CF93DF93D7
:10555000EC017B018A01BA010E94352A81110BC03E
:10556000CE010E945D2ACE01DF91CF911F910F9154
:10557000FF90EF9008951D830C83B7018881998176
:105580000E942675F0CFCF93DF93EC01FB018617C5
:10559000970749F0608171816115710541F044817F
:1055A00055810E94A22ACE01DF91CF9108950E94D9
:1055B0005D2AF9CFFC0180819181009711F00C9454
:1055C000B37308952F923F924F925F926F927F92A2
:1055D0008F929F92AF92BF92CF92DF92EF92FF9203
:1055E0000F931F93CF93DF9300D01F92CDB7DEB7F9
:1055F0000091300510913105C80168E270E00E9409
:10560000FB7290E080E00E94B46E20E030E040E861
:105610005FE30E944D700E9432716115710509F4BB
:10562000B6C17093D2046093D1044091D1045091DB
:10563000D2049A0121503109A091CF04B091D00435
:105640000E943D70E090C406F090C5066E0D7F1D6F
:10565000811D911D9A0150E040E00E941B702901BC
:105660003A013A8329833093D0042093CF04809168
:10567000E106811102C01092CE048091250782308C
:1056800008F08CC127E333E03093C3062093C206B1
:105690001092CE04909134079B7F90933407109220
:1056A000C1061092C006823009F0D6C18091320541
:1056B00090913305009709F0BEC2F090CE0400919E
:1056C000CF041091D0040E9410199A83898390937B
:1056D000C7068093C606F11028C0809128079091D4
:1056E00029070E948C189093580480935704B0E0C7
:1056F000A0E022E1880F991FAA1FBB1F2A95D1F7AE
:105700008093530490935404A0935504B09356048B
:105710009801AAE0B0E00E943D7060934F0470933E
:10572000500480935104909352042091AA06309122
:10573000AB0680912406909125068217930708F402
:10574000AAC020912206309123064AE0429FC00160
:10575000439F900D11248017910708F49CC0980175
:10576000AAE0B0E00E943D706B017C0189819A81C2
:105770009C0150E040E0201B310B410951090E947F
:1057800008709B01AC01A0913405B09135050E94D1
:1057900008700091530410915404209155043091E5
:1057A00056044B015C01800E911EA21EB31E809117
:1057B0004F0490915004A0915104B0915204A7015C
:1057C0009601281B390B4A0B5B0BA0913605B09153
:1057D00037050E940870860E971EA81EB91E80927B
:1057E0004B0490924C04A0924D04B0924E04C0928F
:1057F0004F04D0925004E0925104F09252048092EF
:10580000530490925404A0925504B092560491E02F
:10581000891691049CEFA9069FE0B90664F080E028
:1058200090E0ACEFBFE080934B0490934C04A093C6
:105830004D04B0934E0480914B0490914C04A09180
:105840004D04B0914E04B7FF08C010924B04109263
:105850004C0410924D0410924E0480914B04909190
:105860004C04A0914D04B0914E0402E1B595A7956A
:10587000979587950A95D1F7813CA3E09A0710F098
:1058800080EC93E0883C910510F488EC90E09093D4
:105890005804809357048091570490915804909332
:1058A000C3068093C20681E08093CE040091340742
:1058B000098380911C0790911D078F35964010F445
:1058C0000C94003C86E30E94EF077C0188E30E9471
:1058D000EF078C0189E30E94EF079701201B310B32
:1058E0000E151F0518F098012E193F098017910712
:1058F00010F00C94E53B081B190B8E159F0510F05A
:105900000C94EB3BD701A81BB90BCD012431310519
:1059100010F00C94EF3B0431110510F00C94EF3BA8
:10592000449710F00C94EF3B80912307909124074B
:10593000892B11F40C94EF3B1092C1041092C00417
:105940008091C0049091C1048E37910510F40C949D
:10595000FA3B01979093C1048093C00409810460CD
:105960000093340720912807309129078091C406BD
:105970009091C5066AE070E00E94FB72CB01B9010C
:105980000E94B6189093C1068093C00665C081E05E
:1059900090E09093D2048093D10447CE843009F0F4
:1059A000B4C0809134078B7F809334078091CE04FC
:1059B00081110AC080912807909129070E948C18B4
:1059C00090934304809342042091AA063091AB0641
:1059D00080912406909125068217930790F12091DB
:1059E0002206309123064AE0429FC001439F900D5A
:1059F000112409811A818017910718F1209141041F
:105A0000809168059091690568E270E00E94FB72E0
:105A10002617170608F475C080914204909143043C
:105A2000109241042091660530916705820F931F03
:105A30008F3F13E0910708F061C090934304809377
:105A4000420480914204909143049093C306809352
:105A5000C20681E08093CE048091C304811103C00B
:105A600081E08093C30480911E07833011F00C9471
:105A7000553C4091B8065091B9062091B00630913E
:105A8000B1068091C204BA01645C7F4F621773074C
:105A900010F00C94473C813B1CF081508093C20471
:105AA0002091C2063091C3069091C20497FD9D5F7C
:105AB00095959595B901690F711D97FD7A956115B9
:105AC00054E0750710F06FEF73E0C9010F900F906D
:105AD0000F900F90DF91CF911F910F91FF90EF905A
:105AE000DF90CF90BF90AF909F908F907F906F90FE
:105AF0005F904F903F902F900C94E51C8FEF93E0B8
:105B00009CCF2F5F209341049CCF833009F0CBCDF5
:105B1000809134078B7F809334078091CE0481116C
:105B20000AC080912807909129070E948C189093B1
:105B30004A04809349042091AA063091AB068091D3
:105B40002406909125068217930708F461C02091DE
:105B5000220630912306AAE0B0E00E943D70930136
:105B600082012227332760177107820793070CF4FD
:105B70004FC020914804809168059091690568E2C2
:105B800070E00E94FB722617170608F450C080913F
:105B9000490490914A04109248042091660530917E
:105BA000670509811A81012B89F49093470480933A
:105BB0004604820F931F8F3F13E0910710F08FEF81
:105BC00093E090934A04809349041EC04091460498
:105BD00050914704609144047091450409811A81F1
:105BE000909347048093460406171707B0F44817AC
:105BF0005907F8F62817390718F4821B930BE1CFE1
:105C000010924A0410924904509245044092440470
:105C10008091490490914A0418CF8417950750F356
:105C2000820F931F8F3F23E0920748F6CACF2F5F62
:105C300020934804EDCF8130910509F02DC3909059
:105C4000CE0480911C0790911D07A090AA06B090E9
:105C5000AB06C0902406D09025068F35964008F4F8
:105C600063C20E9410199093C7068093C6069110D4
:105C70000EC082EE91E0909363048093620490934F
:105C800061048093600490935F0480935E04CA145F
:105C9000DB0408F47AC120915D04C80168E270E079
:105CA0000E94FB722617170608F43AC210925D0490
:105CB000A0905B04B0905C04912C812CE5E1AE16C1
:105CC000B10458F1712C612C9701A4E6B0E00E9458
:105CD0003D7069837A838B839C83ACE9BFEFA3011A
:105CE00095010E94167009811A812B813C81600FF9
:105CF000711F821F931FA30195010E94E96F490143
:105D000037FF04C088249924821A930A15E6811665
:105D100091041CF014E6812E912C00912E05109117
:105D20002F05609128077091290790E080E00E947C
:105D3000B46E2B013C01609150057091510590E0CB
:105D400080E00E94B46E9B01AC01C301B2010E94CD
:105D5000156F2CEA35EC47E257E30E94156F2B01D3
:105D60003C0120E030E0A9010E94617120E030E0B8
:105D700040E05FE387FD27C0C301B2010E944D7080
:105D80000E942B71C0906004D09061042091620445
:105D9000309163043A8329836E157F05C8F4D0924D
:105DA0005F04C0925E043093610420936004C801D4
:105DB00082559F4F8217930708F061C1201B310B5A
:105DC0003A83298361C0C301B2010E944C70D8CFCD
:105DD0006090180770901907B30190E080E00E946E
:105DE000B46E22E430E645E95FE3A4E06A16A6E07B
:105DF0007A0650F420E030E040E450E40E946671FE
:105E000022EA37EE4BE355E30E94156F2B013C016C
:105E100020E030E0A9010E94617120E030E040E024
:105E20005FE387FD34C0C301B2010E944D700E9440
:105E30002B71C801A3E0880F991FAA95E1F7209064
:105E40002206309023069101B3E0220F331FBA954A
:105E5000E1F76217730708F49B012E153F05E0F088
:105E6000D0925F04C0925E0409811A81109361048C
:105E700000936004080F191F1A83098340EC53E054
:105E8000003C134008F0FDC089819A81A3C0C30182
:105E9000B2010E944C70CBCF2801712C612CB0E074
:105EA000A0E09C01AD012419350946095709D40128
:105EB0000E94137024E630E040E050E00E94E96F59
:105EC000420E531E641E751E99E54916510418F0C2
:105ED000F8E54F2E512CEA14FB0408F083C08091A2
:105EE000590490915A04A816B90608F07BC0809115
:105EF0005E0490915F04A981BA81AC15BD05C8F418
:105F0000C816D90608F046C0D0925F04C0925E045D
:105F1000B0936104A0936004A40DB51DBA83A98356
:105F200000EC13E0A03CB34008F0F7C029813A81AF
:105F3000D3C0C816D90670F1D0925F04C0925E0437
:105F400009811A811093610400936004440C551C6C
:105F5000C20182559F4F8017910708F069C004194C
:105F600015091A83098349815A8150936304409328
:105F7000620480915B0490915C0490935A04809336
:105F80005904F0925C04E0925B0480916204909169
:105F9000630485CCD0925F04C0925E0489819A81AB
:105FA0009093610480936004000F111F000F111F74
:105FB000B80190E080E00E94F52970E080916204D1
:105FC000909163049B0122553F4F2817390738F4FD
:105FD000861B970B9093630480936204CACF8EEA6A
:105FE00090E0F8CF2AE0229DC001239D900D11245E
:105FF000AE14BF0408F048C02091590430915A04EF
:106000002A153B0508F040C08E159F0588F1809148
:106010005E0490915F0409811A81C016D10668F070
:106020008C159D05D0F0D0925F04C0925E048ACF9B
:106030002EEA30E03A83298396CF8C159D0568F4CB
:10604000D0925F04C0925E0409811A8110936104AA
:1060500000936004040D151D0FCFD0925F04C09211
:106060005E0409811A81109361040093600481CF5A
:10607000D0925F04C0925E0429813A8194CE4EEAA8
:1060800050E05A83498300CFD0925F04C0925E04EF
:10609000A981BA81B0936104A09360048E159F0515
:1060A00068F1000F111F000F111FB80190E080E090
:1060B0000E94F5292091620430916304862F062EF8
:1060C000000C990B60FF10C0AC0142555F4F4217A6
:1060D000530738F4281B390B309363042093620470
:1060E00048CF2EEA30E0F8CF820F931F803CB3E018
:1060F0009B0708F46FCF80EC93E06CCFC80182550A
:106100009F4FE981FA818E179F0728F4E01BF10B5E
:10611000FA83E9830BCF0EEA10E01A83098306CFD6
:106120002F5F20935D0431CF2091CC043091CD04BA
:10613000A7E0B0E00E943D702B013C014E0C5F1CBB
:10614000611C711C53E076946794579447945A9558
:10615000D1F75A8249825092CD044092CC049110DA
:106160000AC087E593E090936A0480936904909352
:106170006804809367040E9410199093C706809367
:10618000C606CA14DB0408F44CC080916604833050
:1061900008F47EC04091690450916A0480912807F8
:1061A000909129071092660409811A81012BD1F47C
:1061B000509368044093670481329E4468F04B5FBB
:1061C0005F4F4F3F23E05207B8F18FEF93E090937A
:1061D0006A048093690421C046305105D0F04550CF
:1061E00051092AC0E0916704F09168048091640429
:1061F0009091650409811A810817190710F55093C9
:10620000680440936704E417F50780F44E3C510599
:1062100030F710926A04109269045092650440921B
:1062200064048091690490916A0439CB4B5F5F4F9D
:106230004F3F13E0510748F650936A0440936904B6
:10624000ECCF2091220630912306AAE0B0E00E9414
:106250003D70509368044093670464157505860586
:10626000970524F04E175F0788F2A9CF4E175F07F6
:1062700038F04E3C510508F0B2CF88EC90E0A7CF43
:106280004B5F5F4F4F3F33E0530708F09ECFD4CFB3
:106290008F5F80936604C5CF8230910509F047C1B6
:1062A000D090CE040091CF041091D0041A830983BA
:1062B000C0908906E0902807F0902907C7010E9446
:1062C000111A8C01CC2009F42DC1C7010E94BB1901
:1062D0004C01B12CA12C4090BA055090BB05712CFB
:1062E000612C20919E0630919F0650E040E02419D9
:1062F000350946095709B80190E080E06819790925
:106300008A099B090E94EB722091A4053091A50592
:1063100050E040E024193509460957090E94E96F09
:10632000820E931EA41EB51EA40197FCF8C02091F6
:106330002206309123066AE0629FC001639F900DA0
:1063400011248815990508F4AC015093C7064093B1
:10635000C606D11026C0C7010E948C1890937804FD
:1063600080937704B0E0A0E042E1880F991FAA1F54
:10637000BB1F4A95D1F78093730490937404A09344
:106380007504B093760429813A81AAE0B0E00E94B6
:106390003D7060936F0470937004809371049093C8
:1063A00072042091AA063091AB0680912406909148
:1063B00025068217930708F4ADC02091220630917C
:1063C00023064AE0429FC001439F900D112409819A
:1063D0001A818017910708F49DC09801AAE0B0E0E7
:1063E0000E943D706B017C012091C6063091C7066A
:1063F00050E040E0201B310B410951090E94087018
:106400009B01AC01A0913405B09135050E94087044
:1064100000917304109174042091750430917604F6
:106420004B015C01800E911EA21EB31E80916F0471
:1064300090917004A0917104B0917204A70196012B
:10644000281B390B4A0B5B0BA0913605B091370521
:106450000E940870860E971EA81EB91E80926B04BB
:1064600090926C04A0926D04B0926E04C0926F047E
:10647000D0927004E0927104F092720480927304DE
:1064800090927404A0927504B092760411E0811683
:1064900091041CEFA1061FE0B10664F080E090E0DB
:1064A000ACEFBFE080936B0490936C04A0936D04F9
:1064B000B0936E0480916B0490916C04A0916D0474
:1064C000B0916E04B7FF08C010926B0410926C0478
:1064D00010926D0410926E0480916B0490916C0484
:1064E000A0916D04B0916E0432E1B595A795979592
:1064F00087953A95D1F7813C23E0920710F080EC24
:1065000093E0883C910510F488EC90E09093780437
:10651000809377048091770490917804C0C950E00B
:1065200040E013CF9093C7068093C60612CF833006
:10653000910509F06CC24091CF045091D0045A8368
:1065400049838091CE0481112FC0809128079091BA
:1065500029070E948C1890938B0480938A04B0E0E2
:10656000A0E022E1880F991FAA1FBB1F2A95D1F72F
:106570008093860490938704A0938804B093890441
:1065800029813A81AAE0B0E00E943D7060938204C4
:1065900070938304809384049093850480E092E058
:1065A00090930502809304022091AA063091AB06D5
:1065B00080912406909125068217930708F47BC1E9
:1065C00080912206909123062AE0289FF001299FBE
:1065D000F00D112489819A81E817F90708F46BC13D
:1065E00020918104C80168E270E00E94FB722617C6
:1065F000170608F408C2A0910402B0910502109297
:10660000810420917F043091800440917D04509159
:106610007E04809102029091030260912E05709198
:106620002F0509811A810217130708F052C1241798
:10663000350708F0B4C12091000230910102A8177B
:10664000B907B0F48217930750F590930102809335
:106650000002B0930302A09302026A0F7B1F6D3FFA
:1066600013E07107B8F5709305026093040232C01D
:1066700082179307A0F09093010280930002B093D9
:106680000302A0930202CB010A96A817B90710F1E2
:10669000A61BB70BB0930502A09304021BC09093F6
:1066A000010280930002B0930302A0930202660FDE
:1066B000771F660F771F90E080E00E94F529809198
:1066C000040290910502680F792F711D6C3F23E041
:1066D000720748F280917F049091800490937E0429
:1066E00080937D0409811A811093800400937F04B4
:1066F00000910402109105020E941019BC0190E063
:1067000080E00E94B46E4B015C012AE939E949E15D
:106710005FE30E94156F0E942B716B017C012DECD1
:106720003CEC4CEC5FE3C501B4010E94156F0E9484
:106730002B719B01AC012C193D094E095F09D80151
:106740000E94087020E034E040E050E00E94E96FD1
:10675000C20ED31EE41EF51E8091220690912306E0
:106760006AE0689FF001699FF00D1124CE16DF06E4
:1067700008F4F601F093C706E093C60629813A8132
:10678000AAE0B0E00E943D706B017C019F0150E0E7
:1067900040E009811A81201B310B410951090E94F7
:1067A00008709B01AC01A0913405B09135050E94A1
:1067B000087000918604109187042091880430911C
:1067C00089044B015C01800E911EA21EB31E8091B4
:1067D000820490918304A0918404B0918504A70160
:1067E0009601281B390B4A0B5B0BA0913605B09123
:1067F00037050E940870860E971EA81EB91E80924B
:10680000790490927A04A0927B04B0927C04C092A6
:106810008204D0928304E0928404F09285048092F2
:10682000860490928704A0928804B092890411E0B3
:10683000811691041CEFA1061FE0B10664F080E010
:1068400090E0ACEFBFE08093790490937A04A0933A
:106850007B04B0937C048091790490917A04A09198
:106860007B04B0917C04B7FF08C0109279041092A9
:106870007A0410927B0410927C04809179049091A8
:106880007A04A0917B04B0917C0412E1B595A795A0
:10689000979587951A95D1F7813C23E0920710F0E0
:1068A00080EC93E0883C910510F488EC90E09093A4
:1068B0008B0480938A048091040290910502909346
:1068C000C9068093C80680918A0490918B040C9429
:1068D0004F2C2417350708F462C0EE15FF0508F4A5
:1068E0004EC020910002309101028A179B0750F19F
:1068F0002817390708F0BFCE909301028093000259
:10690000B0930302A0930202660F771F660F771FF2
:1069100090E080E00E94F52920912E0530912F050E
:10692000809104029091050260FF1FC0820F931FA7
:106930008D3F43E0940708F0CDCE909305028093FD
:106940000402C8CE28173907B8F690930102809345
:106950000002B0930302A09302026A0F7B1F6D3FF7
:1069600033E0730708F0B6CE7ECEA901465F5F4FD5
:106970008417950708F4AECE821B930BDECF90935D
:10698000010280930002B0930302A09302026A0FF7
:106990007B1F6D3F53E0750708F09CCE64CE90934B
:1069A000010280930002B0930302A0930202EE154D
:1069B000FF0508F468CE660F771F660F771F90E01B
:1069C00080E00E94F5292091040230910502862F73
:1069D000062E000C990B60FF08C0820F931F8D3F9D
:1069E000A3E09A0708F076CEA8CFAC01465F5F4FD0
:1069F0002417350708F46ECE281B390B3093050297
:106A00002093040267CE2F5F2093810471CE8430DF
:106A1000910561F480912C0590912D050E948C18B0
:106A20009093C3068093C2060C94562C8530910532
:106A300009F0A8C24091CF045091D0045A834983F1
:106A40008091CE0481112FC0809128079091290751
:106A50000E948C1890939E0480939D04B0E0A0E067
:106A6000F2E1880F991FAA1FBB1FFA95D1F78093F7
:106A7000990490939A04A0939B04B0939C04298159
:106A80003A81AAE0B0E00E943D7060939504709353
:106A90009604809397049093980480E092E09093FA
:106AA0000B0280930A022091AA063091AB068091D6
:106AB0002406909125068217930708F4BEC18091A1
:106AC0002206909123062AE0289FF001299FF00DCD
:106AD000112489819A81E817F90708F4AEC1209141
:106AE0009404C80168E270E00E94FB722617170642
:106AF00008F441C2A0910A02B0910B0210929404D2
:106B0000209192043091930440919004509191040B
:106B1000809108029091090260912E0570912F05D5
:106B200009811A810217130708F095C12417350748
:106B300008F0EDC12091060230910702A817B907AD
:106B4000B0F48217930750F59093070280930602E2
:106B5000B0930902A09308026A0F7B1F6D3F13E0F8
:106B60007107B8F570930B0260930A0232C0821766
:106B70009307A0F09093070280930602B093090256
:106B8000A0930802CB010A96A817B90710F1A61B1B
:106B9000B70BB0930B02A0930A021BC0909307029D
:106BA00080930602B0930902A0930802660F771F34
:106BB000660F771F90E080E00E94F52980910A021D
:106BC00090910B02680F792F711D6C3F23E07207C3
:106BD00048F2809192049091930490939104809351
:106BE000900409811A811093930400939204E09019
:106BF0000A02F0900B0290908906A0902807B090AE
:106C00002907C5010E94111A6C01809122069091FA
:106C100023062AE0289F8001299F100D1124992026
:106C2000B1F1C5010E94BB194C01B12CA12C4090BF
:106C3000BA055090BB05712C612C20919E063091B5
:106C40009F0650E040E02419350946095709B6016E
:106C500090E080E0681979098A099B090E94EB722B
:106C60002091A4053091A50550E040E02419350994
:106C7000460957090E94E96F820E931EA41EB51E95
:106C8000640197FC7CC10815190508F46801B60178
:106C900090E080E00E94B46E2B013C012DEC3CECB6
:106CA0004CE45FE30E94156F0E942B714B015C0165
:106CB0002AE939E949E95FE3C301B2010E94156F8E
:106CC0000E942B719B01AC01281939094A095B0903
:106CD000D7010E9408702FEF33E040E050E00E949F
:106CE000E96FBA01A901480D591D6A1D7B1D0417E2
:106CF000150708F4A8015093C7064093C6062981DA
:106D00003A81AAE0B0E00E943D706B017C0170E026
:106D100060E09A01AB0109811A81201B310B410906
:106D200051090E9408709B01AC01A0913405B091FB
:106D300035050E9408700091990410919A042091E1
:106D40009B0430919C044B015C01800E911EA21E9D
:106D5000B31E8091950490919604A0919704B091F0
:106D60009804A7019601281B390B4A0B5B0BA091D5
:106D70003605B09137050E940870860E971EA81E32
:106D8000B91E80928C0490928D04A0928E04B092D1
:106D90008F04C0929504D0929604E0929704F092EA
:106DA00098048092990490929A04A0929B04B092C5
:106DB0009C0411E0811691041CEFA1061FE0B106AE
:106DC00064F080E090E0ACEFBFE080938C0490939F
:106DD0008D04A0938E04B0938F0480918C049091C5
:106DE0008D04A0918E04B0918F04B7FF08C010925B
:106DF0008C0410928D0410928E0410928F04809156
:106E00008C0490918D04A0918E04B0918F0432E196
:106E1000B595A795979587953A95D1F7813C23E04D
:106E2000920710F080EC93E0883C910510F488EC18
:106E300090E090939E0480939D0480910A0290912B
:106E40000B029093C9068093C80680919D0490918F
:106E50009E040C944F2C2417350708F458C0EE15E7
:106E6000FF0508F444C020910602309107028A17FA
:106E70009B0750F12817390708F07CCE9093070242
:106E800080930602B0930902A0930802660F771F51
:106E9000660F771F90E080E00E94F52920910A029A
:106EA00030910B02862F062E000C990B60FF55C007
:106EB000820F931F8D3F43E0940708F08ACE909392
:106EC0000B0280930A0285CE28173907B8F69093F3
:106ED000070280930602B0930902A09308026A0F8A
:106EE0007B1F6D3F33E0730708F073CE3BCE90936A
:106EF000070280930602B0930902A09308026A0F6A
:106F00007B1F6D3F53E0750708F063CE2BCE909347
:106F1000070280930602B0930902A0930802EE15BF
:106F2000FF0508F42FCE660F771F660F771F90E0DE
:106F300080E00E94F52920910A0230910B02862FF1
:106F4000062E000C990B60FF08C0820F931F8D3F27
:106F5000A3E09A0708F03DCEB2CFAC01465F5F4F89
:106F60002417350708F435CE281B390B30930B0254
:106F700020930A022ECE2F5F2093940438CED12C7A
:106F8000C12C85CE8630910531F5209118073091BE
:106F9000190750E040E02059314041095109A8EE5D
:106FA000B0E80E94087028EE33E040E050E00E9414
:106FB000E96FDA01C90180519A4AAF4FBF4F893654
:106FC0003FEB9307A105B10508F428CD88E69FEBB8
:106FD000A0E0B0E023CD8730910509F0F5C24091E3
:106FE000CF045091D0045A8349838091CE048111FB
:106FF0002FC080912807909129070E948C189093A8
:10700000B1048093B004B0E0A0E022E1880F991FA2
:10701000AA1FBB1F2A95D1F78093AC049093AD04AF
:10702000A093AE04B093AF0429813A81AAE0B0E006
:107030000E943D706093A8047093A9048093AA04F1
:107040009093AB0480E092E0909311028093100241
:107050002091AA063091AB068091240690912506D6
:107060008217930708F492C180912206909123061B
:107070002AE0289F6001299FD00C112489819A81E0
:10708000C816D90608F482C12091A704C80168E295
:1070900070E00E94FB722617170608F41FC2809149
:1070A0001002909111021092A7044091A5045091F2
:1070B000A604E091A304F091A40420910E02309163
:1070C0000F0260912E0570912F0509811A81041716
:1070D000150708F069C14E175F0708F0CBC1409152
:1070E0000C0250910D0282179307B0F42417350754
:1070F00038F530930D0220930C0290930F02809389
:107100000E02680F791F6D3F13E07107A0F57093B1
:107110001102609310022FC02417350788F03093B6
:107120000D0220930C0290930F0280930E029B019C
:10713000265F3F4F82179307F0F0861B970B68C1BD
:1071400030930D0220930C0290930F0280930E0255
:10715000660F771F660F771F90E080E00E94F52989
:107160008091100290911102680F792F711D6C3F70
:1071700023E0720760F28091A5049091A604909399
:10718000A4048093A30409811A811093A604009398
:10719000A50400911002109111022091280730914E
:1071A0002907273B4FE2340708F09CC1A9E0B0E073
:1071B0000E943D7026EB3FE240E050E00E94E96F04
:1071C00049015A01E0902206F0902306C701B0E081
:1071D000A0E088169906AA06BB0608F4C4015AE086
:1071E000752E789E6001799ED00C1124B60190E036
:1071F00080E00E94B46E20E030E040E05FE30E9457
:10720000156F0E942B714B015C01CC0CDD1C9601AB
:1072100050E040E0281939094A095B09D8010E9469
:10722000087020E034E040E050E00E94E96F820EF8
:10723000931EA41EB51E7E9CA0017F9C500D1124A0
:107240008416950608F4A4015093C7064093C60619
:1072500029813A81AAE0B0E00E943D706B017C0177
:1072600070E060E09A01AB0109811A81201B310BAB
:10727000410951090E9408709B01AC01A09134059D
:10728000B09135050E9408700091AC041091AD04D6
:107290002091AE043091AF044B015C01800E911E31
:1072A000A21EB31E8091A8049091A904A091AA04E3
:1072B000B091AB04A7019601281B390B4A0B5B0B5D
:1072C000A0913605B09137050E940870860E971E72
:1072D000A81EB91E80929F049092A004A092A104BF
:1072E000B092A204C092A804D092A904E092AA0489
:1072F000F092AB048092AC049092AD04A092AE04E4
:10730000B092AF0411E0811691041CEFA1061FE0BA
:10731000B10664F080E090E0ACEFBFE080939F04A2
:107320009093A004A093A104B093A20480919F0421
:107330009091A004A091A104B091A204B7FF08C04D
:1073400010929F041092A0041092A1041092A20423
:1073500080919F049091A004A091A104B091A204F7
:1073600042E1B595A795979587954A95D1F7813CC8
:1073700023E0920710F080EC93E0883C910510F434
:1073800088EC90E09093B1048093B0048091100257
:10739000909111029093C9068093C8068091B00421
:1073A0009091B1040C944F2C4E175F0708F462C003
:1073B000CE14DF0408F44EC040910C0250910D022F
:1073C0002817390750F14217530708F0A8CE309319
:1073D0000D0220930C0290930F0280930E02660F11
:1073E000771F660F771F90E080E00E94F5292091BB
:1073F0002E0530912F05809110029091110260FFAF
:107400001FC0820F931F8D3F43E0940708F0B3CE57
:107410009093110280931002AECE42175307B8F634
:1074200030930D0220930C0290930F0280930E0272
:10743000680F791F6D3F33E0730708F09CCE67CE6D
:10744000A901465F5F4F8417950708F494CE821B0D
:10745000930BDECF30930D0220930C0290930F021A
:1074600080930E02680F791F6D3F53E0750708F097
:1074700082CE4DCE30930D0220930C0290930F02DA
:1074800080930E02CE14DF0408F451CE660F771FEE
:10749000660F771F90E080E00E94F529209110028E
:1074A00030911102862F062E000C990B60FF08C048
:1074B000820F931F8D3FA3E09A0708F05CCEA8CF00
:1074C000AC01465F5F4F2417350708F454CE281BE4
:1074D000390B30931102209310024DCE2F5F209371
:1074E000A70457CE26385FE43507C0F450E040E0EB
:1074F000265B3F4241095109ACE4B0E00E940870AC
:107500002FEC3FE140E050E00E94E96F49015A0151
:1075100089E0880E911CA11CB11C54CE25359FE634
:107520003907C0F450E040E025583F444109510973
:10753000A4E8B0E00E9408702FEC3FE140E050E08A
:107540000E94E96F49015A01A5E58A0E911CA11C10
:10755000B11C38CE2432BFE83B07C0F450E040E015
:1075600024553F4641095109A0ECB0E00E94087043
:107570002FEC3FE140E050E00E94E96F49015A01E1
:10758000E9ED8E0E911CA11CB11C1CCE233FFEEA1E
:107590003F0708F017CE50E040E023523F48410932
:1075A0005109A1EFB0E00E9408702FEC3FE140E0EC
:1075B00050E00E94E96F49015A0189E9880E81E093
:1075C000981EA11CB11CFECD889709F0FBC020912C
:1075D0002807309129074091CE040091CF041091E3
:1075E000D00480912C0590912D056AE070E00E94F6
:1075F000FB727A8369837093C7066093C606411154
:1076000025C0C9010E948C189093BF048093BE04CA
:10761000B0E0A0E032E1880F991FAA1FBB1F3A9586
:10762000D1F78093BA049093BB04A093BC04B093A9
:10763000BD049801AAE0B0E00E943D706093B604DA
:107640007093B7048093B8049093B9042091AA066C
:107650003091AB06809124069091250682179307FE
:1076600008F4AAC020912206309123064AE0429FE6
:10767000C001439F900D11248017910708F49CC00E
:107680009801AAE0B0E00E943D706B017C01898105
:107690009A819C0150E040E0201B310B41095109C7
:1076A0000E9408709B01AC01A0913405B091350592
:1076B0000E9408700091BA041091BB042091BC0490
:1076C0003091BD044B015C01800E911EA21EB31EC1
:1076D0008091B6049091B704A091B804B091B90418
:1076E000A7019601281B390B4A0B5B0BA0913605AD
:1076F000B09137050E940870860E971EA81EB91E0D
:107700008092B2049092B304A092B404B092B504F3
:10771000C092B604D092B704E092B804F092B904D3
:107720008092BA049092BB04A092BC04B092BD04B3
:1077300091E0891691049CEFA9069FE0B90664F0D8
:1077400080E090E0ACEFBFE08093B2049093B3048C
:10775000A093B404B093B5048091B2049091B304A3
:10776000A091B404B091B504B7FF08C01092B20460
:107770001092B3041092B4041092B5048091B20434
:107780009091B304A091B404B091B50422E1B595F1
:10779000A795979587952A95D1F7813CA3E09A07FD
:1077A00010F080EC93E0883C910510F488EC90E0B8
:1077B0009093BF048093BE048091BE049091BF0457
:1077C0000C944F2C82EE91E02BC9AC01401B510B65
:1077D0008A010C947D2C8E199F090C94862C809123
:1077E000C0049091C10401969093C1048093C00499
:1077F0000C94A02C19811B7F109334070C94B22C8D
:107800008091230790912407892BC1F58091CB04A7
:107810008E3780F109810460009334072091280796
:10782000309129078091C4069091C5066AE070E006
:107830000E94FB72CB01B9010E94B618AC01909373
:10784000C1068093C0062091CF043091D00490915E
:107850003407B90183E0769567958A95E1F7641757
:10786000750798F42D32314080F09460909334077E
:107870000C942C2D8F5F8093CB04D0CF1092CB042F
:1078800019811B7F10933407C9CF9B7FEFCF245CF6
:107890003F4F2417350710F00C94502D803514F00D
:1078A0000C94502D8F5F0C944E2D1092C2040C94AA
:1078B000502D4F925F926F927F928F929F92AF92D4
:1078C000BF92CF92DF92EF92FF920F931F93CF93CD
:1078D000DF93D09033074D2D4870D2FE54C02091D5
:1078E000AC063091AD068091AE069091AF06411185
:1078F00054C030931F0520931E0580901A05909068
:107900001B05A0901C05B0901D05C501B4012CED10
:1079100035E040E050E00E941B703093A3062093B6
:10792000A20680913907803309F03EC0E09024051B
:10793000F09025050091200510912105C0912205A8
:10794000D0912305209118053091190580911A02D4
:1079500090911B02482F5AE0259F400D112440931F
:10796000A1062130310509F466C1D0F1223031057C
:1079700009F4DEC12330310509F4FFC11092190565
:1079800010921805B3C08091AE069091AF064111D8
:1079900006C02091AC063091AD06820F931F9093E4
:1079A0001F0580931E05A9CF883169F4E0905A0520
:1079B000F0905B050091030610910406C0915405F8
:1079C000D0915505BFCFE0905C05F0905D0500912A
:1079D000050610910606C0915605D0915705B2CF05
:1079E000809116078C7F80931607ED2DE87020910B
:1079F000380530913905A9E1B0E00E943D70AB0136
:107A0000BC01D2FECBC0EE2309F4E7C01093A5065B
:107A10000093A40640931A0550931B0560931C0520
:107A200070931D0580911A0590911B05A0911C056E
:107A3000B0911D0584179507A607B70770F082E07F
:107A400090E090931B0280931A0240931A05509382
:107A50001B0560931C0570931D051092E1061092A2
:107A600017051092160580912507809315056FEF75
:107A700073E08FEF93E00E94181E6FEF73E08FEFBB
:107A800093E00E941C1D0E94E22A80913307982FE8
:107A90009E7F90933307909130079D7F909330079E
:107AA000982F9C7024E030E09C3049F020911A021D
:107AB00030911B022430310531F422E030E0309364
:107AC0001B0220931A0290912507923078F0982F8C
:107AD000947082FFA7C02091DF06222309F4A2C080
:107AE00081E090E090931905809318058091250717
:107AF000809315058091300780FD1092E10685FD89
:107B00001092E10683FD1092E1069091320791FDFB
:107B10001092E1069091310791111092E10681FFD8
:107B200006C080911B06811102C01092E10680916F
:107B3000E006882321F08091DF06811102C01092B7
:107B4000E10680913907803309F0A6C380912405AE
:107B500090912505845D9E4F20912E0730912F072F
:107B60008217930710F41092E1068091E10660E01D
:107B7000811101C061E086E1DF91CF911F910F91EA
:107B8000FF90EF90DF90CF90BF90AF909F908F903D
:107B90007F906F905F904F900C94900780912C078E
:107BA00090912D07E11193C320912E0730912F075B
:107BB0008217930790F59093A5068093A4068017EB
:107BC000910708F08CC32017310708F088C31FEF16
:107BD000811A910AA10AB10A11C080912E079091D1
:107BE0002F079093A5068093A4068017910708F0AD
:107BF00076C38FEF881A980AA80AB80A80921A05E5
:107C000090921B05A0921C05B0921D050BCF0FEFA3
:107C1000801A900AA00AB00AF1CF3093A5062093EB
:107C2000A406CDCF2091E00683FF47C3211158CF92
:107C3000911156CF5BCF81E08093E10610921A0537
:107C400010921B0510921C0510921D050E94E22A3D
:107C500080911F06909120068B3F2EE9920708F035
:107C600064C0B0E0A0E025E0880F991FAA1FBB1FE9
:107C70002A95D1F749E45FED63E170E08A019B0149
:107C8000081B190B2A0B3B0BC901B8012DEC35E081
:107C900040E050E00E941B70C901BC010E94181E08
:107CA00090E080E0C5391FE7D10748F485E99FE7F8
:107CB0008C1B9D0B68E170E00E94FB72CB01BC0144
:107CC0000E941C1D80911E0590911F05892B49F073
:107CD0008091160590911705019690931705809352
:107CE00016052091DD063091DE06809152059091B7
:107CF00053052817390730F083E090E09093190579
:107D00008093180580911605909117058D37910580
:107D100030F082E090E090931905809318058091EF
:107D20002507823008F0E2CE29CE90E080E0B5CF82
:107D30001092E10610921A0510921B0510921C0574
:107D400010921D0510921705109216058D2D806159
:107D50008093330770E060E090E080E00E94181E9E
:107D600070E060E090E080E00E941C1D6FEF73E027
:107D70008FEF93E00E94E51CD2CF21E02093E10633
:107D80008230910509F462C158F4009709F445C0A6
:107D9000019709F4E1C010921B0210921A02BDC0B3
:107DA0008330910509F414C20497A9F7809116074E
:107DB0008E7F82608093160700911F061091200627
:107DC000E0901E05F0901F05C80186549109E81641
:107DD000F90638F480911E07807319F0C8010E94DB
:107DE0004F1EC8018A5B9F4FE816F90618F0C801BC
:107DF0000E944F1E90E080E0C5393FE7D30748F46A
:107E000085E99FE78C1B9D0B68E170E00E94FB7287
:107E1000CB01BC010E941C1DD2C190911E07292FCD
:107E20002C70922E80911607222309F458C082608C
:107E300080931607809116078E7F80931607E09037
:107E40001F06F0902006C0901E05D0901F059701D8
:107E500026543109C216D30628F4907319F0C701CD
:107E60000E944F1EA090DD06B090DE06CE01865423
:107E70009109A816B90628F4992019F0CE010E949C
:107E8000531DC7018A5B9F4FC816D90618F0C7015A
:107E90000E944F1ECE018A5B9F4FA816B90618F0AC
:107EA000CE010E94531D10921A0510921B051092CC
:107EB0001C0510921D0590913307892F887092FD43
:107EC00010C081111DC080912C0790912D07801743
:107ED000910718F580912E0790912F0715C08D7F7F
:107EE000A7CF20912E0730912F072017310730F4AC
:107EF00021E030E030931B0220931A02882369F0BE
:107F000080912C0790912D078017910730F481E024
:107F100090E090931B0280931A020E94E22A209123
:107F2000DD063091DE0680915205909153052817A9
:107F3000390720F410921905109218059091250721
:107F400080911505981709F4D1CD933009F016CD1D
:107F5000843009F013CDCACD809116078C7F8093B1
:107F60001607C090DD06D090DE06D092A506C0921E
:107F7000A406E0901F06F090200660901E05709009
:107F80001F05C701865491096816790638F4809157
:107F90001E07807319F0C7010E944F1ECE01865440
:107FA0009109C816D90638F480911E078C7019F013
:107FB000CE010E94531DC7018A5B9F4F6816790648
:107FC00018F0C7010E944F1ECE018A5B9F4FC81652
:107FD000D90618F0CE010E94531D3FEF831A930A71
:107FE000A30AB30A80921A0590921B05A0921C0561
:107FF000B0921D052091380530913905A9E1B0E016
:108000000E943D7086169706A806B90670F082E0B9
:1080100090E090931B0280931A0210921A0510921E
:108020001B0510921C0510921D0580912C07909144
:108030002D078017910708F470CF80912E0790913B
:108040002F078017910708F468CFA5CE80911607F7
:108050008C7F80931607C0901F06D090200640901A
:108060001E0550901F05C6018654910948165906F1
:1080700038F480911E07807319F0C6010E944F1ECC
:108080006090DD067090DE06C7018654910968167F
:10809000790638F480911E078C7019F0C7010E9490
:1080A000531DC6018A5B9F4F4816590618F0C6013A
:1080B0000E944F1EC7018A5B9F4F6816790618F011
:1080C000C7010E94531D50E4851657E795065BE1F2
:1080D000A506B10468F48FEF881A980AA80AB80AAE
:1080E00080921A0590921B05A0921C05B0921D0566
:1080F0008091A4069091A50680179107E8F420913D
:108100005E0530915F05A9E1B0E00E943D700091ED
:108110001A0510911B0520911C0530911D050617AD
:1081200017072807390740F46C167D0628F0809160
:10813000330781608093330780913307282F28709D
:1081400082FD11C021112AC080912C0790912D072A
:108150008C179D0770F580912E0790912F078C1733
:108160009D0738F5DACE40912E0750912F07C701B1
:10817000845691094817590770F083E090E0909376
:108180001B0280931A0210921A0510921B0510927E
:108190001C0510921D05222309F4BFCE04E6E01A47
:1081A000F10880912C0790912D078E159F0508F4FA
:1081B000B4CE83E090E090931B0280931A02109259
:1081C0001A0510921B0510921C0510921D05A5CED4
:1081D00090911E07192F1C70712E80911607112384
:1081E00009F458C0816080931607809116078D7F2F
:1081F00080931607C0911F06D091200600911E059E
:1082000010911F059E01265431090217130728F407
:10821000907319F0CE010E944F1EC090DD06D090E1
:10822000DE06C70186549109C816D90628F47720BE
:1082300019F0C7010E94531DCE018A5B9F4F08179A
:10824000190718F0CE010E944F1EC7018A5B9F4F8D
:10825000C816D90618F0C7010E94531D2FEF821AC5
:10826000920AA20AB20A80921A0590921B05A09265
:108270001C05B0921D052091620530916305ACED9F
:10828000B5E00E943D7086169706A806B90608F06C
:1082900082CD43CE8E7FA7CF883129F480915A05B5
:1082A00090915B0557CC8C3029F480915C059091BE
:1082B0005D0550CC90E080E04DCC911117CC22238D
:1082C00009F414CC8091DF0681110ACC0FCC909375
:1082D000A5068093A4068017910708F498CC109205
:1082E0001A0510921B0510921C0510921D059ACBC1
:1082F000EF92FF920F931F93CF93DF937C018B013B
:108300000E94D36FD82FD801EC91F0E0E558FD4FD3
:10831000E081C82FCE27CC93C70101960E94D36F6E
:10832000EC2FF0E0E558FD4F90819827F8019083FD
:108330002D2F30E0322F2227820F932F911DDF91B6
:10834000CF911F910F91FF90EF9008952F923F9240
:108350004F925F926F927F928F929F92AF92BF9255
:10836000CF92DF92EF92FF920F931F93CF93DF9301
:10837000CDB7DEB767970FB6F894DEBF0FBECDBF9F
:108380008091C105813009F464C038F1823009F46C
:1083900008C1833009F4C4C78091C10590E00196FB
:1083A000837099278093C10567960FB6F894DEBF56
:1083B0000FBECDBFDF91CF911F910F91FF90EF9036
:1083C000DF90CF90BF90AF909F908F907F906F90F5
:1083D0005F904F903F902F9008958091C0058093BB
:1083E0003D0780933E072091BC053091BD0540912B
:1083F000BE055091BF0562E070E080E490E00E940D
:10840000930F882309F180918906811119C0809109
:10841000BA059091BB059093B9058093B80583E0A8
:1084200080933D072091BC053091BD054091BE056C
:108430005091BF0561E070E08BE090E00E94930FE7
:1084400081E080938906A8CF109289061092C0051A
:10845000A3CF10929F0610929E0610929D06109236
:108460009C0610929B0610929A0610929906809193
:108470008906882309F490CFE090B405F090B50503
:108480000091B6051091B70525E130E045E150E0D7
:108490006EE770E081E00E9474106531710581051E
:1084A000910509F079CF60914407862F90E0982FCD
:1084B000882760914307680F792F711D072E000CE4
:1084C000880B990B0E94B66E27E93FEF40E65FE309
:1084D0000E94156F6B017C0120E030E0A9010E9431
:1084E000617120E030E040E05FE387FD50C0C701EC
:1084F000B6010E944D700E942B7170939F0660938D
:108500009E0660913E07862F90E0982F8827609105
:108510003D07680F792F711D072E000C880B990BF2
:108520000E94B66E26EF38E24CE250E40E94156FCE
:108530006B017C0120E030E0A9010E94617120E024
:1085400030E040E05FE387FD27C0C701B6010E942D
:108550004D700E942B7170939D0660939C068091D4
:10856000500790E0982F882720914F07820F911D88
:1085700044E6489F9001499F300D112430939B069B
:1085800020939A06809151078093990605CFC701E1
:10859000B6010E944C70AFCFC701B6010E944C706B
:1085A000D8CF80911B0781118DC42091A2053091F5
:1085B000A3053B832A832130310509F074C3409120
:1085C0009C0650919D065F874E8723E333E343E388
:1085D0005FE360917F0B7091800B8091810B909194
:1085E000820B0E94156F6B017C01AE85BF85BD01BA
:1085F000BB0F880B990B0E94B66E2AE939E949E94D
:108600005EE30E94156F9B01AC01C701B6010E9499
:108610004D7060937F0B7093800B8093810B9093D0
:10862000820B00E010E0980140E050E068E472EC5A
:1086300083E89BE00E94990A83E89BE00E945F0424
:108640006091A0057091A10590E080E00E94B46E59
:108650002FE632E143E85AE30E94156F6C837D8375
:108660008E839F836093BF0B7093C00B8093C10B6D
:108670009093C20B60919E0570919F0590E080E001
:108680000E94B46E2FE632E143E85AE30E94156F70
:10869000688779878A879B876093C30B7093C40B25
:1086A0008093C50B9093C60B209118073091190742
:1086B0003D872C87B90190E080E00E94B46E6B0189
:1086C0007C01C092CF0BD092D00BE092D10BF092F4
:1086D000D20B60919C0570919D0590E080E00E9416
:1086E000B46E6093C70B7093C80B8093C90B9093C3
:1086F000CA0B2090BA053090BB056091A40570911B
:10870000A50590E080E00E94B46E4B015C01B101D0
:1087100090E080E00E94B46EAB01BC019501840141
:1087200083ED9BE00E94990A83ED9BE00E945F0429
:1087300061E070E083ED9BE00E94470A60919A053A
:1087400070919B0590E080E00E94B46E2CEA35ECBD
:1087500047E257E30E94156F688B798B8A8B9B8B5E
:1087600060930F0C7093100C8093110C9093120C6B
:10877000609198057091990590E080E00E94B46E38
:108780002CEA35EC47E257E30E94156F2B013C01C0
:108790004092130C5092140C6092150C7092160CAF
:1087A000609196057091970590E080E00E94B46E0C
:1087B0002CEA35EC47E257E30E94156F6C8B7D8BFA
:1087C0008E8B9F8B6093170C7093180C8093190CF1
:1087D00090931A0C80919405909195059093A9051A
:1087E0008093A80580919205909193059093AB0595
:1087F0008093AA0580919005909191059093AD0585
:108800008093AC054C855D85452B09F471C1809141
:108810001A0781116DC180918906882309F468C106
:108820002BE735EC4EE25AE3C701B6010E94156F03
:108830009B01AC010E94156F4B015C018C859D85ED
:108840008D3B924008F42FC120E030E048EC52EC20
:10885000C501B4010E94156F6093770B7093780B7C
:108860008093790B90937A0B61E070E083E89BE052
:108870000E94470A2091830B3091840B4091850B15
:108880005091860B6C817D818E819F810E94AF6E9D
:10889000811110C02091870B3091880B4091890B7A
:1088A00050918A0B688579858A859B850E94AF6E79
:1088B000882379F0C12CD12C7601088519852A8569
:1088C0003B854C815D816E817F8183E89BE00E94C6
:1088D0001A0B8091BD0B882321F083E89BE00E9456
:1088E000E5082AE939E949E95EE3C501B4010E94D6
:1088F000AF6E87FDEBC020E030E040E450E4C501FE
:10890000B4010E94617118162CF4812C912CF0E4B2
:10891000AF2EBA2CA5019401688979898A899B892F
:108920000E94156F6C837D838E839F8360930F0CF1
:108930007093100C8093110C9093120CA50194016C
:10894000C301B2010E94156F2B013C014092130C30
:108950005092140C6092150C7092160CA5019401A3
:108960006C897D898E899F890E94156F6B017C01BE
:10897000C092170CD092180CE092190CF0921A0CBD
:108980002091D30B3091D40B4091D50B5091D60B45
:108990006C817D818E819F810E94AF6E81111CC090
:1089A0002091D70B3091D80B4091D90B5091DA0B15
:1089B000C301B2010E94AF6E81110EC02091DB0B8A
:1089C0003091DC0B4091DD0B5091DE0BC701B601FD
:1089D0000E94AF6E882351F0930182014C815D812A
:1089E0006E817F8183ED9BE00E941A0B0E944512ED
:1089F00020917B0B30917C0B40917D0B50917E0B35
:108A00006091CB0B7091CC0B8091CD0B9091CE0BE4
:108A10000E944D706B017C0120E030E0A9010E94B2
:108A2000617120E030E040E05FE387FD57C0C7019F
:108A3000B6010E944D700E942B716215730540F0C3
:108A40002090A4053090A5056215730508F41B015C
:108A50003092B9052092B80580919E0690919F06AC
:108A60008215930508F03FC0281A390A21143104F1
:108A700059F040918E0550918F055B834A832416EF
:108A8000350610F43B822A828A819B819093AF0540
:108A90008093AE0580918C0590918D059093B105E2
:108AA0008093B005FCC01092BD0B1092770B109212
:108AB000780B1092790B10927A0B10927B0B10921C
:108AC0007C0B10927D0B10927E0BD4CEEAE98E2E99
:108AD000E9E99E2EA92CEEE3BE2E1CCFC701B601FC
:108AE0000E944C70A8CF9C01221933091901BECFF6
:108AF0001092BD0B1092770B1092780B1092790B9D
:108B000010927A0B10927B0B10927C0B10927D0BC3
:108B100010927E0B80E090E0AAE7B4EC8093C70B44
:108B20009093C80BA093C90BB093CA0B10920F0C73
:108B30001092100C1092110C1092120C20E030E0E8
:108B400040E05FE3C301B2010E94156F4B015C017D
:108B50008092130C9092140CA092150CB092160CEB
:108B60001092170C1092180C1092190C10921A0CEB
:108B700020E030E0A9016091D30B7091D40B80917B
:108B8000D50B9091D60B0E94AF6E81111DC0209124
:108B9000D70B3091D80B4091D90B5091DA0BC5010E
:108BA000B4010E94AF6E81110FC020E030E0A90136
:108BB0006091DB0B7091DC0B8091DD0B9091DE0BF3
:108BC0000E94AF6E882359F0C12CD12C76019501FB
:108BD0008401B701A60183ED9BE00E941A0B0E945D
:108BE0004512C090CB0BD090CC0BE090CD0BF09009
:108BF000CE0B20E030E0A901C701B6010E946171EF
:108C000020E030E040E05FE387FD3DC0C701B601F2
:108C10000E944D700E942B717093B9056093B80546
:108C200084E190E09093AF058093AE058AE090E0F8
:108C30009093B1058093B00580919E0690919F0618
:108C40002816390628F5DC01A219B3091D01B5E083
:108C50002B16310400F52E853F852F3C3F4F14F035
:108C60001092C0058091B305833009F466C208F400
:108C700048C2843009F4EAC28091B3058F5F8370E3
:108C80008093B30589CBC701B6010E944C70C2CF57
:108C9000281A390ADCCF5BE02516310418F381E08D
:108CA0008093C005DFCF8A819B810297E1F42091F8
:108CB0008A0530918B058091BA059091BB052817E4
:108CC000390740F08091A4059091A5052817390730
:108CD00008F4C9019093B9058093B80580918E0579
:108CE00090918F05D3CEAA81BB81AB2B09F0B8CF71
:108CF00020911807309119072115310509F49AC000
:108D000080911A07811196C080918905823008F4FC
:108D10008DC01092890580919C0590919D058217C8
:108D2000930710F1809187059091880544E6489F4C
:108D30009001499F300D11248091280790912907B7
:108D40002817390788F08091C4069091C506609174
:108D50008505709186052AE0269FA001279F500D6A
:108D6000112448175907B0F5809184052091B80562
:108D70003091B905811101C081E0281B3109809132
:108D8000BA059091BB052817390740F08091A405DA
:108D90009091A5052817390708F4C9019093B905E2
:108DA0008093B80580918E0590918F059093AF05C3
:108DB0008093AE0580918C0590918D059093B105BF
:108DC0008093B00581E08093C005109281051092D8
:108DD000800548CF6091820570918305269FA00190
:108DE000279F500D112484179507E0F68091840584
:108DF0002091B8053091B905811101C081E0820F41
:108E0000932F911D2091BA053091BB0582179307CE
:108E100040F02091A4053091A5058217930708F42E
:108E20009C013093B9052093B805BCCF8F5F809328
:108E30008905B8CF80918005909181058032910598
:108E400020F420911A072223D9F18091BA0590913C
:108E5000BB059093B9058093B80520918E0530919C
:108E60008F053093AF052093AE0520918C0530918E
:108E70008D053093B1052093B00520919E06309169
:108E80009F062817390770F0281B390B263031054B
:108E900090F41092C00580E290E090938105809359
:108EA0008005E0CE821B930B8630910590F34597A9
:108EB00008F4D8CE87CF2531310508F4D3CE82CF40
:108EC0000196EBCF84E090E09093AF058093AE05E0
:108ED00082E390E09093B1058093B005E091A705FF
:108EE000E83008F091C0F0E08827E658F84B8F4F43
:108EF0000C940F7382479247B747D14710483648C2
:108F000049487C481092C00581E080931A0720915F
:108F1000180730911907232BF1F58093A7051092BC
:108F2000A60572C081E08093C0058091A405909150
:108F3000A5052091BA053091BB05820F931F969528
:108F400087959093B9058093B80520919E0630913E
:108F50009F068217930740F4A901481B590BCA01C9
:108F60000597C8F482E0D9CF821B930BF9CF80918B
:108F70009C0690919D068139914024F01092C00585
:108F800083E0CBCF81E08093C00588E097E09093A9
:108F9000B9058093B8058091A6058F5F8093A605DB
:108FA00033C08091A6058330C0F380919E069091D6
:108FB0009F0601979093A5058093A4050E945327CF
:108FC0000E94DB1C81E08983BE016F5F7F4F84E7D5
:108FD00090E00E9478419093A5058093A405845663
:108FE00091098134964058F08091310781608093D7
:108FF00031078AE194E09093A5058093A40510922F
:10900000A60584E08093A7058091A605893C08F415
:1090100029CE10921B071092A7051092A60522CE0A
:1090200081E08093C0058091A4059091A5052091D1
:10903000BA053091BB05820F931F96958795909343
:10904000B9058093B80520919E0630919F0682173E
:10905000930748F4A901481B590BCA01059708F06A
:109060009ACF85E05ACF821B930BF8CF80919C0654
:1090700090919D0680379E4F24F41092C00586E0A3
:109080004CCF81E08093C0051092B9051092B805CD
:1090900082CF8091A605833008F47FCF80919E0611
:1090A00090919F0601969093BB058093BA050E940C
:1090B00053270E94DB1C81E08983BE016F5F7F4FD5
:1090C00086E790E00E9478419093BB058093BA05B3
:1090D000845691098D3D954058F08091310781600B
:1090E0008093310784E893E09093BB058093BA05A1
:1090F0001092A60587E086CF10921B071092A70555
:109100000ECFE090B405F090B5050091B605109132
:10911000B70521E030E041E050E066E470E081E036
:109120000E947410613071058105910509F0A4CD8C
:1091300080913D07809398069FCD0E941D27109235
:109140003D0781E080933E0780E180933F07809355
:109150004007809128079091290764E670E00E94FB
:10916000FB72709341076093420780913307282F69
:10917000287082FD0FC0211113C020912E0730915D
:109180002F0780912C0790912D072817390760F43D
:10919000C9010AC080912E0790912F07222321F048
:1091A00080912C0790912D0790934307809344075B
:1091B0008091AE069091AF062091AC063091AD063D
:1091C000820F931F909345078093460780919806DE
:1091D0008093470780919906809348078091AA065B
:1091E0009091AB069093490780934A07809123079B
:1091F0009091240790934B0780934C0780919E0693
:1092000090919F0690934D0780934E07EDE3F7E012
:1092100090E080E02191820F911DB7E0EF34FB07D1
:10922000C9F790934F07809350070E941D2744E190
:1092300050E06DE377E08CEA98E00E94F0048CEA5D
:1092400098E00E9422060E94321216CDEDE3F7E06C
:1092500086E497E011928E179F07E1F7E090B4053E
:10926000F090B5050091B6051091B70529E030E002
:1092700049E050E064E670E08AE00E9474106930D2
:10928000710581059105C9F580913E0790E0982F01
:10929000882720913D07820F911D90938F06809320
:1092A0008E068091400790E0982F882720913F07F5
:1092B000820F911D90938D0680938C0680914207BA
:1092C00090E0982F882720914107820F911D90935D
:1092D0009106809390068091430780939206809137
:1092E000450790E0982F882720914407820F911D11
:1092F00090938B0680938A06BFCC10928F061092B3
:109300008E0610928D0610928C0610929106109285
:1093100090061092920610928B0610928A06ACCCA0
:1093200080918906882309F437C88091B2058F5F40
:10933000853608F05AC08093B2058090BC059090A5
:10934000BD05A090BE05B090BF058091B2058823F1
:1093500009F453C09091B0058091B10590933D07F9
:1093600080933E0710923F07109240079091AE0500
:109370008091AF0590934107809342071092430775
:10938000109244076091B8057091B90590E080E0B3
:109390000E94B46E2EE633EA41E95FE30E94156F46
:1093A0006B017C0120E030E0A9010E94617120E0A6
:1093B00030E040E05FE387FD1BC0C701B6010E94BB
:1093C0004D700E942B716093450770934607109271
:1093D000470710924807A50194016CE070E08CE605
:1093E00090E00E94930F0C94CC411092B205A5CF4F
:1093F000C701B6010E944C70E4CF9091AC058091FA
:10940000AD0590933D0780933E079091AA0580910A
:10941000AB0590933F07809340079091A8058091FA
:10942000A905909341078093420710924307109239
:109430004407109245071092460710924707109272
:109440004807A50194016CE070E080E590E0C9CF89
:109450008F929F92AF92BF92CF92DF92EF92FF9244
:109460000F931F93CF93DF931F921F92CDB7DEB759
:109470001A8281E08983BE016F5F7F4F90E080E0B8
:109480000E94784190936B0580936A05893E9340D2
:1094900058F08091310781608093310782E390E03A
:1094A00090936B0580936A05BE016F5F7F4F82E0EA
:1094B00090E00E94784190931E0680931D06893C9F
:1094C0009F4A58F08091310781608093310780E492
:1094D0009CE990931E0680931D06BE016F5F7F4F2F
:1094E00084E090E00E94784190936905809368053C
:1094F0008897813C934058F0809131078160809338
:10950000310788E790E09093690580936805BE0174
:109510006F5F7F4F86E090E00E94784190936705EF
:10952000809366058536910558F0809131078160FA
:109530008093310785E090E09093670580936605FE
:10954000BE016F5F7F4F88E090E00E94784190936A
:10955000650580936405BE016F5F7F4F8AE090E0F0
:109560000E94784190930C0680930B0681329340C1
:1095700058F08091310781608093310788E592E04F
:1095800090930C0680930B06BE016F5F7F4F8CE0BB
:1095900090E00E9478419093630580936205813D3D
:1095A000974058F08091310781608093310788E6B9
:1095B00091E09093630580936205BE016F5F7F4FDA
:1095C0008EE090E00E947841909361058093600561
:1095D000813D974058F08091310781608093310739
:1095E00080ED92E09093610580936005BE016F5F0E
:1095F0007F4F80E190E00E94784190935F058093D7
:109600005E05813D974058F08091310781608093DD
:1096100031078FE090E090935F0580935E05BE0177
:109620006F5F7F4F82E190E00E94784190935D05EB
:1096300080935C05885293428137974158F080911E
:1096400031078160809331078CED97E390935D053E
:1096500080935C05BE016F5F7F4F84E190E00E94C4
:10966000784190935B0580935A05885293428930E4
:10967000924558F08091310781608093310788EBE3
:109680009FE690935B0580935A05BE016F5F7F4F05
:1096900086E190E00E9478419093590580935805A7
:1096A00081369A4E58F0809131078160809331075E
:1096B00080ED97E09093590580935805BE016F5F48
:1096C0007F4F88E190E00E94784190935705809306
:1096D0005605885293428137974158F0809131075F
:1096E00081608093310788EE95E3909357058093CE
:1096F0005605BE016F5F7F4F8AE190E00E9478417E
:109700009093550580935405885293428930924531
:1097100058F08091310781608093310780ED9BE69E
:109720009093550580935405BE016F5F7F4F8CE188
:1097300090E00E94784190935305809352058136C2
:109740009A4E58F08091310781608093310788E20A
:1097500093E29093530580935205BE016F5F7F4F54
:109760008EE190E00E947841909306068093050672
:10977000885293428137974158F080913107816038
:109780008093310780E092E390930606809305066C
:10979000BE016F5F7F4F80E290E00E94784190931E
:1097A000040680930306885293428930924558F00C
:1097B0008091310781608093310780E094E6909337
:1097C000040680930306BE016F5F7F4F82E290E044
:1097D0000E9478419093150780931407813A9F4027
:1097E00058F0809131078160809331078EEE92E0CE
:1097F0009093150780931407BE016F5F7F4F84E23B
:1098000090E00E9478419093220780932107813A4B
:109810009F4058F08091310781608093310786E93D
:1098200090E09093220780932107BE016F5F7F4FE6
:1098300086E290E00E947841909351058093500514
:10984000853B934C58F080913107816080933107BC
:1098500080E49CE99093510580935005BE016F5FB1
:109860007F4F88E290E00E94784190932306809396
:1098700022068D3B924058F08091310781608093A1
:10988000310788E592E09093230680932206BE017B
:109890006F5F7F4F8AE290E00E94784190934F057E
:1098A00080934E05813A9C4F58F08091310781603A
:1098B0008093310780E49FE190934F0580934E059C
:1098C000BE016F5F7F4F8CE290E00E9478419093E1
:1098D0004D0580934C05813A9C4F58F0809131079B
:1098E00081608093310780E49FE190934D058093E0
:1098F0004C05BE016F5F7F4F8EE290E00E94784181
:1099000090934B0580934A05813A9C4F58F0809183
:10991000310781608093310780E49FE190934B058C
:1099200080934A05BE016F5F7F4F80E390E00E9405
:1099300078419093FF058093FE0580549F418136C6
:109940009D4D58F08091310781608093310780EC04
:109950009AED9093FF058093FE05BE016F5F7F4FE8
:1099600082E390E00E947841909302068093010682
:1099700080549F4181369D4D58F080913107816020
:109980008093310780E69AEE909302068093010659
:10999000BE016F5F7F4F84E390E00E947841909317
:1099A000490580934805813A9C4F58F080913107D2
:1099B00081608093310780E49FE190934905809313
:1099C0004805BE016F5F7F4F86E390E00E947841BB
:1099D0009093F9058093F805853F914058F0809168
:1099E000310781608093310784E690E09093F90518
:1099F0008093F805BE016F5F7F4F88E390E00E947F
:109A000078419093F5058093F4058B3F910558F0CC
:109A10008091310781608093310782E390E09093D9
:109A2000F5058093F405BE016F5F7F4F8AE390E0F8
:109A30000E9478419093FB058093FA05893E9340FC
:109A400058F08091310781608093310784E690E07F
:109A50009093FB058093FA05BE016F5F7F4F8CE307
:109A600090E00E9478419093250680932406893ED9
:109A7000934058F08091310781608093310780E2F4
:109A800093E09093250680932406BE016F5F7F4F7D
:109A90008EE390E00E9478419093450580934405C1
:109AA000BE016F5F7F4F80E490E00E947841909309
:109AB000430580934205BE016F5F7F4F82E490E0D3
:109AC0000E9478419093410580934005BE016F5FED
:109AD0007F4F84E490E00E94784190933F0580930B
:109AE0003E05BE016F5F7F4F86E490E00E947841A3
:109AF0009093470580934605459758F0809131072C
:109B000081608093310785E090E0909347058093D2
:109B10004605BE016F5F7F4F88E490E00E94784168
:109B200090933D0580933C05813A9C4F58F080917D
:109B3000310781608093310788E893E190933D0578
:109B400080933C05BE016F5F7F4F8AE490E00E94E6
:109B5000784190933B0580933A05813A9F4058F0B5
:109B60008091310781608093310788EC90E0909379
:109B70003B0580933A05BE016F5F7F4F8CE490E018
:109B80000E9478419093390580933805813B944039
:109B900058F0809131078160809331078CE291E029
:109BA0009093390580933805BE016F5F7F4F8EE437
:109BB00090E00E9478419093370580933605BE016E
:109BC0006F5F7F4F80E590E00E947841909335056C
:109BD00080933405BE016F5F7F4F82E590E00E9465
:109BE00078419093E3068093E206039748F08091D2
:109BF00031078160809331071092E3061092E206EC
:109C0000BE016F5F7F4F84E590E00E9478419093A2
:109C10003305809332058F3F910561F058F08091B4
:109C2000310781608093310783E090E090933305A2
:109C300080933205BE016F5F7F4F86E590E00E9402
:109C400078419093310580933005889789379F40FC
:109C500058F08091310781608093310788E790E068
:109C60009093310580933005BE016F5F7F4F88E58B
:109C700090E00E94784190932F0580932E058536C1
:109C8000910558F08091310781608093310785E01C
:109C900090E090932F0580932E05BE016F5F7F4F5C
:109CA0008AE590E00E94784190932D0580932C05E1
:109CB000BE016F5F7F4F8CE590E00E9478419093EA
:109CC0000F0680930E068536910558F08091310776
:109CD00081608093310784E690E090930F06809333
:109CE0000E06BE016F5F7F4F8EE590E00E947841C7
:109CF00090931D0780931C07019649F480913107CA
:109D000081608093310710921D0710921C07BE01DD
:109D10006F5F7F4F80E690E00E94784190936F05DF
:109D200080936E05019649F480913107816080939C
:109D3000310710926F0510926E05BE016F5F7F4F65
:109D400082E690E00E94784190936D0580936C05C7
:109D5000019649F480913107816080933107109218
:109D60006D0510926C05BE016F5F7F4F84E690E039
:109D70000E9478419093150680931406885293426E
:109D8000893B9B4058F08091310781608093310777
:109D90008CEE9CE29093150680931406BE016F5FD3
:109DA0007F4F86E690E00E9478419093130680935F
:109DB000120680519742813A9F4058F080913107B6
:109DC00081608093310788E19EE29093130680932F
:109DD0001206BE016F5F7F4F88E690E00E947841D7
:109DE0009093110680931006805E9E42813A9F40B8
:109DF00058F08091310781608093310780E092E3D1
:109E00009093110680931006BE016F5F7F4F8AE624
:109E100090E00E9478419093250580932405885214
:109E200093428933974C58F0809131078160809339
:109E3000310780E79FED9093250580932405BE01AF
:109E40006F5F7F4F8CE690E00E94784190932305EE
:109E500080932205885293428933974C58F0809121
:109E6000310781608093310780EA97ED9093230555
:109E700080932205BE016F5F7F4F8EE690E00E94C7
:109E8000784190932105809320058852934289332D
:109E9000974C58F08091310781608093310780E0C2
:109EA00098EC9093210580932005BE016F5F7F4F52
:109EB00080E790E00E94784180933807833038F043
:109EC0008091310781608093310710923807BE017D
:109ED0006F5F7F4F82E790E00E9478419093A305E7
:109EE0008093A205049758F0809131078160809398
:109EF000310781E090E09093A3058093A205BE0115
:109F00006F5F7F4F84E790E00E9478419093A505B2
:109F10008093A405845691098134964058F080912D
:109F200031078160809331078AE194E09093A50521
:109F30008093A405BE016F5F7F4F86E790E00E948B
:109F400078419093BB058093BA05845691098D3D65
:109F5000954058F08091310781608093310784E803
:109F600093E09093BB058093BA05BE016F5F7F4F6E
:109F700088E790E00E947841809384058150883C76
:109F800040F0809131078160809331078AE08093AF
:109F90008405BE016F5F7F4F8AE790E00E947841A1
:109FA00090938805809387058732924058F080917E
:109FB000310781608093310784EF91E090938805A9
:109FC00080938705BE016F5F7F4F8CE790E00E9412
:109FD000784190932B0580932A058732924058F060
:109FE0008091310781608093310788EC90E09093F5
:109FF0002B0580932A05BE016F5F7F4F8EE790E0AF
:10A000000E94784190939D0580939C0589389341E7
:10A0100058F08091310781608093310780E496E0A9
:10A0200090939D0580939C05BE016F5F7F4F80E8F4
:10A0300090E00E9478419093290580932805893803
:10A04000934158F08091310781608093310784E813
:10A0500093E09093290580932805BE016F5F7F4FA1
:10A0600082E890E00E947841909386058093850570
:10A070008935924058F08091310781608093310793
:10A0800086E292E09093860580938505BE016F5F1E
:10A090007F4F84E890E00E947841909383058093FD
:10A0A00082058935924058F0809131078160809314
:10A0B00031078CE291E09093830580938205BE0185
:10A0C0006F5F7F4F86E890E00E94784190939B05F8
:10A0D00080939A05BE016F5F7F4F88E890E00E94F1
:10A0E00078419093990580939805BE016F5F7F4FEB
:10A0F0008AE890E00E9478419093970580939605B6
:10A10000BE016F5F7F4F8CE890E00E947841909392
:10A110008D0580938C0597FF0BC08091310781607E
:10A120008093310784E690E090938D0580938C05B1
:10A13000BE016F5F7F4F8EE890E00E947841909360
:10A140008F0580938E0597FF0BC08091310781604A
:10A150008093310784E690E090938F0580938E057D
:10A16000BE016F5F7F4F80E990E00E94784190933D
:10A170002705809326058131974258F08091310759
:10A1800081608093310788EE93E090932705809358
:10A190002605BE016F5F7F4F82E990E00E94784103
:10A1A00090938B0580938A0581319E4058F0809171
:10A1B000310781608093310780E293E090938B05B3
:10A1C00080938A05BE016F5F7F4F84E990E00E9413
:10A1D000784190939505809394058115904458F0AB
:10A1E0008091310781608093310780E49FE19093F3
:10A1F000950580939405BE016F5F7F4F86E990E0DF
:10A200000E94784190939305809392058115904424
:10A2100058F08091310781608093310780EE9EE293
:10A220009093930580939205BE016F5F7F4F88E9FD
:10A2300090E00E947841909391058093900581155C
:10A24000904448F0809131078160809331071092EB
:10A25000910510929005BE016F5F7F4F8AE990E0F3
:10A260000E9478419093A1058093A005BE016F5F85
:10A270007F4F8CE990E00E94784190939F058093F6
:10A280009E05E981F0E0E558FD4F80818983BE019C
:10A290006E5F7F4F8CEA90E00E9478419981981719
:10A2A00009F49EC122E330E030936B0520936A05E8
:10A2B00060E47CE970931E0660931D0698E7A92E62
:10A2C000B12CB0926905A0926805E5E0F0E0F0934A
:10A2D0006705E0936605109265051092640548E5F0
:10A2E00052E050930C0640930B06A8E6B1E0B09301
:10A2F0006305A0936205A0EDB2E0B0936105A09361
:10A3000060050FE010E010935F0500935E05ACED73
:10A31000B7E3B0935D05A0935C05A8EBBFE6B093EF
:10A320005B05A0935A05A0E7BFEDB0932505A09368
:10A330002405A0EDB7E0B0935905A0935805A8EE09
:10A34000B5E3B0935705A0935605A0EDBBE6B093D7
:10A350005505A0935405A0EAB7EDB0932305A0934B
:10A360002205A8E2B3E2B0935305A0935205C12C95
:10A37000A2E3DA2ED0920606C0920506A0E0B4E66B
:10A38000B0930406A0930306A0E0B8ECB0932105B7
:10A39000A0932005AEEEB2E0B0931507A09314078A
:10A3A000A6E9B0E0B0932207A0932107709351056E
:10A3B00060935005509323064093220640E45FE1EA
:10A3C00050934F0540934E0550934D0540934C05D7
:10A3D00050934B0540934A0560EC7AED7093FF056E
:10A3E0006093FE0560E67AEE7093020660930106C4
:10A3F000509349054093480564E670E07093F90571
:10A400006093F8053093F5052093F4057093FB05F0
:10A410006093FA05A0E2B3E0B0932506A09324066A
:10A4200028EC30E0309345052093440530934305F4
:10A430002093420590E9E92EFF24F394F092410520
:10A44000E092400530933F0520933E05F093470589
:10A45000E093460598E8E92E93E1F92EF0923D0548
:10A46000E0923C0530933B0520933A059CE2E92EAF
:10A47000FF24F394F0923905E092380510923705E5
:10A480001092360530933505209334051092E3067B
:10A490001092E20693E0892E912C909233058092DF
:10A4A0003205B0923105A0923005F0932F05E0936C
:10A4B0002E0510922D0510922C0570930F066093B7
:10A4C0000E069CEEA92E9CE2B92EB0921506A09223
:10A4D000140698E1A92E9EE2B92EB0921306A0921E
:10A4E0001206D0921106C092100610923807CC24A2
:10A4F000C394D12CD092A305C092A2059AE1C92E93
:10A5000094E0D92ED092A505C092A40594E8C92E56
:10A5100093E0D92ED092BB05C092BA059AE09093F1
:10A52000840594EFA92EBB24B394B0928805A09221
:10A53000870530932B0520932A0520E436E03093DD
:10A540009D0520939C05D0922905C092280526E2FE
:10A5500032E03093860520938505F0928305E092E2
:10A56000820510939B0500939A052EE630E0309308
:10A5700099052093980523E230E0309397052093C6
:10A58000960570938D0560938C0570938F0560938D
:10A590008E0528EE33E03093270520932605B093EF
:10A5A0008B05A0938A05509395054093940520EE62
:10A5B0003EE23093930520939205109291051092FC
:10A5C0009005F093A105E093A00529E130E03093D8
:10A5D0009F0520939E0590913107926090933107DB
:10A5E000809340040F900F90DF91CF911F910F91B6
:10A5F000FF90EF90DF90CF90BF90AF909F908F90A3
:10A600000895CF92DF92EF92FF920F931F93CF9313
:10A61000DF93CDB7DEB76D970FB6F894DEBF0FBEF0
:10A62000CDBF40E051EE60E070E08DE098E00E9428
:10A63000950480EA93E00E94222A8BEB93E00E942B
:10A64000222A0E942718109285061092F70610926F
:10A65000E6061092E5061092E4061092E8061092C3
:10A66000E706109284061092830640E052EC61E007
:10A6700070E080E797E00E9495046AE070E080E077
:10A6800090E00E94350868EC73E080E797E00E9454
:10A69000182A62E370E080E090E00E94350881E0D3
:10A6A00089838E010F5F1F4FB8018EE590E00E94F5
:10A6B000784190931D0780931C07019649F480917F
:10A6C000310781608093310710921D0710921C079B
:10A6D00080911C0790911D07198E188E1B8E1A8E63
:10A6E0001D8E1C8E4AE0B8010E94856EF801019013
:10A6F0000020E9F73197AF01401B510BB801CE01A3
:10A7000048960E94A22A8C8D9D8D1B8A1A8A1D8ACA
:10A710001C8A1F8A1E8A069708F04CC041E050E050
:10A7200061ED73E0CE0142960E94A22ABE01685EEE
:10A730007F4FCE0142960E946F2A1A8219821C8294
:10A740001B821E821D82BC01C8010E94C32A888D03
:10A75000998D0097F1F069817A8161157105B9F0E1
:10A760004A8D5B8D2D813E814217530780F00E94F8
:10A7700026758D819E819D8F8C8F1E821D82C801C2
:10A780000E94DA2ACE0142960E94DA2ABCCF0E94A9
:10A79000B37389819A81998F888F8B819C819B8FDC
:10A7A0008A8F8D819E819D8F8C8F1A8219821C8247
:10A7B0001B82E3CF4DE050E063ED73E0CE014296A3
:10A7C0000E94A22ABE01685E7F4FCE0142960E947F
:10A7D0006F2A1A8219821C821B821E821D82BC0172
:10A7E000C8010E94C32A4D815E8169817A8180E718
:10A7F00097E00E94F004C8010E94DA2ACE01429636
:10A800000E94DA2A6AE070E080E090E00E94350859
:10A810001B8A1A8A1D8A1C8A1F8A1E8A4DE050E0F4
:10A8200061EE73E0CE0142960E94A22ABE01685EEC
:10A830007F4FCE0142960E946F2A1A8219821C8293
:10A840001B821E821D82BC01C8010E94C32A4D8149
:10A850005E8169817A8180E797E00E94F004C801F7
:10A860000E94DA2ACE0142960E94DA2A6AE070E05B
:10A8700080E090E00E9435086FEE73E080E797E09B
:10A880000E94182A6AE070E080E090E00E9435089B
:10A8900080E797E00E946705892B29F080E797E021
:10A8A0000E944505F5CF6AE070E080E090E00E94EC
:10A8B000350811E010938506CE0148960E94DA2AE9
:10A8C00010922D0710922C0710922F0710922E072E
:10A8D0001092AF061092AE061092AD061092AC0622
:10A8E0001092DE061092DD061092A5061092A406C4
:10A8F0001092E1061092B9061092B8061092B106B5
:10A900001092B0061092A3061092A2061092BF06F3
:10A910001092BE061092B7061092B6061092BD06AF
:10A920001092BC061092B5061092B4061092BB06A7
:10A930001092BA061092B3061092B20610921E0739
:10A9400020E43CE93093200620931F061092C906AC
:10A950001092C80662E370E070936B0560936A051D
:10A9600030931E0620931D06A8E7B0E0B09369055A
:10A97000A093680545E050E0509367054093660555
:10A980001092650510926405E8E5F2E0F0930C067C
:10A99000E0930B0688E691E090936305809362054F
:10A9A00080ED92E090936105809360058FE090E0E8
:10A9B00090935F0580935E058CED97E390935D0522
:10A9C00080935C0588EB9FE690935B0580935A0526
:10A9D00080E79FED909325058093240580ED97E017
:10A9E000909359058093580588EE95E39093570509
:10A9F0008093560580ED9BE6909355058093540512
:10AA000080EA97ED909323058093220588E293E2F4
:10AA1000909353058093520580E092E3909306064D
:10AA20008093050680E094E69093040680930306E5
:10AA300080E098EC909321058093200588EC90E0CD
:10AA40009093450580934405909343058093420578
:10AA500000E9E02EFF24F394F0924105E0924005D6
:10AA600090933F0580933E0510923705109236056E
:10AA700090933505809334050CE2E02EFF24F39487
:10AA8000F0923905E09238051092E3061092E20642
:10AA900003E0E02EF12CF0923305E0923205B09302
:10AAA0003105A093300550932F0540932E05109249
:10AAB0002D0510922C0510921F0510921E05109264
:10AAC0000F05109214051092E0061092DF06109206
:10AAD000240710922307109219071092180710925A
:10AAE000D3051092D20510922907109228071092D0
:10AAF000200710921F0710922B0710922A0710931D
:10AB000026071092270710922507ACE0A09339077B
:10AB10001092C5061092C4061092C1061092C0068B
:10AB2000AEEEB2E0B0931507A0931407A6E9B0E02B
:10AB3000B0932207A093210730935105209350052D
:10AB4000F0932306E093220620E43FE130934F0583
:10AB500020934E0530934D0520934C0530934B05C3
:10AB600020934A05E0ECFAEDF093FF05E093FE0533
:10AB7000E0E6FAEEF0930206E09301063093490511
:10AB800020934805509347054093460528E833E154
:10AB900030933D0520933C0590933B0580933A0507
:10ABA000109230071092310710923207109233073B
:10ABB00010923407109235071092160710921B0658
:10ABC00010923B0710923C0788EF9FE19093A906F3
:10ABD0008093A80680E090E69093A7068093A6064F
:10ABE0001092AB061092AA0688EE93E09093F705B8
:10ABF0008093F60584E690E09093F9058093F8053C
:10AC00007093F5056093F4059093FB058093FA0526
:10AC100020E233E0309325062093240690930F061C
:10AC200080930E0610921D0710921C0710926F055C
:10AC300010926E0510926D0510926C05A89580918A
:10AC400060008861809360008AE0809360001092C9
:10AC50004004279A15B860E087E30E94BE0760E0D1
:10AC600086E30E94BE0760E088E30E94BE0760E0C2
:10AC700089E30E94BE0760E08AE30E94BE0760E0AD
:10AC80008BE30E94BE0760E08CE30E94BE0760E099
:10AC90008DE30E94BE0760E08EE30E94BE0760E085
:10ACA0008FE30E94BE0760E080E40E94BE0760E080
:10ACB00081E40E94BE0760E082E40E94BE0760E07B
:10ACC00083E40E94BE0760E084E40E94BE0760E067
:10ACD00085E40E94BE0760E08CE10E94BE0760E050
:10ACE00086E20E94BE0760E08FE00E94BE071092DD
:10ACF0000401109205016F9861E08BE00E94BE078D
:10AD000061E08CE00E94BE0761E08DE00E94BE071A
:10AD100061E086E00E94BE0761E087E00E94BE0716
:10AD200061E088E00E94BE0761E08EE20E94BE07FB
:10AD300061E08DE20E94BE0761E08CE20E94BE07E6
:10AD400061E084E00E94BE0780E48AB98BB961E0CB
:10AD50008AE20E94BE0761E086E10E94BE0761E0D0
:10AD600087E10E94BE0761E088E10E94BE0761E0C2
:10AD70008FE10E94BE0761E08EE10E94BE0761E0A4
:10AD80008AE10E94BE0761E08BE10E94BE0761E09C
:10AD900085E50E94BE0761E086E10E94900761E0C0
:10ADA00087E10E94900710921E0283E284BD15BDC8
:10ADB00080E888BD3BEA3093800029E02093810041
:10ADC000109289001092880010928B0010928A00D5
:10ADD00010928D0010928C001092B00087E080934A
:10ADE000B10082EB8093B2001092900083EC8093CC
:10ADF00091003093A0002093A1008FEF93E09093F7
:10AE0000A9008093A8009093AB008093AA00909330
:10AE1000AD008093AC0030932001209321019093EA
:10AE200029018093280190932B0180932A0190930C
:10AE30002D0180932C010E94284A0E94284A0E94DA
:10AE40005327809170008160809370008091710021
:10AE500081628093710078940E94DB1C0E94321200
:10AE600040E051EE60E070E085E39BE00E94FD1160
:10AE700080E090E0A0E0B0E480934B0990934C090F
:10AE8000A0934D09B0934E09EDE3F7E08FE697E00C
:10AE900011928E179F07E1F784E091E0A0E0B0E007
:10AEA0008093BC059093BD05A093BE05B093BF05EC
:10AEB00088E592E0A0E0B0E08093B4059093B505FA
:10AEC000A093B605B093B70520E43FE13093A90500
:10AED0002093A8053093AB052093AA051092AD05E9
:10AEE0001092AC058091BA059091BB059093B9057D
:10AEF0008093B80582E090E09093AF058093AE0513
:10AF00009093B1058093B0051092C00581E090E068
:10AF10009093A3058093A2058AE194E09093A50500
:10AF20008093A40584E893E09093BB058093BA05D1
:10AF30004AE04093840544EF51E0509388054093E4
:10AF4000870548EC50E050932B0540932A059093D9
:10AF500029058093280540E456E050939D054093D1
:10AF60009C0546E252E050938605409385054CE2ED
:10AF700051E050938305409382054FE050E0509399
:10AF80009B0540939A054EE650E0509399054093F7
:10AF9000980543E250E0509397054093960545E0AD
:10AFA00050E05093A1054093A00530939505209360
:10AFB000940520EE3EE23093930520939205109283
:10AFC00091051092900524E630E030938D05209392
:10AFD0008C0530938F0520938E0528EE33E0309357
:10AFE00027052093260520E233E030938B0520933C
:10AFF0008A0590939F0680939E0610929D0610925C
:10B000009C06109299061092980610929B06109238
:10B010009A061092890681E080931A0710921B0706
:10B0200010928F0610928E0610928D0610928C064A
:10B0300010929106109290061092920610928B0632
:10B0400010928A0681E599E4ADE1B9E380930F0C93
:10B050009093100CA093110CB093120C80EE9DE213
:10B06000A0E9BAE38093130C9093140CA093150CF1
:10B07000B093160C84E390E8A7EBB9E38093170C28
:10B080009093180CA093190CB0931A0C1092CF0B3C
:10B090001092D00B1092D10B1092D20B1092C70BC2
:10B0A0001092C80B1092C90B1092CA0B80E090E06E
:10B0B000A1E6B4E48093CB0B9093CC0BA093CD0B83
:10B0C000B093CE0B6091010C7091020C8091030C37
:10B0D0009091040C0E94B46E9B01AC0160E070E59D
:10B0E00081E995E40E94B9706B017C01AC019B0180
:10B0F0006091E30B7091E40B8091E50B9091E60B6E
:10B100000E94156F6093E30B7093E40B8093E50B43
:10B110009093E60BA70196016091E70B7091E80B05
:10B120008091E90B9091EA0B0E94B9706093E70B54
:10B130007093E80B8093E90B9093EA0B8AE292E11B
:10B14000A0E0B0E08093010C9093020CA093030C5C
:10B15000B093040C8BE097EDA3EABBE38093BF0BA5
:10B160009093C00BA093C10BB093C20B60919E054E
:10B1700070919F0590E080E00E94B46E2FE632E16E
:10B1800043E85AE30E94156F6093C30B7093C40B9E
:10B190008093C50B9093C60B10927F0B1092800B7F
:10B1A0001092810B1092820B1092770B1092780BF9
:10B1B0001092790B10927A0B10927B0B10927C0BF1
:10B1C00010927D0B10927E0B83E080933D0724E06C
:10B1D00031E040E050E061E070E08BE090E00E9400
:10B1E000930F81111BC080913A078230B9F0109201
:10B1F0003A070E94271888EF93E00E94222A6D9652
:10B200000FB6F894DEBF0FBECDBFDF91CF911F9177
:10B210000F91FF90EF90DF90CF90089582E08093A0
:10B220003A0789E194E0E9CF1F920F920FB60F928F
:10B2300011240BB60F922F933F934F935F936F930D
:10B240007F938F939F93AF93BF93EF93FF938CEA7A
:10B2500098E00E94B305FF91EF91BF91AF919F914C
:10B260008F917F916F915F914F913F912F910F90AF
:10B270000BBE0F900FBE0F901F9018951F920F924C
:10B280000FB60F9211240BB60F922F933F934F934B
:10B290005F936F937F938F939F93AF93BF93EF933E
:10B2A000FF938CEA98E00E941D05FF91EF91BF91FA
:10B2B000AF919F918F917F916F915F914F913F914E
:10B2C0002F910F900BBE0F900FBE0F901F901895EF
:10B2D0001F920F920FB60F9211240BB60F922F935D
:10B2E0003F934F935F936F937F938F939F93AF930E
:10B2F000BF93EF93FF9380E797E00E94B305FF9120
:10B30000EF91BF91AF919F918F917F916F915F91DD
:10B310004F913F912F910F900BBE0F900FBE0F904A
:10B320001F9018951F920F920FB60F9211240BB613
:10B330000F922F933F934F935F936F937F938F93CE
:10B340009F93AF93BF93EF93FF9380E797E00E94A3
:10B350001D05FF91EF91BF91AF919F918F917F91CB
:10B360006F915F914F913F912F910F900BBE0F9076
:10B370000FBE0F901F9018951F920F920FB60F924D
:10B3800011240BB60F922F933F934F935F936F93BC
:10B390007F938F939F93AF93BF93EF93FF938DE032
:10B3A00098E00E94B305FF91EF91BF91AF919F91FB
:10B3B0008F917F916F915F914F913F912F910F905E
:10B3C0000BBE0F900FBE0F901F9018951F920F92FB
:10B3D0000FB60F9211240BB60F922F933F934F93FA
:10B3E0005F936F937F938F939F93AF93BF93EF93ED
:10B3F000FF938DE098E00E941D05FF91EF91BF91B2
:10B40000AF919F918F917F916F915F914F913F91FC
:10B410002F910F900BBE0F900FBE0F901F9018959D
:10B420001F920F920FB60F9211242F933F938F9379
:10B430009F93AF93BF938091D6059091D705A0912C
:10B44000D805B091D9053091D50526E0230F2D37C9
:10B4500058F50296A11DB11D2093D5058093D60500
:10B460009093D705A093D805B093D9058091DA05BC
:10B470009091DB05A091DC05B091DD050196A11D41
:10B48000B11D8093DA059093DB05A093DC05B093A2
:10B49000DD05BF91AF919F918F913F912F910F90BB
:10B4A0000FBE0F901F90189529E8230F0396A11D3A
:10B4B000B11DD2CF1F920F920FB60F9211248F930E
:10B4C0009F938FEF9FEF9093C7058093C6059F9141
:10B4D0008F910F900FBE0F901F9018951F920F9293
:10B4E0000FB60F9211248F939F93809196009091A5
:10B4F00097009093C7058093C6051092950010920F
:10B5000094009F918F910F900FBE0F901F901895F0
:10B510001F920F920FB60F9211248F9382EB80939C
:10B52000B2008FEF80933C078F910F900FBE0F906A
:10B530001F901895AF92BF92CF92DF92EF92FF9239
:10B540000F931F93CF93DF93CCEAD8E01B821A822C
:10B5500048EE53E060E070E04C835D836E837F8350
:10B560008FE793E09983888325ED30E03D872C8732
:10B5700024ED30E03F872E8720ED30E0398B288B9B
:10B5800021ED30E03B8B2A8B22ED30E03D8B2C8B84
:10B5900026ED30E03F8B2E8B198E1A8E1B8E1C8E63
:10B5A000E0E7F7E013821282448355836683778352
:10B5B000918380832DEC30E0358724872CEC30E0BC
:10B5C0003787268728EC30E0318B208B29EC30E060
:10B5D000338B228B2AEC30E0358B248B2EEC30E041
:10B5E000378B268B118E128E138E148EEDE0F8E0C1
:10B5F0001382128244835583668377839183808389
:10B6000085EC90E09587848784EC90E09787868727
:10B6100080EC90E0918B808B81EC90E0938B828B1F
:10B6200082EC90E0958B848B86EC90E0978B868BF8
:10B63000118E128E138E148EA090130CB090140CD9
:10B64000C090150CD090160CE0900F0CF090100CE0
:10B650000091110C1091120C80911A0C8F93809113
:10B66000190C8F938091180C8F938091170C8F93E6
:10B6700027EC3BE04BEC5BE06FEC7BE083ED9BE089
:10B680000E941A26A090C30BB090C40BC090C50BAB
:10B69000D090C60BE090BF0BF090C00B0091C10B97
:10B6A0001091C20B1F921F921F921F9227E73BE03F
:10B6B0004BE75BE06FE77BE083E89BE00E941A26A4
:10B6C000E9E4F9E01092320B1092340B1092330B34
:10B6D000168E80E090E0A0E0B0E482839383A483A0
:10B6E000B58381E08683108688EC818780E291EAC9
:10B6F000A7E0B0E082879387A487B587868797877E
:10B70000A08BB18B178E10A211A21092370BA5E35C
:10B71000BBE081E993E011969C938E93D093390B13
:10B72000C093380B8EE190E090933B0B80933A0BE3
:10B730008FE190E090933D0B80933C0B40E051EE05
:10B7400060E070E040933E0B50933F0B6093400BE2
:10B750007093410BB093AB08A093AA08B183A08368
:10B760008DB79EB708960FB6F8949EBF0FBE8DBFDB
:10B77000DF91CF911F910F91FF90EF90DF90CF90CD
:10B78000BF90AF900895789484B5826084BD84B5ED
:10B79000816084BD85B5826085BD85B5816085BDCC
:10B7A00080916E00816080936E0010928100809184
:10B7B000810082608093810080918100816080930C
:10B7C0008100809180008160809380008091B10031
:10B7D00084608093B1008091B00081608093B0005C
:10B7E00080919100826080939100809191008160AE
:10B7F000809391008091900081608093900080916F
:10B80000A10082608093A1008091A100816080935B
:10B81000A1008091A00081608093A000809121010F
:10B8200082608093210180912101816080932101B8
:10B830008091200181608093200180917A00846052
:10B8400080937A0080917A00826080937A00809160
:10B850007A008E7F80937A0080917A00806880934E
:10B860007A001092C1000E940153A3E02A2E312CCD
:10B8700080913C07882309F438C210923C07D0918C
:10B880003B07D13009F44FC258F0D23011F40C9478
:10B89000B365D33011F40C94886710923B0723C230
:10B8A00080913A07823011F40E94A6410E94E11F64
:10B8B0000E94211B809136079091370782309105B5
:10B8C00009F4D6C0A0F5009709F457C0019709F410
:10B8D00092C080912507823061F480912807909171
:10B8E0002907813C9A4D28F0C1E080911E07811103
:10B8F00001C0C0E080911C0790911D078F359640D4
:10B9000008F031C1C11147C180911B07811143C1AA
:10B910008091160710921A0791E0909326071092D3
:10B9200017078B7780931607109213075CC183303B
:10B93000910509F4D1C0049761F680912807909190
:10B940002907883538E9930788F430923707209221
:10B950003607873E9B4150F480911F079091200746
:10B96000892B21F4109237071092360781E08093DB
:10B9700027071092260784E067C08091330782FD75
:10B980000BC020912E0730912F0780912C079091AA
:10B990002D078217930730F421E030E0309337070A
:10B9A0002093360780912A0790912B07813E3EE233
:10B9B000930780F0309237072092360781E080931A
:10B9C000270790913407911102C0809326071092A7
:10B9D00025077FCF873E9B4188F78091280790916C
:10B9E00029078932934250F362E070E07093370781
:10B9F00060933607E3CF8091330783FD0BC020911E
:10BA00002C0730912D0780912E0790912F078217D8
:10BA1000930720F4109237071092360780912A0777
:10BA200090912B07813E7EE2970788F0309237078E
:10BA30002092360781E08093270790913407911177
:10BA400002C08093260781E08093250742CF873E7E
:10BA50009B4180F780912807909129078932934272
:10BA600048F322E030E03093370720933607E2CFE7
:10BA7000809128079091290740912307509124072E
:10BA800020912107309122074217530778F4209123
:10BA90002A0730912B07213E4EE2340738F0281751
:10BAA000390788F03092370720923607873E9B414E
:10BAB00050F48091330782FF0AC061E070E0709318
:10BAC0003707609336071092270782E0BDCF1092A8
:10BAD000370710923607F7CF20912A0730912B07AE
:10BAE00040912807509129078091210790912207C2
:10BAF0008C599F4F609123077091240786179707F1
:10BB000030F0C90188579C4E8417950730F482E0C5
:10BB100090E0909337078093360741345C4930F0CA
:10BB2000E4E0F0E0F0933707E0933607273E3B412F
:10BB300050F48091330782FF11C021E030E0309350
:10BB400037072093360781E08093270790913407C9
:10BB5000911102C08093260783E076CF10923707B9
:10BB600010923607F0CF8CE10E94670720911007F2
:10BB700030911107892B09F0BBC081E08093120737
:10BB80002F5F3F4F309311072093100780911207CA
:10BB9000882309F4B7CE51E050931A078091180713
:10BBA0009091190740911607009709F4ACC02091B5
:10BBB0001407309115072817390708F4B0C0809191
:10BBC00033078C708C3009F4AAC0809113078A3433
:10BBD00008F099C08F5F80931307509326074B7F1F
:10BBE0004068409316078091260761E0811101C0EB
:10BBF00060E087E10E9490078091350784FD1092F4
:10BC000027078091300784FD10922707809127072E
:10BC100060E0811101C061E088E10E9490070E940C
:10BC2000DB1C80910F07813041F5D091FD068D2FEF
:10BC300090E09093FC068093FB06C091FE06CC2317
:10BC400069F06091FF0670E0762F6627809100070B
:10BC5000680F711D8D2F0E948814CFEF81E08093B3
:10BC6000FA068D2F0E94A0129093F9068093F80691
:10BC700010920F07C1110E9453270E94DB1C809174
:10BC8000F706813069F5C091E9068C2F0C2E000C67
:10BC9000990B9093E8068093E7068091EA06D0E03E
:10BCA00018167CF46091EB06062E000C770B762FAD
:10BCB00066278091EC06680F711D8C2F0E948814F6
:10BCC000DFEF8FEF8093E6068C2F0E94A0129093F7
:10BCD000E5068093E4061092F706D1110E945327DF
:10BCE00081E080933B070E94DB1C0E948312C0CD41
:10BCF0002A3F310508F444CF109212071092110721
:10BD00001092100743CF10922607809117078A3FA1
:10BD100018F48F5F809317074F77446062CF81E0FC
:10BD2000809326075CCF0E94E11F0E94211B909107
:10BD3000030180911E0790FF98C0877F80931E07A4
:10BD40009091030180911E0791FF91C08B7F80939A
:10BD50001E079091030180911E0792FF8AC08F7D7C
:10BD600080931E079091030180911E0793FF83C06B
:10BD70008F7E80931E079091030180911E0794FF90
:10BD80007CC08D7F80931E079091030180911E07D8
:10BD900095FF75C08E7F80931E078091E20690917B
:10BDA000E306009709F0E4C08091E1068111DBC051
:10BDB00080912F02909130028F3E72E0970708F435
:10BDC000CCC01092E00620912C0730912D0728322C
:10BDD00083E2380708F055C08FEF8093E006309378
:10BDE0002E0220932D021092DF0680912E07909153
:10BDF0002F078832F3E29F0708F055C04FEF4093BA
:10BE0000DF0690932C0280932B02409133075091D0
:10BE1000E006552309F481C05091DF06552309F44B
:10BE20007CC0283273E2370710F00C94A16D242FE8
:10BE300024602093330710922A028832E3E29E079F
:10BE400010F00C94C86D4C60409333071092290297
:10BE500090912902809133078F7B911101C09CE062
:10BE600090932802809333075BC0886067CF84601B
:10BE70006ECF806275CF80617CCF826083CF81601E
:10BE80008ACF80912D0290912E022817390730F425
:10BE9000821B930B409708F49FCFA1CFF901E81BB9
:10BEA000F90BCF01F7CF40912B0250912C02841750
:10BEB000950738F4481B590B4031510508F49ECFC3
:10BEC000A0CFBC01641B750BAB01F6CF883273E2C7
:10BED000970710F00C94C86D90912A02992309F4E9
:10BEE000B7CF209129028091330721110BC0909385
:10BEF00028028F7BB7CF2CE0209329020C94D56DBC
:10BF000098E1EFCF291799F3921720F49093280224
:10BF10008064A8CF20932802FBCF4064409333076E
:10BF20009091280290933907E091DC06ED3008F0FB
:10BF30007EC2F0E08827E056F04A8F4F0C940F73D2
:10BF40004F607F609E60BF601B616B618E61AF61FF
:10BF5000D461F8618E62B562D86201969093300226
:10BF600080932F02DDCF1092300210922F02D8CF93
:10BF70008130910539F58CE0809328028FEF809312
:10BF8000E0068093DF0640912C0750912D07483240
:10BF9000F3E25F0738F480913307846080933307BE
:10BFA00010922A0220912E0730912F07283263E247
:10BFB000360758F5809133078860809333071092D5
:10BFC000290223C08230910509F045C088E18093A1
:10BFD00028028FEF8093E0068093DF0640912C07C4
:10BFE00050912D07403576E4570738F48091330798
:10BFF00084608093330710922A0220912E0730919B
:10C000002F07203586E43807A8F28091DD0690914D
:10C01000DE0688579C4E8417950728F44091330715
:10C020004B7F409333078217930728F4809133079F
:10C03000877F8093330780912A02811105C0809108
:10C0400033078F7B8093330780912902811168CF5A
:10C05000809133074ECF039709F062CF80E380933E
:10C0600028028FEF8093E0068093DF0640912C0733
:10C0700050912D07403A9CE8590738F480913307D6
:10C0800084608093330710922A0220912E0730910A
:10C090002F07203AECE83E0708F0B7CF8BCF10927D
:10C0A000CA0687E08093CB068091230790912407EE
:10C0B0009093CC068093CD068091C8069091C906D6
:10C0C0009093CE068093CF06809126078093D0066A
:10C0D0008091C6069091C7069093D1068093D206B0
:10C0E0008AE08093D3068DE08093D4064BE050E045
:10C0F0006AEC76E08DE098E00E94F00498C181E05F
:10C100008093CA0687E08093CB06809128079091A0
:10C1100029079093CC068093CD0680911F079091BC
:10C1200020079093CE068093CF06809125078093B9
:10C13000D0068091C4069091C506CECF82E0809350
:10C14000CA0687E08093CB0680912A0790912B073F
:10C150009093CC068093CD06809127078093CE06DE
:10C160008091C2069091C3060E9461189093CF06F9
:10C170008093D0068091C0069091C106ADCF83E038
:10C180008093CA0688E08093CB068091BE0690918A
:10C19000BF060E9461189093CC068093CD068091D3
:10C1A000BC069091BD068115F4E09F0710F08FEF5B
:10C1B00093E048E1489F9001499F300D112485E9A3
:10C1C0009FE7821B930B9093CE068093CF0620911E
:10C1D000BA063091BB062E3643E0340710F02DE648
:10C1E00033E0ADECB5E00E943D7029E43FED43E162
:10C1F00050E0261B370B480B590BDA01C90155E0FB
:10C20000B695A795979587955A95D1F79093D006AF
:10C210008093D1068091B8069091B9069093D2068A
:10C220008093D3068AE08093D4068DE08093D50670
:10C230004CE050E05DCF84E08093CA0688E08093B4
:10C24000CB068091B6069091B7060E946118909334
:10C25000CC068093CD068091B4069091B5068115E9
:10C2600034E0930710F08FEF93E048E1489F90018E
:10C27000499F300D112485E99FE7821B930B909312
:10C28000CE068093CF062091B2063091B3062E36AB
:10C2900043E0340710F02DE633E0ADECB5E00E944A
:10C2A0003D7029E43FED43E150E0261B370B480B7E
:10C2B000590BDA01C90145E0B695A7959795879581
:10C2C0004A95D1F79093D0068093D1068091B0061D
:10C2D0009091B106A3CF85E08093CA0688E0809351
:10C2E000CB0680912C0790912D079093CC068093DC
:10C2F000CD0680912E0790912F079093CE068093C4
:10C30000CF068091AE069091AF069093D0068093B1
:10C31000D1068091AC069091AD0680CF86E08093E7
:10C32000CA0688E08093CB0680911E078093CC06D6
:10C330009093CD068091AA069091AB069093CE067D
:10C340008093CF068091A8069091A9069093D0067D
:10C350008093D1068091A6069091A7065FCF87E0D3
:10C360008093CA0688E08093CB068091DD06909189
:10C37000DE069093CC068093CD068091A406909122
:10C38000A5069093CE068093CF068091A206909149
:10C39000A3069093D0068093D1068091E106809306
:10C3A000D2068091A1063CCF88E08093CA06809394
:10C3B000CB06809130078093CC0680913107809323
:10C3C000CD06809132078093CE068091330780930B
:10C3D000CF06809134078093D006809135078093F3
:10C3E000D1068091A0068093D2068091160718CFBF
:10C3F0008091FB068093CA0682E08093CB068091F1
:10C40000F8069091F9069093CC068093CD068AE0C9
:10C410008093CE068DE08093CF0646E050E06AEC34
:10C4200076E08DE098E00E94F0041092FA06809188
:10C43000DC068F5F8093DC06893039F48091FA0640
:10C44000811103C08AE08093DC068091DC068A308B
:10C4500039F480918906811103C08BE08093DC065A
:10C460008091DC068B3039F480918806811103C0FD
:10C470008CE08093DC068091DC068C3019F48DE032
:10C480008093DC068091DC068D3010F01092DC0683
:10C49000809186069091870689393AE3930708F4DC
:10C4A000BAC01092850680918306909184068F3FD2
:10C4B000980729F0019690938406809383068091D3
:10C4C0008306909184068A3F9105C1F0883E53E02F
:10C4D0009507A1F0803D67E0960781F0803A7FE004
:10C4E000970761F08034EFE19E0741F08038FEE36A
:10C4F0009F0721F081159D4709F093C060E084E516
:10C500000E94900761E070E080E090E00E943508B2
:10C5100061E084E50E94900782E0E3CB8AE08093AB
:10C52000CA0698E09093CB0690919E0620919F06B4
:10C530002093CC069093CD0690919C0620919D0669
:10C540002093CE069093CF0690919A0620919B0659
:10C550002093D0069093D106909199069093D2069D
:10C56000909198069093D3065ECE8BE08093CA0696
:10C5700085E08093CB0680919606909197069093E4
:10C58000CC068093CD06809195068093CE0680914F
:10C5900094068093CF06809193068093D0068AE01C
:10C5A0008093D1068DE08093D20649E050E0A0CD83
:10C5B0008CE08093CA0689E08093CB068091920636
:10C5C0008093CC0680919006909191069093CD0631
:10C5D0008093CE0680918E0690918F069093CF0621
:10C5E0008093D00680918C0690918D069093D10611
:10C5F0008093D20680918A0690918B069093D30601
:10C600008093D4068AE08093D5068DE08093D60689
:10C610004DE050E06DCD019690938706809386069D
:10C6200042CFE0912702ED3008F0EDC1F0E088271D
:10C63000E35EFC498F4F0C940F732A634F6388634A
:10C64000A9630564556478649B64C064E4643665DA
:10C650005D6580651092690687E080936A06809127
:10C6600023079091240790936B0680936C0680912A
:10C67000C8069091C90690936D0680936E068091CE
:10C68000260780936F068091C6069091C706909307
:10C690007006809371068AE0809372062DC081E057
:10C6A0008093690687E080936A06809128079091BD
:10C6B000290790936B0680936C0680911F079091D9
:10C6C000200790936D0680936E06809125078093D6
:10C6D0006F068091C4069091C5064AE0489F90017C
:10C6E000499F300D112430937006849F802D1124B2
:10C6F00080937106409372068DE0809373064BE041
:10C7000050E069E676E080E797E00E94F0047BC1A4
:10C7100082E08093690687E080936A0680912A0709
:10C7200090912B0790936B0680936C06809127075E
:10C7300080936D068091C2069091C3060E94611895
:10C7400090936E0680936F068091C0069091C1060B
:10C750009ECF83E08093690688E080936A0680918B
:10C76000BE069091BF060E94611890936B0680935D
:10C770006C068091BC069091BD06811534E093074C
:10C7800010F08FEF93E048E1489F9001499F300DF2
:10C79000112485E99FE7821B930B90936D0680938C
:10C7A0006E062091BA063091BB062E3643E0340760
:10C7B00010F02DE633E0ADECB5E00E943D7029E4C9
:10C7C0003FED43E150E0261B370B480B590BDA01D4
:10C7D000C90135E0B695A795979587953A95D1F714
:10C7E00090936F06809370068091B8069091B90679
:10C7F00090937106809372068AE0809373068DE0B1
:10C80000809374064CE050E07CCF84E0809369060E
:10C8100088E080936A068091B6069091B7060E94E0
:10C82000611890936B0680936C068091B40690918A
:10C83000B506811534E0930710F08FEF93E048E1DF
:10C84000489F9001499F300D112485E99FE7821B85
:10C85000930B90936D0680936E062091B2063091F3
:10C86000B3062E3643E0340710F02DE633E0ADEC8E
:10C87000B5E00E943D7029E43FED43E150E0261B06
:10C88000370B480B590BDA01C90125E0B695A7957E
:10C89000979587952A95D1F790936F0680937006A8
:10C8A0008091B0069091B106A3CF85E08093690690
:10C8B00088E080936A0680912C0790912D079093D1
:10C8C0006B0680936C0680912E0790912F079093B2
:10C8D0006D0680936E068091AE069091AF069093A0
:10C8E0006F06809370068091AC069091AD0680CF64
:10C8F00086E08093690688E080936A0680911E072F
:10C9000080936B068091390780936C068091AA060C
:10C910009091AB0690936D0680936E068091A80669
:10C920009091A90690936F06809370068091A60659
:10C930009091A7065DCF87E08093690688E0809399
:10C940006A068091DD069091DE0690936B068093D7
:10C950006C068091A4069091A50690936D06809335
:10C960006E068091A2069091A30690936F06809325
:10C9700070068091E106809371068091A1063ACFFE
:10C9800088E08093690680936A06809130078093DF
:10C990006B068091310780936C06809132078093FB
:10C9A0006D068091330780936E06809134078093E3
:10C9B0006F0680913507809370068091A006809362
:10C9C00071068091160716CF8091E706809369065D
:10C9D00082E080936A068091E4069091E506909348
:10C9E0006B0680936C068AE080936D068DE08093E1
:10C9F0006E0646E050E069E676E080E797E00E9448
:10CA0000F0041092E606809127028F5F8093270240
:10CA1000893039F48091E606811103C08AE0809361
:10CA20002702809127028A3039F48091890681118A
:10CA300003C08BE080932702809127028B3039F46A
:10CA400080918806811103C08CE080932702809139
:10CA500027028C3019F48DE0809327028091270201
:10CA60008D3008F459CD1092270256CD8AE080937C
:10CA7000690698E090936A0690919E0620919F0621
:10CA800020936B0690936C0690919C0620919D06D6
:10CA900020936D0690936E0690919A0620919B06C6
:10CAA00020936F069093700690919906909371066B
:10CAB0009091980690937206A0CE8BE080936906C1
:10CAC00085E080936A0680919606909197069093F0
:10CAD0006B0680936C068091950680936D0680911D
:10CAE000940680936E068091930680936F068AE089
:10CAF000809370068DE08093710649E050E001CE8E
:10CB00008CE08093690689E080936A0680919206A2
:10CB100080936B06809190069091910690936C069D
:10CB200080936D0680918E0690918F0690936E068D
:10CB300080936F0680918C0690918D06909370067D
:10CB40008093710680918A0690918B06909372066D
:10CB5000809373068AE0809374068DE08093750657
:10CB60004DE050E0CECD61E08BE10E949007C09196
:10CB70003A07C11177C1109168061F5F10936806CC
:10CB800080916706823009F495C028F4882369F003
:10CB90000E94321226C0833009F409C18630C1F7E1
:10CBA0000E943212109267061CC00E943212193085
:10CBB00020F010926806D09367068091880688233B
:10CBC00081F08091630690916406A0916506B09112
:10CBD00066068B349105A105B10508F45FC010927B
:10CBE00088060E94E11F0E94211B8091E106882394
:10CBF00009F469C1E0912406F09125068091AA0606
:10CC00009091AB06E81BF90B8091C4069091C50684
:10CC10006AE070E00E94FB722091220630912306A8
:10CC2000261B370B40911D0650911E06BF01660F53
:10CC3000771F660F771FF5FD02C037FF19C180917E
:10CC40002106811120C18091AE069091AF06E0913E
:10CC5000AC06F091AD06E80FF91F6F01F12CE12C45
:10CC600081E080932106621773070CF03CC180912C
:10CC70001C068B3F08F40EC1CB01770FAA0BBB0B30
:10CC80008C0D9D1DAE1DBF1D10921C066C017D01FB
:10CC9000F7FE03C1C12CD12C7601FFC00196A11D66
:10CCA000B11D8093630690936406A0936506B093CC
:10CCB000660697CF10924F0681E08093500680E180
:10CCC00080935106809352068091280790912907FE
:10CCD00064E670E00E94FB72709353066093540602
:10CCE00080913307282F287082FD0FC0211113C0B7
:10CCF00020912E0730912F0780912C0790912D07BE
:10CD00002817390760F4C9010AC080912E07909155
:10CD10002F07222321F080912C0790912D079093CB
:10CD20005506809356068091AE069091AF062091ED
:10CD3000AC063091AD06820F931F909357068093F7
:10CD400058061092590610925A068091AA069091A0
:10CD5000AB0690935B0680935C06809123079091CD
:10CD6000240790935D0680935E0610925F061092F2
:10CD70006006EFE4F6E021E636E090E080E04191E5
:10CD8000840F911D2E173F07D1F790936106809372
:10CD900062060E941D2744E150E06FE476E08CEAD1
:10CDA00098E00E94F00486E0809367061ACF0E9404
:10CDB000321280914E0690E0BC0162507109FB0175
:10CDC000EA5DF94F408150E0542F44278B5D994F25
:10CDD000FC018081480F511D30E020E08C2F90E055
:10CDE0008617970744F48A5D994FFC018081280FCC
:10CDF000311DCF5FF3CF4217530709F0D3CE809197
:10CE00002706823109F0CECE809126068111CACE46
:10CE100080912806803109F0C5CE80912A0690E0E5
:10CE2000982F882720912B06820F911D90939706AB
:10CE30008093960680912C068093950680912D060E
:10CE40008093940680912E068093930681E08093D0
:10CE5000880610926306109264061092650610927E
:10CE60006606A0CEC23009F0BCCE0E94A641B9CE63
:10CE700080911E07807311F4109221068091210683
:10CE80006A01882321F0C0901F06D0902006F12C63
:10CE9000E12CE9CE8F5F80931C0670E060E0C41641
:10CEA000D506E606F7060CF4A60180911B0688233A
:10CEB00051F14938F3E15F0730F188E893E190934D
:10CEC000200680931F060E94DB2181110E94284AC0
:10CED0000E94DB1C83E080933B0760E08BE10E94B3
:10CEE00090070C94735EC901330FAA0BBB0BC2E011
:10CEF000880F991FAA1FBB1FCA95D1F78C0D9D1DC6
:10CF0000AE1DBF1DC3CE5093200640931F06DBCF3E
:10CF10000E94E11F0E94211B0E94593C80911A0629
:10CF20008F3308F04AC08F5F80931A0680911906EC
:10CF30008F3318F48F5F8093190680912507823014
:10CF400008F45FC081E08093A0062091160630911E
:10CF50001706A7E0B0E00E943D702091C406309112
:10CF6000C5064B015C01820E931EA11CB11CA3E0FF
:10CF7000B694A79497948794AA95D1F7C4019092F8
:10CF8000170680921606209139072C3009F055C0FB
:10CF900020913307422F487022FD36C041113AC01C
:10CFA00040912E0750912F0720912C0730912D078B
:10CFB0004217530798F59A0131C08F3750F48F5FAD
:10CFC00080931A0680911906882309F4B6CF815000
:10CFD000B2CF10921A06209116078091260298E08F
:10CFE000382F322309F0A3C5915009F4A7C5803822
:10CFF00011F0880FF5CF81E0F3CF880F80932602E0
:10D000009CCF1092A006A1CF20912E0730912F0720
:10D01000442321F020912C0730912D074091A00648
:10D02000442309F45EC0413009F40DC11092A006FA
:10D0300050E040E010E000E003C1283121F52091EC
:10D040003307422F487022FD0FC0411115C0C09018
:10D050002C07D0902D0720912E0730912F072C15EB
:10D060003D0570F096010CC020912E0730912F07DE
:10D0700036952795442391F220912C0730912D0766
:10D0800036952795CBCF203349F520913307422F92
:10D09000487022FD0FC0411118C0C0902C07D090DD
:10D0A0002D0720912E0730912F072C153D0588F074
:10D0B00096010FC020912E0730912F0736952795A6
:10D0C00036952795442309F4A9CF20912C07309158
:10D0D0002D073695279536952795A0CF30E020E08F
:10D0E0009DCF80901406909015068216930608F046
:10D0F0009FCFE0911206F0911306A0911906B0E0BF
:10D10000A55CBD4F4C90512C712C612CE217F3079C
:10D1100030F1B12CA12C50E040E0281939094A091E
:10D120005B09ABE3BAE00E9408709F0150E040E069
:10D13000281939094A095B090E94E96FC301B20144
:10D140000E94EB7256E096958795779567955A956C
:10D15000D1F7EB0150E040E010E000E04BC08090E0
:10D160001006909011068216930608F458C0CF015D
:10D17000B0E0A0E06901F12CE12CC81AD90AEA0A52
:10D18000FB0AB12CA12C881A990AAA0ABB0AA5ECA1
:10D19000B5EFA70196010E941670A50194010E94A7
:10D1A000E96F255C354F4F4F5F4FC301B2010E94BD
:10D1B000EB7226E096958795779567952A95D1F736
:10D1C000EB01ABE3BAE0A70196010E940870A5014C
:10D1D00094010E94E96FC301B2010E94EB728B01BE
:10D1E0009C0146E036952795179507954A95D1F706
:10D1F00050E040E080911806883009F485C108F0BD
:10D20000B0C0813009F4C2C008F4C6C0823009F44D
:10D210006DC1843009F46EC110921806BDC0ABE335
:10D22000BAE0A30192010E9408708B019C0186E084
:10D2300036952795179507958A95D1F750E040E0E8
:10D24000D0E0C0E0D7CF893522E0920720F5A6E0F4
:10D25000B4E0A50194010E94087028E532E040E0A6
:10D2600050E00E94E96F2C5E3F4F4F4F5F4FE90146
:10D27000A6E0B5E0A50194010E94087028E532E01F
:10D2800040E050E00E94E96FBA01A901475E5F4F9C
:10D290006F4F7F4F61CF813B34E0930750F548E5F6
:10D2A000841A42E0940AA108B108A6EEBBEFA501DA
:10D2B00094010E94167028E532E040E050E00E94A0
:10D2C000E96F265E3B4F4F4F5F4FE901ACE1B5E0A0
:10D2D000A50194010E94087028E532E040E050E08A
:10D2E0000E94E96FBA01A901415E5A4F6F4F7F4F0B
:10D2F00033CF813659E09507A0F4A5019401205B56
:10D30000344041095109ABE3BAE00E94087020EBB8
:10D3100034E040E050E00E94E96F89014BE35AE0BD
:10D320008FCF4BE35AE00BE31AE0CBE3DAE0813C2A
:10D33000924108F05FCFA501940120563940410980
:10D340005109ABE3BAE00E94087020E639E040E002
:10D3500050E00E94E96FE9014BE35AE00BE31AE069
:10D3600049CF803209F4D6C038F4803109F054CF67
:10D3700080911A068C7ECBC0803409F4DBC08038E3
:10D3800009F04ACF80911A068670B7C080911A06BC
:10D390008C7F882309F4D2C0E0910E06F0910F062D
:10D3A0009E01DF010E943D70472E582E692E772482
:10D3B0009F01D8010E943D70872E982EA92EBB2474
:10D3C000E401DA010E943D70C72ED82EE92EFF2419
:10D3D0008601809180004114510409F0B6C0877F16
:10D3E0008093800060E08DE00E9490078091800033
:10D3F000CD2B09F0B2C08F7D8093800060E08CE07F
:10D400000E94900780918000012B09F0AEC08F77B9
:10D410008093800060E08BE00E949007C091AE0690
:10D42000D091AF06E091AC06F091AD068E010E0FE3
:10D430001F1F2091DD063091DE0648EEE42E43E00A
:10D44000F42EC801B7010E94FB726B01C901B7013C
:10D450000E94FB72C69EA001C79E500DD69E500D25
:10D46000112480911D0690911E068053984F8017BD
:10D47000910708F082C080910D068D3718F48F5FF8
:10D4800080930D0680910D068D3728F0809130072E
:10D4900081608093300780910B0690910C06845D2B
:10D4A0009E4F8417950708F06BC080910A068D3750
:10D4B00018F48F5F80930A0680910A068D3728F052
:10D4C000809130078062809330078091300790917F
:10D4D00025029E3109F4F2C008F055C09A3009F4D3
:10D4E00082C0943109F4D9C08AE0E5C080911A065F
:10D4F000807F4FCF80911A06807F81114DCF4BE303
:10D500005AE010E000E01EC080911A068C7F88234C
:10D5100051F042CF80911A06982F9C7E21F08C7F8B
:10D52000803209F039CF50E040E010E000E0CBE37A
:10D53000DAE032CF80911A068C7CE9CF50E040E0EF
:10D540000BE31AE0D0E0C0E027CF88608093800032
:10D5500050928D0040928C0049CF80628093800071
:10D5600090928B0080928A004DCF806880938000DB
:10D57000D0928900C092880051CF10920D0682CFC0
:10D5800010920A0699CF983209F49CC0923309F0A0
:10D59000ABCF40912C0750912D0740575E4F42175B
:10D5A000530708F49DC040912E0750912F07405714
:10D5B0005E4F4217530708F493C0909109069F5F8E
:10D5C00090930906909109069A3F40F08D7F8093D1
:10D5D0003007109209068AE0809325028091300777
:10D5E00081FD38C081CF8D7F8093300710921B065C
:10D5F00080912C0790912D0780579E4F821793079B
:10D6000018F4C93ED34060F480912E0790912F0703
:10D6100080579E4F8217930778F5E93EF34060F1FB
:10D62000809109068F5F80930906809108068A3FE2
:10D6300010F010920706809109068D3758F08091FE
:10D6400007068A3018F188E28093250210920906B5
:10D650001092080690913907809135079C3009F0A7
:10D6600042C0909125072091050630910606923020
:10D6700008F443C08B7F52C01092090680910806BF
:10D680008A3F98F68F5F80930806CFCF94E19093FE
:10D6900025028F5F80930706D9CF82608093300781
:10D6A000809109068F5F823318F480930906D2CFE8
:10D6B000109209068EE180932502CCCF8D7F809356
:10D6C000300712CF8260809330078FEF80931B0664
:10D6D00010920706109208061092090682E3EBCF1B
:10D6E000109209066FCF9831D9F4909125079230A6
:10D6F00008F6209103063091040640912C075091C2
:10D700002D072417350708F4B5CF40912E07509107
:10D710002F072417350708F4ADCF846080933507B1
:10D7200040912A0750912B078091010690910206A3
:10D730008417950708F019C1809100068D3718F4F9
:10D740008F5F80930006809100068D3728F08091CE
:10D750003507806180933507483E9BE1590728F4DF
:10D76000809135078F7E80933507809123079091B4
:10D770002407209127072111FBC060912807709191
:10D7800029072091FE053091FF052617370708F07D
:10D79000EFC0009709F4ECC02091FC053091FD0525
:10D7A000243EE7E53E0730F42F5F3F4F3093FD0501
:10D7B0002093FC052091FC053091FD05243E374562
:10D7C00028F020913407216020933407892B29F415
:10D7D000809134078E7F809334078091AA069091C0
:10D7E000AB0620912406309125062817390750F4FE
:10D7F0006091160770913407726070933407686007
:10D80000609316076091FA057091FB05860F971FCC
:10D810002817390750F080911607909134079D7FA3
:10D8200090933407877F809316078091F805909135
:10D83000F9052091F6053091F705E091320760E097
:10D8400078E0681B790B2617370728F0985F821756
:10D85000930708F092C0E260E09332078091F405EC
:10D860009091F505E091320760E078E0681B790B54
:10D870002617370728F0985F8217930708F07FC0B4
:10D88000E160E0933207483E5B4128F48091300725
:10D890008F7E8093300790913407809116072091F6
:10D8A000350724FD02C090FF6CC08062809316078C
:10D8B000809116072091300721110DC0209131076A
:10D8C000211109C020913207211105C02091330791
:10D8D000207509F458C0806480931607809116075C
:10D8E00092FF53C0806180931607C091F305C13049
:10D8F00009F488C008F44BC0C23009F4BEC080915E
:10D90000A6069091A7062091A8063091A906821735
:10D91000930708F4F3C0821B930B9093F705809351
:10D92000F605C23008F0EFC0CF5FC093F3058091D9
:10D930003807813011F00C944D5C0E94DB1C809103
:10D94000F205813011F00C944D5C8091E005282F98
:10D9500030E03093DF052093DE059091E1059111D1
:10D96000D5C01092F2050C944D5C10920006EBCEDF
:10D970001092FD051092FC051DCFED7F6DCFEE7F5F
:10D9800080CF8F7D93CF8F7BA7CF8F7EACCF84E46A
:10D990000E94071B582F492F20911F02309120020F
:10D9A000AFE1B0E00E943D708B019C01852F942F68
:10D9B000811540E1940710F08FEF9FE0B0E0A0E008
:10D9C000D3E0880F991FAA1FBB1FDA95D1F7800FEC
:10D9D000911FA21FB31F8C019D0185E036952795ED
:10D9E000179507958A95D1F71093200200931F028F
:10D9F00093E0169507959A95E1F71093A906009381
:10DA0000A8067DCF85E40E94071B582F492F20913F
:10DA1000210230912202AFE1B0E00E943D708B0103
:10DA20009C01852F942F811550E1950710F08FEF01
:10DA30009FE0B0E0A0E0F3E0880F991FAA1FBB1F92
:10DA4000FA95D1F7800F911FA21FB31F8C019D0182
:10DA5000A5E03695279517950795AA95D1F71093C8
:10DA6000220200932102B3E016950795BA95E1F7DB
:10DA70001093A7060093A60642CF87E30E94071BD8
:10DA8000582F492F2091230230912402A7E0B0E0C3
:10DA90000E943D708B019C01852F942F811560E1C0
:10DAA000960710F08FEF9FE0B0E0A0E043E0880F12
:10DAB000991FAA1FBB1F4A95D1F7800F911FA21F64
:10DAC000B31F9C01AD0163E05695479537952795A7
:10DAD0006A95D1F73093240220932302ADE7B0E09A
:10DAE0000E940870ECE09695879577956795EA9582
:10DAF000D1F77093AB066093AA0601CF1092F70599
:10DB00001092F6050ECF1092F30511CF6091E20549
:10DB100070E0762F66279091E305690F711D0E94D2
:10DB200088141092F2050E9453270C944D5C809348
:10DB30001806803809F061CA81E060CA10921806A0
:10DB4000FBCF883273E2970728F44860409333078D
:10DB500010922902409133074B7F40933307A9016C
:10DB60004852534249355B4118F44CE040932A0235
:10DB700020553644213B364310F00C94665F28E173
:10DB800020932A02883253E2950710F40C94805FA8
:10DB900020913307277F209333079C01285233427B
:10DBA00029353B4110F40C947B5F80559644813BB2
:10DBB000964310F00C946C5F88E1809329020C94DA
:10DBC0006C5F8F929F92AF92BF92CF92DF92EF9253
:10DBD000FF92CF93DF93EC01688179818A819B81E9
:10DBE000611571058105910521F464E279ED8BE5FC
:10DBF00097E02DE133EF41E050E00E94E96F4901E9
:10DC00005A019B01AC01A7EAB1E40E9408706B01C4
:10DC10007C01ACEEB4EFA50194010E941670C60E13
:10DC2000D71EE81EF91EF7FE06C081E0C81AD1080B
:10DC3000E10880E8F80AC882D982EA82FB82C7013B
:10DC4000B6019F77DF91CF91FF90EF90DF90CF905B
:10DC5000BF90AF909F908F9008958F929F92AF92B8
:10DC6000BF92CF92DF92EF92FF926091310270915A
:10DC70003202809133029091340261157105810561
:10DC8000910521F464E279ED8BE597E02DE133EF26
:10DC900041E050E00E94E96F49015A019B01AC014B
:10DCA000A7EAB1E40E9408706B017C01ACEEB4EF0E
:10DCB000A50194010E941670C60ED71EE81EF91E1B
:10DCC000F7FE06C081E0C81AD108E10880E8F80A2A
:10DCD000C0923102D0923202E0923302F0923402CA
:10DCE000C701B6019F77FF90EF90DF90CF90BF9074
:10DCF000AF909F908F90089560933102709332029D
:10DD000080933302909334020895BB27FB0155277B
:10DD1000AA27880F991FAA1FA41710F0A41B839588
:10DD20005051B9F7A05DAA3308F0A95DA1930097FF
:10DD300079F7B111B1931192CB010C949F6EDC0174
:10DD4000FC01672F71917723E1F7329704C07C9132
:10DD50006D9370836291AE17BF07C8F308950E9458
:10DD6000F16E08F481E00895E89409C097FB3EF451
:10DD700090958095709561957F4F8F4F9F4F992318
:10DD8000A9F0F92F96E9BB279395F6958795779596
:10DD90006795B795F111F8CFFAF4BB0F11F460FF56
:10DDA0001BC06F5F7F4F8F4F9F4F16C0882311F0AE
:10DDB00096E911C0772321F09EE8872F762F05C0C2
:10DDC000662371F096E8862F70E060E02AF09A955D
:10DDD000660F771F881FDAF7880F9695879597F952
:10DDE0000895990F0008550FAA0BE0E8FEEF1616EC
:10DDF0001706E807F907C0F012161306E407F5073F
:10DE000098F0621B730B840B950B39F40A2661F0B2
:10DE1000232B242B252B21F408950A2609F4A14055
:10DE2000A6958FEF811D811D08950E94286F0C9487
:10DE3000996F0E948B6F38F00E94926F20F09523AB
:10DE400011F00C94826F0C94886F11240C94CD6F98
:10DE50000E94AA6F70F3959FC1F3950F50E0551F74
:10DE6000629FF001729FBB27F00DB11D639FAA272F
:10DE7000F00DB11DAA1F649F6627B00DA11D661F7E
:10DE8000829F2227B00DA11D621F739FB00DA11D9F
:10DE9000621F839FA00D611D221F749F3327A00D59
:10DEA000611D231F849F600D211D822F762F6A2FF5
:10DEB00011249F5750409AF0F1F088234AF0EE0F5A
:10DEC000FF1FBB1F661F771F881F91505040A9F787
:10DED0009E3F510580F00C94826F0C94CD6F5F3F94
:10DEE000E4F3983ED4F3869577956795B795F795C3
:10DEF000E7959F5FC1F7FE2B880F911D969587953B
:10DF000097F9089597F99F6780E870E060E00895B9
:10DF10009FEF80EC089500240A9416161706180641
:10DF20000906089500240A9412161306140605061D
:10DF30000895092E0394000C11F4882352F0BB0FAE
:10DF400040F4BF2B11F460FF04C06F5F7F4F8F4F11
:10DF50009F4F089557FD9058440F551F59F05F3F4C
:10DF600071F04795880F97FB991F61F09F3F79F0FB
:10DF700087950895121613061406551FF2CF46957D
:10DF8000F1DF08C0161617061806991FF1CF8695FF
:10DF90007105610508940895E894BB2766277727E3
:10DFA000CB0197F90895F999FECF92BD81BDF89AFA
:10DFB000992780B50895262FF999FECF1FBA92BDF3
:10DFC00081BD20BD0FB6F894FA9AF99A0FBE01965A
:10DFD0000895052E97FB1EF400940E94007057FDD3
:10DFE00007D00E941B7007FC03D04EF40C94007005
:10DFF00050954095309521953F4F4F4F5F4F089575
:10E0000090958095709561957F4F8F4F9F4F0895A4
:10E010000E943D70A59F900DB49F900DA49F800D10
:10E02000911D11240895B7FF0C9408700E94087088
:10E03000821B930B0895A1E21A2EAA1BBB1BFD01A4
:10E040000DC0AA1FBB1FEE1FFF1FA217B307E407D7
:10E05000F50720F0A21BB30BE40BF50B661F771F2F
:10E06000881F991F1A9469F760957095809590950F
:10E070009B01AC01BD01CF010895A29FB001B39FE8
:10E08000C001A39F700D811D1124911DB29F700DC1
:10E09000811D1124911D08955058BB27AA270E9465
:10E0A00064700C94996F0E948B6F38F00E94926F8D
:10E0B00020F039F49F3F19F426F40C94886F0EF485
:10E0C000E095E7FB0C94826FE92F0E94AA6F58F34A
:10E0D000BA17620773078407950720F079F4A6F54D
:10E0E0000C94CC6F0EF4E0950B2EBA2FA02D0B01E3
:10E0F000B90190010C01CA01A0011124FF27591B8D
:10E1000099F0593F50F4503E68F11A16F040A22F92
:10E11000232F342F4427585FF3CF46953795279503
:10E12000A795F0405395C9F77EF41F16BA0B620B02
:10E13000730B840BBAF09150A1F0FF0FBB1F661F49
:10E14000771F881FC2F70EC0BA0F621F731F841F8C
:10E1500048F4879577956795B795F7959E3F08F0B2
:10E16000B0CF9395880F08F09927EE0F9795879574
:10E1700008950E94CD700C94996F0E94926F58F090
:10E180000E948B6F40F029F45F3F29F00C94826F5E
:10E1900051110C94CD6F0C94886F0E94AA6F68F394
:10E1A0009923B1F3552391F3951B550BBB27AA2750
:10E1B00062177307840738F09F5F5F4F220F331F8A
:10E1C000441FAA1FA9F335D00E2E3AF0E0E832D052
:10E1D00091505040E695001CCAF72BD0FE2F29D055
:10E1E000660F771F881FBB1F261737074807AB0727
:10E1F000B0E809F0BB0B802DBF01FF2793585F4F9C
:10E200003AF09E3F510578F00C94826F0C94CD6FDC
:10E210005F3FE4F3983ED4F3869577956795B7957D
:10E22000F7959F5FC9F7880F911D9695879597F988
:10E230000895E1E0660F771F881FBB1F6217730701
:10E240008407BA0720F0621B730B840BBA0BEE1F16
:10E2500088F7E09508950E9432716894B1110C948A
:10E26000CD6F08950E94B26F88F09F5798F0B92F34
:10E270009927B751B0F0E1F0660F771F881F991FFB
:10E280001AF0BA95C9F714C0B13091F00E94CC6F62
:10E29000B1E008950C94CC6F672F782F8827B85F72
:10E2A00039F0B93FCCF3869577956795B395D9F753
:10E2B0003EF490958095709561957F4F8F4F9F4F5D
:10E2C00008950E94F16E08F48FEF0895FA01EE0FA1
:10E2D000FF1F309621053105A1F16115710561F42B
:10E2E0008038BFE39B0749F168949038810561F05D
:10E2F0008038BFEF9B0741F099234AF5FF3FE105C6
:10E300003105210519F1E8940894E795D901AA236C
:10E3100029F4AB2FBE2FF85FD0F310C0FF5F70F46D
:10E32000A695E0F7F73950F019F0FF3A38F49F77E7
:10E330009F930DD00F9007FC9058089546F00C94D1
:10E34000886F60E070E080E89FE308954FE79F7773
:10E350005F934F933F932F930E9461722F913F9150
:10E360004F915F910E94156F0C94BE7129F416F0C5
:10E370000C94826F0C94CC6F0C94886F0E94B26FD7
:10E38000A8F39638A0F707F80F92E8942BE33AEA3F
:10E3900048EB5FE70E942B6F0F920F920F924DB7E1
:10E3A0005EB70F920E94A972E4EEF0E00E94F07155
:10E3B0004F915F91EF91FF91E595EE1FFF1F49F09F
:10E3C000FE57E0684427EE0F441FFA95E1F74195A8
:10E3D000550B0E9423720F9007FE0C94177208953C
:10E3E000DF93CF931F930F93FF92EF92DF927B0106
:10E3F0008C01689406C0DA2EEF010E94286FFE019E
:10E40000E894A5912591359145915591A6F3EF0199
:10E410000E946470FE019701A801DA9469F7DF9009
:10E42000EF90FF900F911F91CF91DF9108959B0185
:10E43000AC0160E070E080E89FE30C94B9700C944C
:10E44000826F0C94DD720E94B26FD8F39923C9F3E6
:10E45000940F511DA3F39150504094F059F088232C
:10E4600032F0660F771F881F91505040C1F79E3FD2
:10E4700051052CF7880F911D9695879597F908956A
:10E480005F3FACF0983E9CF0BB27869577956795EB
:10E49000B79508F4B1609395C1F7BB0F58F711F425
:10E4A00060FFE8CF6F5F7F4F8F4F9F4FE3CF0C949C
:10E4B000CD6F16F00C94DD720C94886F68940C94F8
:10E4C000826F0E94B26FA8F39923C1F3AEF3DF937A
:10E4D000CF931F930F93FF92C92FDD2788232AF034
:10E4E0002197660F771F881FDAF720E030E040E8B9
:10E4F0005FEB9FE3883920F0803E38F021968F77DC
:10E500000E944D70ECE0F1E004C00E944D70E9E320
:10E51000F1E00E94F0718B01BE01EC01FB2E6F5700
:10E5200071097595771F880B990B0E94B66E28E1CB
:10E5300032E741E35FE30E94286FAF2D9801AE01FF
:10E54000FF900F911F91CF91DF910E9464700C9406
:10E55000996FFA01DC01AA0FBB1F9B01AC01BF57E9
:10E5600028F4222733274427507820C0B75190F44D
:10E57000AB2F0024469537952795011CA395D2F320
:10E58000002071F0220F331F441FB395DAF30ED031
:10E590000C944C7061307105A0E88A07B94630F4DC
:10E5A0009B01AC016627772788279078309621F069
:10E5B000208331834283538308959F3F31F09150EC
:10E5C00020F4879577956795B795880F911D969557
:10E5D000879597F90895DB018F939F930E940870A8
:10E5E000BF91AF91A29F800D911DA39F900DB29FEF
:10E5F000900D11240895AA1BBB1B51E107C0AA1F4F
:10E60000BB1FA617B70710F0A61BB70B881F991FD3
:10E610005A95A9F780959095BC01CD010895EE0F0C
:10E62000FF1F881F8BBF0790F691E02D19940F9361
:10E630001F93CF93DF938230910510F482E090E036
:10E64000E0911D0CF0911E0C30E020E0B0E0A0E065
:10E65000309799F42115310509F44AC0281B390B6C
:10E6600024303105D8F58A819B816115710589F1C6
:10E67000FB0193838283FE0111C04081518102819D
:10E68000138148175907E0F04817590799F4109774
:10E6900061F012960C93129713961C933296CF0149
:10E6A000DF91CF911F910F91089500931D0C10934E
:10E6B0001E0CF4CF2115310551F04217530738F0E5
:10E6C000A901DB019A01BD01DF01F801C1CFEF0112
:10E6D000F9CF90931E0C80931D0CCDCFFE01E20F5D
:10E6E000F31F819391932250310939832883D7CF27
:10E6F00020911B0C30911C0C232B41F420913702EC
:10E700003091380230931C0C20931B0C2091350261
:10E71000309136022115310541F42DB73EB74091B5
:10E72000390250913A02241B350BE0911B0CF091F9
:10E730001C0CE217F307A0F42E1B3F0B2817390718
:10E7400078F0AC014E5F5F4F2417350748F04E0F4D
:10E750005F1F50931C0C40931B0C819391939FCF90
:10E76000F0E0E0E09CCFCF93DF930097E9F0FC016D
:10E77000329713821282A0911D0CB0911E0CED01F4
:10E7800030E020E01097A1F420813181820F931FA7
:10E7900020911B0C30911C0C2817390709F061C01F
:10E7A000F0931C0CE0931B0CDF91CF910895EA01CC
:10E7B000CE17DF07E8F54A815B819E0141155105BF
:10E7C000B1F7E901FB83EA8349915991C40FD51F41
:10E7D000EC17FD0761F4808191810296840F951FEB
:10E7E000E90199838883828193819B838A83F0E006
:10E7F000E0E012968D919C9113970097B9F52D91B9
:10E800003C911197CD010296820F931F20911B0C12
:10E8100030911C0C2817390739F6309751F51092B2
:10E820001E0C10921D0CB0931C0CA0931B0CBCCFA3
:10E83000D383C28340815181840F951FC817D907A4
:10E8400061F44E5F5F4F88819981480F591F518352
:10E8500040838A819B81938382832115310509F04E
:10E86000B0CFF0931E0CE0931D0C9ECFFD01DC0198
:10E87000C0CF13821282D7CF4F925F926F927F9256
:10E880008F929F92AF92BF92CF92DF92EF92FF92C0
:10E890000F931F93CF93DF938C01009799F4CB01D3
:10E8A000DF91CF911F910F91FF90EF90DF90CF906C
:10E8B000BF90AF909F908F907F906F905F904F90A0
:10E8C0000C941773FC01E60FF71F9C0122503109CD
:10E8D000E217F30708F4AEC0D901CD91DC9111978E
:10E8E000C617D70720F1C530D10578F0CE010497BF
:10E8F0008617970750F0C61BD70B2297C193D19369
:10E900006D937C93CF010E94B373C801DF91CF91C7
:10E910001F910F91FF90EF90DF90CF90BF90AF903D
:10E920009F908F907F906F905F904F9008955B01C4
:10E93000AC1ABD0A4C018C0E9D1EA0911D0CB0910D
:10E940001E0C512C412CF12CE12C109731F58091AB
:10E950001B0C90911C0C8815990509F05CC046169B
:10E96000570608F058C08091350290913602009702
:10E9700041F48DB79EB74091390250913A02841B01
:10E98000950BE817F90708F055C0F0931C0CE093BD
:10E990001B0CF90171836083B8CF8D919C91119705
:10E9A00012966C90129713967C901397A815B90540
:10E9B00059F56C0142E0C40ED11CCA14DB0420F1ED
:10E9C000AC014A195B09DA011296159780F0628250
:10E9D000738251834083D9016D937C93E114F104D8
:10E9E00071F0D7011396FC93EE9312978ECF229677
:10E9F0008C0F9D1FF90191838083F301EFCFF0937A
:10EA00001E0CE0931D0C81CF4816590608F42C010A
:10EA10007D01D3019ACFCB010E9417737C0100972F
:10EA200049F0AE01B8010E941D75C8010E94B37380
:10EA300087016BCF10E000E068CFFB01DC0102C072
:10EA400001900D9241505040D8F70895FB01DC0130
:0EEA500001900D920020E1F70895F894FFCF99
:10EA5E000002000200020002000200020002000298
:10EA6E00000200C0FF0000C0FF000200F00501F828
:10EA7E001F0060C8000A01050C0C0C28232823FF78
:10EA8E00FF0100000000001F0C80000202020203C2
:10EA9E00030304040506070708090A0B0D0E0F10E1
:10EAAE001213151618191B1C1E2021232526282982
:10EABE002B2C2E2F31323335363738393A3A3B3C00
:10EACE003C3D3D3E3E3E3F3F3F3F3F00316253C4E3
:10EADE00F5A697B988DBEA7D4C1F2E43722110876D
:10EAEE00B6E5D4FACB98A93E0F5C6D86B7E4D54255
:10EAFE007320113F0E5D6CFBCA99A8C5F4A7960151
:10EB0E003063527C4D1E2FB889DAEB3D0C5F6EF9E7
:10EB1E00C89BAA84B5E6D7407122137E4F1C2DBA2E
:10EB2E008BD8E9C7F6A59403326150BB8AD9E87F2A
:10EB3E004E1D2C02336051C6F7A495F8C99AAB3C12
:10EB4E000D5E6F4170231285B4E7D67A4B1829BE3D
:10EB5E008FDCEDC3F2A1900736655439085B6AFD70
:10EB6E00CC9FAE80B1E2D344752617FCCD9EAF3854
:10EB7E00095A6B4574271681B0E3D2BF8EDDEC7B4C
:10EB8E004A192806376455C2F3A091477625148397
:10EB9E00B2E1D0FECF9CAD3A0B586904356657C032
:10EBAE00F1A293BD8CDFEE79481B2AC1F0A392052A
:10EBBE0034675678491A2BBC8DDEEF82B3E0D1460E
:10EBCE007724153B0A5968FFCE9DAC00000000D596
:10EBDE0005F00436052206670545055905000000B7
:10EBEE00002B12F211E711DC1190113E110D0A00EB
:10EBFE00726573657420332E3038203139206A7572
:10EC0E00696C6C65742032303231006361727465E8
:10EC1E002031322D3234560041542B52454E455739
:10EC2E0000300041542B4E414D4243562D30332D72
:10EC3E000041542B4E414D4543562D30332D00414E
:10EC4E00542B524553455400525334383520706F6F
:10EC5E006D7065206879647261756C697175652077
:10EC6E003936303020627073005253343835206597
:10EC7E006F6C69656E6E6520353736303020627088
:02EC8E00730011
:00000001FF
